:020000040000FA
:10000000021F4E022003FFFFFFFFFF02200BFFFF36
:10001000FFFFFF022013FFFFFFFFFF02201BFFFF78
:10002000FFFFFF022023FFFFFFFFFF02202BFFFF48
:10003000FFFFFF022033FFFFFFFFFF02203BFFFF18
:10004000FFFFFF022043FFFFFFFFFF02204BFFFFE8
:10005000FFFFFF022053FFFFFFFFFF02205BFFFFB8
:10006000FFFFFF022063FFFFFFFFFF02206BFFFF88
:10007000FFFFFF022073FFFFFFFFFF02207BFFFF58
:10008000FFFFFF022083FFFFFFFFFF02208BFFFF28
:10009000FFFF70DFFFFF040000000002000000C847
:1000A000030002030369A5020269A532730000017F
:1000B00000000000000400FFFFFFFFFFFFFFFF0440
:1000C00003090424035400650078006100730020D4
:1000D0000049006E0073007400720075006D0065C9
:1000E000006E007400730024035400490020004394
:1000F000004300320035003300310020005500532A
:10010000004200200043004400430000035F005F02
:100110000030005800000000000000000000000057
:1001200000000000000000000000000000000000CF
:100130000000000000303132333435363738394171
:1001400042434445463C1C911C911C911C911C99B6
:100150001C74F8121BD6900391E060159003027492
:10016000FEF0900304744DF0A37405F07A011207B9
:100170000C7F01021D7B74F8121BD674FF121EC582
:100180007E00801F851882851983E064FE700690CA
:1001900003877401F0851882851983E0F890038441
:1001A000E068F07901AA18AB191210DFE9700302B8
:1001B000027E851882851983E064EF70027E07E075
:1001C000C0E0900387E0F8900385E0FAE82AF8E4BD
:1001D000340012075BD0E0F0900387E060A6146063
:1001E0000E14602A14603A14605014606680A69061
:1001F0000384E4F0851882851983E0900386F0C3B8
:1002000094809003874003E4808A74028086851876
:1002100082851983E0900382F090038774030201C2
:1002200094851882851983E0900383F0900386E01B
:1002300060199003877404020194900385E004F030
:10024000F8900386E06860030201959003877405C7
:10025000020194900385E4F0900387F0900384E01A
:10026000F8851882851983E0686003020195900380
:1002700082E0644D60030201951203B68002EEF93C
:100280007401121E4602017174F7121BD674FB1220
:100290001EC5EAFEEBFF7508047509007808121EFA
:1002A000DF7402121F467A907B0079041218F274F0
:1002B00002121E461206FE121F97E0687003A3E0AA
:1002C000697012851882851983E0F47003A3E0F445
:1002D00060030203917404121F3E1207678A088BA1
:1002E00009A808A9097402121F97E8F0A3E9F0749D
:1002F00004121F97E0600879011201510203AA85D8
:100300001882851983E0687003A3E0697076851808
:1003100082851983E0F47003A3E0F470197402126B
:100320001F977410F0A37420F085188285198374C8
:1003300010F0A37420F07508017509007808121EEA
:10034000DF7402121F467A247B0812197774021296
:100350001E467508047808121EDF7402121F467AC2
:10036000907B0079041218F27402121E461206FEE7
:10037000121F97E0687003A3E06970047902800699
:100380007904800279031201518E828F83741E805A
:10039000058E828F83E4F01206FE121F97E06870CC
:1003A00003A3E06970047901800279007405121ECC
:1003B000467F02021D7B74ED121BD674F8121EC517
:1003C000900307E0FA900306E0FB8B08EAF8E4C824
:1003D000F9EB28FEE93408FF751001880C750D064D
:1003E0008F0974027808121F2BC39508F8E4950949
:1003F000F9740228F50E740339F50F8E088F09740D
:10040000097808121F5DE508F511EE2410F508E4DF
:100410003FF509EEF50AEF5401F50B900383E01464
:1004200060541470030204EB147003020566146038
:100430001024FE70030206211470030206D1020686
:10044000E1750D03794E1213B29003071206F4748E
:1004500002F0A374401206F274081206F2F0A3F040
:10046000751012AA10A90C12070CA90D7408121EFF
:10047000467F0C021D7B750D04794E1213B2EE45BA
:100480000B7005A9111219DDC3EE9425EF940850E5
:100490003CC3E5089424E50994084031E50E249610
:1004A000F8E50F3420F988828983E0701BA3AA82C3
:1004B000AB83E070139003887401F08882898374A1
:1004C000A5F08A828B838004900388E4F07508107D
:1004D0007509007808121EDF7C087D03EEFAEFFB39
:1004E0001219777402121E46020463750D05E51198
:1004F000C394794006750C010204637512407513AC
:10050000007812121EDF7C097D037402780A121F24
:100510002BAA0AAB0BA9111218F27402121E4690F4
:100520000307E0A3F0900306E0A3F0751043C3EEC9
:100530009425EF94084003020463C3E5089424E57E
:100540000994085003020463900388E070030204D6
:1005500063E50E2497F8E50F3420F988828983E457
:10056000F0A3F00204637508047509007808121EF0
:10057000DF7402121F467A907B0079041218F2741D
:1005800002121E467402121F97E0F8A3E0F98518C4
:1005900082851983E0687003A3E069851882851954
:1005A00083700BE0F47003A3E0F470578009E0F46B
:1005B0007003A3E0F4700D8518828519837410F020
:1005C000A37420F01206FE121F97E8F0A3E9F0755D
:1005D00008017808121EDF7402121F467A247B0875
:1005E0001219777402121E467508047808121EDF6D
:1005F0007402121F467A907B0079041218F274027A
:10060000121E461206FE121F97E0687003A3E069EF
:100610007006750D01020463750D02750C07020466
:10062000639003D6E0600764026003020463EAFF9C
:100630007A01790012070CE060030206C5800312FC
:10064000117B121162E970F77404121F971206E60B
:100650007404121F977808121F7B85080C85090DFA
:10066000850A0E850B0F9003C2780C121F057404C7
:10067000121F97780C121F6CE5084509450A450BB7
:1006800070CE8EC2E5C554E04FF5C57404121F97B5
:100690001206E67404121F977808121F7B85080C57
:1006A00085090D850A0E850B0F9003C2780C121F69
:1006B000057404121F97780C121F6CE50845094554
:1006C0000A450B70CE7A01790012070C79080204F2
:1006D0006CEB900391F07003020463750D09020442
:1006E00063790602046CE4F0A37426F0A3E4F0A39B
:1006F000F022F0A3E4F0A3F0A3F0A3F0A322851866
:1007000082851983E0F8A3E0F974022274F6121BC3
:10071000D6EAFE900305E0D2E7F0E9A3F0EE9003FD
:1007200003F08E0A74042AFE7A028004E0620A0A48
:10073000EAF83395E012075B8E08C3E89508E99460
:1007400000A2D265D03340E4E50AF0740128F97ABA
:10075000027B0312111D7F03021D7BF9740228F531
:1007600082740339F5832274E9121BD675820075F1
:1007700083FE121E288A168B177514007515008AC1
:10078000828B83E4F09003D6E07006D2AAD2AF80C9
:1007900004640270057900120151750C00750D207A
:1007A000750E00750F009003D6E0600464027015AA
:1007B00012117B120176E9F874096860030208A33C
:1007C0007900120151E064027007A292400302080E
:1007D0007E7508007509027808121EDF7402121F68
:1007E00046850C08850D09AA08E5095407FB850E06
:1007F0000A850F0B740B7808121E96A9081218F2BE
:100800007402121E467E007F009003CAC0828E10C2
:10081000EFF5113395E0F512F513850C08850D09F8
:10082000850E0A850F0B78087910121F189003C6E1
:100830007808121F05758303D0827808121E0950AC
:100840001D851882851983E5822EF582E5833FF5A3
:1008500083E0F9AA14AB151208D28A148B150EEE98
:1008600070010FC3EF940240A09003CE780C121FCA
:10087000059003D2780C121E0940030207A67900E6
:10088000AA14AB151208D279001208D28B15900366
:10089000D6E07004C2AFC2AAEA451570277AA57BDC
:1008A000A58021E870030207C5740668700302077B
:1008B000C574076870030207C5851682851783749F
:1008C00001F080BA758200758302121E287F100223
:1008D0001D7BC008C0097C088A088B09740F780842
:1008E000121F5DEA25E0FAEB33FBE9A2E75004743E
:1008F000014AFAE508A2E0500874216AFA74106B04
:10090000FBE9C333F91CEC70CFD009D0082274F78F
:10091000121BD6120F2860030209E9A3E0F8A3E036
:1009200060030209E9A3E064027002A3E06003022D
:1009300009E99003B8E02480600914604F14605CFA
:100940000209E9E860030209E99003B2E060047873
:1009500001800278009003C0E8F0A3E4F09003B1B6
:10096000E0600A9003C0E04402F0A3E4F09003A624
:10097000E0640460149003B374C0F0A37403F0A3A4
:10098000E4F0A37402120F8AF002100A90039FE0B1
:10099000640470559003C0E4F0A380D0E8547FF560
:1009A0000890039FE064047040E508C39406503942
:1009B000749F2508F582E43403F583E854806018B9
:1009C000A3A3A3A3A3A3A3E06403700478018002FC
:1009D00078009003C0E88091E582240CF5825002F3
:1009E0000583E0640370E980E39003A674048098B3
:1009F00074F7121BD6E9FE9003BE120F2B600302A0
:100A00000AD190039FE06404600B9003BC120F2B8B
:100A10006003020AD19003B8E0541F6009146030EB
:100A2000146020020AD19003BAE064017022EE90B3
:100A300003B1F060047905800279067A00121BD4B4
:100A4000020AD79003BCE0547FFA9003BAE0600535
:100A50007900020AD9EAC394065076EA90620EF051
:100A6000749F2AF8E43403F99003BCE05480602CAE
:100A7000EE6004741080027440906211F0EE600425
:100A800074038001E488828983A3A3A3A3A3A3A3FF
:100A9000F0EE6004790880307907802CEE600474F1
:100AA0002080027480906214F0EE60047403800170
:100AB000E4C0E0E8240CF582E439F583D0E0F0EE00
:100AC0006004790A80027909121BD490620EE480D6
:100AD000059003A67404F0790102100A7900120946
:100AE000F0E97003121BC32279011209F0E97003C7
:100AF000121BD222C082C0839003BC120F2B701530
:100B0000A3120F2B700F9003BA120CD05480FAE985
:100B1000FBEA4B60079003A67404801AE890620019
:100B2000F090039F6009E06402700C74038007E09A
:100B3000640370037402F0D083D0822274F3121B1A
:100B4000D69003BAE0FAA3E01460081460101460B1
:100B500039805712175F120CADA37B80804179005A
:100B6000121781120CAD7B80E92402F9E43AFA12E3
:100B70001E7CFC1919E0FAA3E92403F9E43AFA12FD
:100B80001E7CF9ECA3F0A3E9801CEAF91217EF90A0
:100B900003B3EAF0A3EBF0A3E4120CBCA37B0012B6
:100BA0001E7CA3F0A3E4F0020C679003B3E4F0A36F
:100BB000F0A3F0F50B90047DE0FAA3E0FB020C42F9
:100BC00075090074037808121F2BEA2508F8EB3525
:100BD00009F99003BA120CC6E493C0E0EFFCD0E030
:100BE0006C705DA3E4936E70579003BC120CC6A3A7
:100BF000A3E493C0E0EFFCD0E06C7044888289836A
:100C0000A3A3A3E4936E703888828983A3A3A3A3CC
:100C1000E493F508740193F5099003B3E508F0A394
:100C2000E509F0A37480F088828983A3A3A3A3A31A
:100C3000A3E493F8740193F99003B6E8F0A3E9F004
:100C4000050B850B0890047F120CD0C39AF50CE9B4
:100C50009BF50D7403780C121F5DC3E508950CE439
:100C6000950D5003020BC09003B3E0FCA3E0FDA37D
:100C7000E0FEEC4D4E9003A6700474048029E064FD
:100C80000460259003BEE0FAA3E0FB9003B6E0F811
:100C9000A3E0F9C3EA98EB9950089003B6EAF0A3F1
:100CA000EBF09003A67401F07F06021D7B9003B366
:100CB000EAF0A3EBF0A37480120CBC22F09003B313
:100CC000E0F9A3E0FA22E0FEA3E0FF888289832214
:100CD000E0F8A3E0F9E82274EE121BD6EA2404F847
:100CE000E43BF9880889098882F583E493602590BC
:100CF0000481120CD0FEE9FF8007EE2404FE5001AF
:100D00000F8E828F83E493F8740193F9EA6870027E
:100D1000EB6970E6750C00803F9062147490F0747B
:100D200010120E2A7003750D408E828F83A3A3A329
:100D3000E49355106006E50DD2E0F50DE50D9062E7
:100D400015F0EA906213F0EC240CF582E43DF58393
:100D5000E4F090620EF0050C850882850983E49327
:100D6000F8E50CC3984003020E257A0079051216A7
:100D7000F28A0E8B0FEA450F60DCEA2402F8E435B4
:100D80000FF9880A890B8882F583E493540FF512D2
:100D900090620EF0750D008A828B83A3A3A3A3E457
:100DA000932407F510A3E4933400F511740378102D
:100DB000121F5DAA10851210749F2510F8E43403E9
:100DC000F9E8FCE9FD751001751100E512781012C3
:100DD0001F2BE50E2403F8E4350FF9850A82850BF5
:100DE00083E493A2E74003020D199062117448F066
:100DF0007408120E2A7003750D408E828F83A3A390
:100E0000E49355106006E50DD2E0F50DE50D906216
:100E100012F0EA906210F08C828D83A3A3A3A3A3A7
:100E2000A3A3020D507F0B021D7BF088828983E40F
:100E3000935403640122C082C083120F287010A350
:100E4000120F2B700AA3E064017002A3E060079008
:100E500003A67404800C9003B374A0F0A37403126F
:100E60000F80F0020B3774F4121BD690039FE064DE
:100E70000260149003BC120F2B700CA3120F2B7086
:100E8000069003BBE060099003A67404F0020F23F0
:100E90007A007901121BD49003BAE060717A00F9EC
:100EA0001217818A088B09EA4509605A90039F74DA
:100EB00004F09003BAE09003A0F0750C008508825E
:100EC000850983A3A3A3A3E493F8E50CC398504C2E
:100ED000850C0A74A1250AF8E43403F9E8FEE9FF59
:100EE0008E828F83E4F07A0079041216F28A828B64
:100EF00083A3A3A3E493F88E828F83E06870E71244
:100F00000CD7050C80B79003A67404F0800E9003F4
:100F1000A0F090039F7403F0F91216587A0079023A
:100F2000121BD47F05021D7B9003BAE0F8A3E0F901
:100F3000E8492274F6121BD690039FE064047019EE
:100F40009003B8E064817011120F28700C9003BEFA
:100F5000E064017002A3E060079003A67404801AA5
:100F60009003BCE024A1F508A3E03403F509900345
:100F7000B3E508F0A3E509120F80F07F03021D7BA3
:100F8000F0A3E4F0A304120F8A22F0A3E4F090038C
:100F9000A6042274F7121BD690039FE064047064C9
:100FA0009003B8E06401705C9003BE120F2B705484
:100FB0009003BAE0FB9003BCE0FA9003A0E0F912C2
:100FC00017B98A088B09AE08AF09EE4F6036900357
:100FD000BCE0FA7903121BD49003BAE0C0E090039E
:100FE000BCE024A1F8A3E03403F988828983D0E02F
:100FF000F0EEFAEFFB120CD79003BCE0FA79041282
:101000001BD480069003A67404F07F02021D7BC0EF
:1010100082C0838003121A39A2E840F9A823E85459
:101020000460097823E654FBF6121402A823E8545E
:101030001060097823E654EFF6121420A823E8A2E2
:10104000E05005782354FCF690620EE0FA7404F048
:10105000906214E0A2E0503AE5A8F8C2AF906216A0
:10106000E0F9A3E0E9FBE8A2E792AF8017906228DD
:10107000E0C0E0900393E0F8121112D0E0F090038A
:1010800093E004F0EBFC74FF2C1B0470E0906214FE
:10109000E4F0EA90620EF0E0FD7404F0906211E07A
:1010A000A2E04031900395E0F8900394E068602559
:1010B0007A40900394121155E0906228F0900394C6
:1010C000E004F008900395E06860041AEA70E39089
:1010D00062117401F0ED90620EF0D083D082227420
:1010E000F8121BD6E9FE79008012121112E08A82F2
:1010F0008B83F0900392E00412114A09900392E06E
:10110000F8900393E0686005E9C39E40DD7F01022B
:101110001D7B748528F582E43404F58322C082C0E7
:1011200083E9FC80188A828B83E0C0E090039512EB
:101130001155D0E012114A900395E004F0ECF874D8
:10114000FF281C0470DF79018090F08A828B83A3D2
:10115000AA82AB8322E0F8748528F582E43405F591
:101160008322C082C083900395E0F8900394E068E6
:1011700060047901800279000210DA02100F74FB1A
:10118000121EC57E009006857808121F7B794A12D0
:1011900013B29006857401F0A3F0A37469F0A374F0
:1011A000A5F09003D77808121EF070030E801590FA
:1011B00003DB7808121EF06008E59D541864107077
:1011C00003022000EEF9121329C280D291EEA2E0B0
:1011D00050030212DCAA18AB19120288E97003024C
:1011E00012DCC291851882851983E0C3943C500EAD
:1011F000E0F8743CC398F50895E0F5098006750899
:1012000000750900E4F50AF50B9003DF780C121F56
:101210007B7808790C121ADA790612015112100F34
:10122000120176E9F8740968700779061201518095
:10123000277407686016A2935012E8600874066865
:1012400060030212DCA292400F0212DC75080075E6
:101250000900750A00750B0085080C85090D850AC3
:101260000E850B0F9003C27808121F05E50C450D83
:10127000450E450F70A7D2807907120151800312E5
:10128000100F121162E970F77E007F007401121FC7
:1012900097E4F0A37426F0A3E4F0A3F07401121F06
:1012A000977808121F7B85080C85090D850A0E8525
:1012B0000B0F9003C2780C121F057401121F977850
:1012C0000C121F6CE5084509450A450B70CEA29229
:1012D00050FCA29350F81213AD022000D280D2919C
:1012E000794E1213B2750800750900750A00750B66
:1012F00000790512015112100F120176E9F87409F4
:101300006860EE74016870EE12100F9003E37808C5
:10131000121F059003E77808121E0950EB1213AD57
:101320000220007405121E462274F8121BD6E9FE34
:1013300053BEFBE59DA2E650FA0078F8790100E87B
:1013400024FF18E934FFF9E84970F375C68074800A
:10135000659E70FA43BE049062707408F01213A286
:10136000EE700853F4FEC29043FE017403F5D57588
:10137000D489900396E4F0A374C2F0A37401F0A39F
:10138000E4F0A3F0A3F0A37408F01213C87AFF7B73
:10139000FF1219F453F4FED29043FE011213A2027D
:1013A000110DD28043FD01C29143FE0222D280C2C0
:1013B0009122781075B60FE5B4A2E750FAE5BBC3E9
:1013C0009940F118E870ED22C082C0837A0079015B
:1013D0001217818A828B83A3A3A3A3A3A3A3E4935D
:1013E000A2E69003B2500474018001E4F09003B1CE
:1013F000E4F090620F7403F0E0A2E750FBD083D0DA
:101400008222C082C08390039F7402F0A3E4F09014
:1014100003A6F0790312165875210075220080DDAD
:1014200074F6121BD690620EE0FEE4F0906211E0BA
:10143000FFA2E4501D7480F09003A67407F0E5212C
:1014400045226009852182852283121FA69003A66A
:10145000E4F0EFA2E2500B906211E4F09003A6F0EA
:1014600080669003A6E0F87402687045906216E00A
:10147000FF9003B3121DBBEFF97A207B6212168C2A
:101480007403121E468F089003B612163C121634CF
:101490002F121647E0F8A3E0F9E849600474408091
:1014A000027448906211F0E849600302162A02169D
:1014B000067406687009852182852283121FA69012
:1014C00003A6E060030215B1EFA2E0400302162A72
:1014D0007508B8750903750A007808121EDB7908CB
:1014E0007A207B6212168C7403121E4675210075D9
:1014F00022009003B8E054E0601D24E07003021560
:101500008D24E0607224C0604824E07003021598C6
:1015100024E0606E0215A3A3E014602624FE601D83
:1015200024FE600A24FC601F24FE60208075120ADD
:10153000F49003A6E06404707274608070120AE88C
:1015400080EF120ADC80EA120E6680E5120F9380AB
:10155000E0A3E0600E24FA600F24FE601024FE6019
:1015600011804012090E80C9120B3C80C4120E3645
:1015700080BF120F3380BA7521BF75221B121BBFAB
:1015800080AF7521C175221B121BC180A475215A21
:1015900075221B121B5A809975218A75221B121BFA
:1015A0008A808E9003A67404F0808E74409062113D
:1015B000F09003A6E0F874016870617F029003B6B2
:1015C000E0F8A3E0F9C3E89420E994005007E8F5B7
:1015D0000A7F0A8003750A209003B3121DBBA90A73
:1015E0007A207B621216B77403121E46850A08120F
:1015F0001634250812164712163CEF906211F0E5DA
:101600000AC394205024E521452260098521828562
:101610002283121FA69003A6E4F0800E7405687062
:1016200009852182852283121FA6EE90620EF07F2B
:1016300003021D7B9003B31216E4E922C3E0950870
:10164000F0A3E09400F022F9E43AFA9003B3E9F051
:10165000A3EAF0A3EBF0A32274F7121BD678007470
:10166000A728F582E43403F583E9F008E8C394057C
:1016700040ED780074AC28F582E43403F583E9F09A
:1016800008E8C3940540ED7F02021D7B74F8121B2D
:10169000D6EAFCEBFDE9F87408121F971216DF601A
:1016A000118C828D83E0121EAFE9240109E43AFA1D
:1016B000D8EF7F01021D7B74F8121BD6EAFCEBFD0C
:1016C000E9F87408121F971216DF6011121E7C8C45
:1016D000828D83F0E9240109E43AFAD8EF80D3122D
:1016E00016E4E822E0F9A3E0FAA3E0FB22D083D0DD
:1016F0008222C082C083E9FCEAFD7A007B0080037D
:1017000012173D90039DE0F8A3E0F990047BE06898
:101710007003A3E069602490039EE0F5838882A3B0
:10172000E493F8EC68700D90039DE0FAA3E0FB12DF
:10173000173D8007ED6870C8ED60C580B090039DCF
:10174000E0F8A3E0F5838882E493F890039DE02815
:10175000F8A3E03400F990039DE8F0A3E9F022C07B
:1017600082C0831217707A0079011216F20216ED08
:10177000900479E0F8A3E0F990039DE8F0A3E9F084
:101780002274F7121BD6E9FEEAFF1217707A00796D
:10179000021216F2EA4B601CEE60108A828B83A361
:1017A000A3A3A3A3E4936E70E48009EFF874FF2869
:1017B0001F0470D97F02021D7B74F5121BD6EAFF4D
:1017C0008B087A001217817A0279041216F2EA4B1A
:1017D00060188A828B83A3A3E4936F70EA8A828B5A
:1017E00083A3A3A3E493650870DD7F04021D7B74CB
:1017F000F7121BD674F0121EC5E97A007B00600C4C
:101800001460101460141460180218DB7AF37B0360
:101810000218DB7AF77B030218DB7A1B7B040218C1
:10182000DB90043FE060030218D79003EB740812CA
:101830001F467408121DE8750808F5097808121E7D
:10184000DF7402121F467AE87B07797F1218F27460
:1018500002121E467808121EDF740A121F46740216
:10186000121F3E121C997402121E468B09EA45098A
:1018700070197509007808121EDF7C0C7D787402DF
:10188000121F3E121D357402121E467C287D0085F3
:101890001882851983E5822DF582E43583F583E08E
:1018A000FF743F2CF8E43404F9EF1218E3888289BE
:1018B00083F0EFC41218E3C0E0E824FEF582E934B7
:1018C000FFF583D0E0F00D74FC2CFCEDC3940840D0
:1018D000BE90043F742AF07A3F7B047410121E46B7
:1018E0000217B4540FFA74692AF582E43404F583BC
:1018F000E02274F5121BD68908740F5508F50A7595
:101900000B00740B780A121F2BEA2400F8EB3480CA
:10191000F9E82400E9350BF9E5C7F509A2AFE4338E
:10192000F50AC2AFE508C4540FFAE5C754F84AF502
:10193000C7740B121F97E0FAA3E0FB801C88828912
:1019400083E08C828D83F088828983A3A882A98317
:101950008C828D83A3AC82AD83EAFEEBFFEE24FF85
:101960001AEF34FFFBEE4F70D48509C7E50AA2E0F9
:1019700092AF7F04021D7B74F7121BD6ED90038992
:10198000F0ECA3F0A37462F0A37473F0A3E0541F0F
:10199000F07409121F97E0F508A3E0F509E5083394
:1019A0003354FC90038EF074067808121F5DE5082E
:1019B00090038DF090038F7412F0A37442F075D1F0
:1019C000FE75D601EA906271F0EBA3F0906270E0D0
:1019D000D2E1F0E0A2E740FB7F02021D7BC082C0A3
:1019E00083E9C333906272F0906270E0D2E0F0D08D
:1019F00083D0822274F7121BD675230075240075DC
:101A000025008A268B27EA90620BF08A088B0974DE
:101A1000047808121F5DE508906207F08A088B09B8
:101A200074097808121F5DE508543E906209F0754C
:101A30008B00C2E87F02021D7B74F7121BD6E59D66
:101A4000A2E650FA906206E0FAA2E25035A826E833
:101A500090620BF0F50885270974047808121F5D61
:101A6000E508906207F0852608852709740978083B
:101A7000121F5DE508543E906209F0906201E0D2C9
:101A8000E0F07823EA46F6906202E0F50875090076
:101A900074047808121F2B7823E50846F608E50938
:101AA00046F6906204E0F50875090074097808129A
:101AB0001F2B7824E50946F6EAA2E05003752501BC
:101AC00074065A6003752500E58BA2E55006758BF8
:101AD000DF752500121BD5021A2F080808EAC0E09E
:101AE000EBC0E086F0E7A4FA180986F0E7A42AFA2A
:101AF000180986F0E7A42AFA180986F0E7A42AFA5A
:101B00001986F0E7A4FBE5F02AFA190886F0E7A4A5
:101B10002BFBE5F03AFA190886F0E7A42BFBE5F079
:101B20003AFA18180986F0E7A4C5F02BFBE43AFA54
:101B30001908E7C5F0C6A426F6E5F03BFBE43AFA3F
:101B40001886F0E7A4F6E5F00826F6E43B08F6E48C
:101B50003A08F6D0E0FBD0E0FA22C082C0839003BE
:101B6000B9E0F874226870089003A6E0701A80113A
:101B70007420689003A6700DE0700D121BB19003E5
:101B8000A6740280027404F08043C082C083900374
:101B9000B9E064219003A67013E07013121BB1A387
:101BA0007407F0A3E4F09003A60480027404F080AC
:101BB0001C9003B37496F0A37403F0A3E4F02280A6
:101BC000028000C082C0839003A67404F0D083D04A
:101BD000822280EF22222518C582C0E0E51934FF59
:101BE000C583C0E0E518C3958224F910AF0885834A
:101BF000198582188008858319858218D2AFCEF0A6
:101C0000A3E520F0A37808E608F0A3DEFAEFF0A33E
:101C1000E58124FBF8E608F0A3E608F0A30808E64F
:101C200008F0A3E608F0A315811581D0E0FED0E00E
:101C3000F815811581E8C0E0EEC0E0221201000233
:101C4000020000205104A816090001020301090244
:101C50004300020100801909040000010202010092
:101C600005240010010424020205240600010524B5
:101C70000100010705820340004009040100020A37
:101C80000000000705840240000007050402400030
:101C900000571C00007A1C000074F5121BD6740B50
:101CA000121F97E0F8A3E08015A3AA82AB838C8271
:101CB0008D83A3AC82AD83E824FF18E934FFF9E8F3
:101CC00049601F8C828D83E0F5088A828B83E0F562
:101CD0000AE508650A60D2E50AC39508FA95E0FBB3
:101CE00080047A007B007F04021D7BE47921780761
:101CF000B800028004F709D8FCE490030278C179A7
:101D0000018002F0A3D8FCD9FA7AC27B0390008E3E
:101D100078C479018015E493A3AD82AE838A828B67
:101D200083F0A3AA82AB838D828E83D8E9D9E71290
:101D3000117E121FA174F7121BD6EAF8EBF9740991
:101D4000121F97E0FEA3E0FF80188C828D83E0884D
:101D5000828983F0A3A882A9838C828D83A3AC821D
:101D6000AD838E088F09E50824FF1EE50934FFFFC7
:101D7000E508450970D47F02021D7B85198385180B
:101D800082E0A3FEE0A3F5207808E0A3F608DFFADE
:101D9000E0A3FFE0A3C0E0E0A3C0E0E0A3C0E0E078
:101DA000A3C0E010AF08858218858319800885825A
:101DB00018858319D2AFD083D0822274038000CCDF
:101DC000C0E0EDC0E0E518C39CCCAD1950011D107A
:101DD000AF068C188D1980068C188D19D2AF121D84
:101DE000E8D0E0FDD0E0FC22CAC0E0E0A3C582CC90
:101DF000C582C583CDC583F0A3C582CCC582C5830A
:101E0000CDC583DAE6D0E0CA22C008C3E096F50863
:101E100008A3E096420808A3E096420808A3E096CB
:101E200045087001D3D00822C5822518C582C58314
:101E3000351910AF07F5198582188007F5198582C5
:101E400018D2AFC5832200C0D0251810AF08F518EE
:101E5000500C05198008F51850020519D2AFD0D0E2
:101E6000222518F58210AF08F518400C15198008C6
:101E7000F51840021519D2AF85198322BB0102E77C
:101E800022C082C08389828A83BB0003E08002E48F
:101E900093D083D082226016080808C6C313C618E0
:101EA000C613C618C613C618C613C6D5E0EA22BBA9
:101EB000000EC082C0838A838982F0D083D08222C0
:101EC000BB0101F722251810AF08F518400C1519B1
:101ED0008008F51840021519D2AF227403800474EB
:101EE000028000C0E0F404121E61D0E0121F8A22BA
:101EF000E066701008A3E066700A08A3E06670044C
:101F000008A3E06622E026F608A3E036F608A3E080
:101F100036F608A3E036F622E627F60809E637F695
:101F20000809E637F60809E637F622700422600D44
:101F300018C6C333C608C633C6D5E0F41822251820
:101F4000FAE43519FB222518FCE43519FD2275D079
:101F50000075813F751802751903021CEB600C08AF
:101F6000C6C313C618C613C6D5E0F422E6F008A30C
:101F7000E6F008A3E6F008A3E6F022E0F608A3E006
:101F8000F608A3E0F608A3E0F622CAC0E0E6F0A354
:101F900008DAFAD0E0FA222518F582E43519F5833B
:101FA0002200000080FBE473FFFFFFFFFFFFFFFF45
:101FB000FFFFFFFFFFFFFFFFFFFFFFFFFFFFFFFF31
:101FC000FFFFFFFFFFFFFFFFFFFFFFFFFFFFFFFF21
:101FD000FFFFFFFFFFFFFFFFFFFFFFFFFFFFFFFF11
:101FE000FFFFFFFFFFFFFFFFFFFFFFFFFFFFFFFF01
:0A1FF600850609433886000000004C
:020000040003F7
:01FFF000F020
:020000040000FA
:10200000022D9002221DFFFFFFFFFFFFFFFFFFFFDA
:10201000FFFFFFFFFFFFFFFFFFFFFFFFFFFFFFFFD0
:10202000FFFFFFFFFFFFFFFFFFFFFF022A68FFFF29
:10203000FFFFFF022240FFFFFFFFFFFFFFFFFFFF49
:10204000FFFFFFFFFFFFFFFFFFFFFFFFFFFFFFFFA0
:10205000FFFFFF022159FFFFFFFFFFFFFFFFFFFF11
:10206000FFFFFFFFFFFFFFFFFFFFFF022A40FFFF11
:10207000FFFFFFFFFFFFFFFFFFFFFF022891FFFFB2
:10208000FFFFFF0221B901FFFFFFFFFFFFFFFFFF7F
:102090001020102001FF01010503010F10FEFF2693
:1020A0004D00000000BE4C00000000FF000000FFDB
:1020B00000010000253A0000000077396F3BBF396E
:1020C000D93A0000AD390000000000000000000017
:1020D0000000000000000000000000000000FF0100
:1020E0000100A507000000FFFF1E08E8036400646C
:1020F00000B80102020008000005020701051E02E7
:10210000051E020A0A0103B80B02803E0102FEFF0F
:10211000E8030A050001FFFF0A01E00020FD0002BC
:1021200006FFFF00035F005F003000580000000062
:10213000000000000000000000000000000000009F
:1021400000000000000000000000000000B12606B2
:10215000270627062706270E27C0E074F21226520C
:10216000A2AFE433FED2AFE5A7FFE5A1F5085F54C7
:1021700010600612440375A1EFE5085F540860087B
:1021800012440975A1F78024E508A2E092F0EFA2BD
:10219000E082F05017906198E0F8900971E0C398E0
:1021A000A2D265D0335002E8F075A1FE751A00EE98
:1021B000A2E092AF7F0102270EC0E074F212265215
:1021C000A2AFE433FED2AF9061A4E0F8759B00E5C6
:1021D0009158540860087591F71244518023E59195
:1021E00058541060087591EF1244578014E591A27D
:1021F000E092F0E8A2E082F05007E0C2E0F0124581
:10220000AD9061A3E0F8E5E9585404600E124583EF
:1022100075E9FB906193E0A2E640F2808FC0E07424
:10222000F2122652A2AFE433FED2AF9061A5E0F8DD
:10223000E5BF585404600675BFFB1245C50221ACCA
:10224000C0E074F1122652E59DA2E650FA906206B3
:10225000E0FAA2E25035A82CE890620BF0F5088570
:102260002D0974047808122DA0E508906207F08506
:102270002C08852D0974097808122DA0E508543E14
:10228000906209F0906201E0D2E0F07829EA46F627
:10229000906202E0F50875090074047808122D2C8C
:1022A0007829E50846F608E50946F6906204E0F567
:1022B0000875090074097808122D2C782AE509465A
:1022C000F6EAA2E05003752B0174065A6003752BE1
:1022D00000E58BA2E55006758BDF752B0012477564
:1022E000758B00C2E87F0202270EC3E498F8E499D8
:1022F000F912232B8026C3E49AFAE49BFBE920E73A
:10230000E912232BE498F8E499F922C3E498F8E45D
:1023100099F912232BE498F8E499F9C3E49AFAE4C2
:102320009BFB22EB20E7CFE920E7E0B90010BB00E0
:1023300008E88AF084F8AAF022E4FBC8FA22EB70DD
:10234000227B10C833C8C933C9335007C39AC3DBD3
:10235000F280069A50012ADBEAC833F4C8C933F484
:10236000C9FA2275F008E4C833C8C933C933C99A19
:10237000C99B5004C92AC93BD5F0ECFBC833F4C84B
:10238000E4C9FA2274F51225EC74FA122C2A7508A5
:10239000047509007808122B527404122BF67AF88F
:1023A0007B0779031242DD7402122B809080F8784B
:1023B00008122DBE7402122E157808122C55704981
:1023C0007508027509007808122B527402122BF658
:1023D0007AF67B0779031242DD7402122B8085188E
:1023E00082851983E0F47003A3E0F4601C851882F1
:1023F000851983E0F8A3E0F9888289837402F0A349
:10240000F0A37469F0A374A5F0C2AF75D69F020063
:10241000007406122B807F040228D4080808EAC042
:10242000E0EBC0E086F0E7A4FA180986F0E7A42AFA
:10243000FA180986F0E7A42AFA180986F0E7A42A10
:10244000FA1986F0E7A4FBE5F02AFA190886F0E706
:10245000A42BFBE5F03AFA190886F0E7A42BFBE57C
:10246000F03AFA18180986F0E7A4C5F02BFBE43A15
:10247000FA1908E7C5F0C6A426F6E5F03BFBE43AF6
:10248000FA1886F0E7A4F6E5F00826F6E43B08F62D
:10249000E43A08F6D0E0FBD0E0FA22122E0AB900A6
:1024A000030224FBE47921780DB800028004F709C7
:1024B000D8FCE49004D17855790C8002F0A3D8FCC4
:1024C000D9FA781A9020867A01BA00028007E4933C
:1024D000A3F608DAF97A257B1090209478C6790162
:1024E0008015E493A3AD82AE838A828B83F0A3AA86
:1024F00082AB838D828E83D8E9D9E7758208758394
:10250000ED7405122B2C75825175834A7400122BC1
:102510002CE4CFC0E0E4CEC0E0E4CDC0E0E4CCC029
:10252000E075F020E626F608E633F608E633F6080E
:10253000E633F6181818EC33FCED33FDEE33FEEFFE
:1025400033FFC3EC9709ED9709EE9709EF97191937
:1025500019400FFFEC97FC09ED97FD09EE97FE1966
:102560001906D5F0BFECF709EDF709EEF709EFF71B
:10257000191919D0E0FCD0E0FDD0E0FED0E0FF2238
:102580002518C582C0E0E51934FFC583C0E0E51811
:10259000C3958224F810AF088583198582188008B6
:1025A000858319858218D2AFCEF0A3E520F0A378F9
:1025B00008E608F0A3DEFAEFF0A3E58124FAF8E6D6
:1025C00008F0A3E608F0A3E608F0A30808E608F080
:1025D000A3E608F0A315811581D0E0FED0E0F81540
:1025E0008115811581E8C0E0EEC0E0222518C58282
:1025F000C0E0E51934FFC583C0E0E518C395822427
:10260000F910AF088583198582188008858319859C
:102610008218D2AFCEF0A3E520F0A37808E608F048
:10262000A3DEFAEFF0A3E58124FBF8E608F0A3E6C9
:1026300008F0A30808E608F0A3E608F0A315811542
:1026400081D0E0FED0E0F815811581E8C0E0EEC051
:10265000E022C0D02518C582C0E0E51934FFC5834B
:10266000C0E0E518C3958224F310AF08858319856F
:1026700082188008858319858218D2AFC8F0A3E933
:10268000F0A3EAF0A3EBF0A37908E709F0A3D8FAE6
:10269000ECF0A3EDF0A3EEF0A3EFF0A3D0E0F0A3F5
:1026A000D0E0F0A3D0E0F0A3E520F0A3E5F0F0A3A4
:1026B0002212010002020000205104A816090001A4
:1026C000020301090243000201008019090400000D
:1026D0000102020100052400100104240202052465
:1026E000060001052401000107058203400040099E
:1026F000040100020A0000000705840240000007F0
:10270000050402400000CC260000EF2600008519D9
:1027100083851882E0C0E0A3E0F9A3E0FAA3E0FB20
:10272000A37808E0F608A3DFFAE0FCA3E0FDA3E04D
:10273000FEA3E0FFA3E0C0E0A3E0C0E0A3E0F5D08B
:10274000A3E0F520A3E0A3F5F010AF088583198579
:1027500082188008858319858218D2AFD082D083F1
:10276000D0E0F8D0E032E47375F0108E218F22852E
:102770008226858325851882851983E0CEA3E0CF44
:10278000852682852583EBC9EAC8EDCBECCAC3E870
:1027900033C8E933C9EA33CAEB33CBC3EA9EF52425
:1027A000EB9FF523B35004AB23AA24EC33CCED33D9
:1027B000CDD5F0DAAE21AF2222D083D082ECC0E0BA
:1027C000EDC0E0E493A3FCE493A3FDED4C600D1297
:1027D0002914EC24FFFCED34FFFD80EFE493A3FC0F
:1027E000E493A3FDED4C600D1229EBEC24FFFCED0E
:1027F00034FFFD80EFD0E0FDD0E0FCE493A3C0E027
:10280000E493C0E022851983851882E0A3FEE0A34B
:10281000F5207808E0A3F608DFFAE0A3FFE0A3C004
:10282000E0E0A3C0E0E0A3C0E0E0A3C0E0E0A3C01C
:10283000E010AF0885821885831980088582188585
:102840008319D2AFD083D082022B32D083D082E9D9
:10285000C0E0E493A3C386F0C5F095F0F908E493D3
:10286000A386F0C5F095F0700BE493A3C3994005DF
:10287000E9048002A3E475F002A42582F582E5F064
:102880003583F583D0E0F9E493A3C0E0E493C0E09E
:1028900022C0E074F2122652A2AFE433FED2AFE5BA
:1028A0008AA2E25007900932E0D2E0F0E58AA2E382
:1028B0005007900932E0D2E1F0758A00C2EB7A103D
:1028C0007B0090092EE0F9123D01EEA2E092AF7F6D
:1028D0000102270E851983851882E0A3FEE0A3F587
:1028E000207808E0A3F608DFFAE0A3FFE0A3C0E049
:1028F000E0A3C0E0E0A3C0E0E0A3C0E010AF088523
:1029000082188583198008858218858319D2AFD0F3
:1029100083D08222C0E0C3E4939608740193961892
:10292000400FE49366700808740193661870007095
:1029300019A3A3C3E49396087401939618A3A34024
:102940000DD0E0D0E0D0E00227F5A3A3A3A3A3A37A
:10295000D0E022D083D082C5F0E493A3C5F0C39524
:10296000F0F5F0E493A3C395F04005E5F004800191
:10297000E475F002A42582F582E5F03583F583E461
:1029800093A3C0E0E493C0E0227404800874038041
:102990000474028000CCC0E0EDC0E0E518C39CCC1C
:1029A000AD1950011D10AF068C188D1980068C18BA
:1029B0008D19D2AF122AAED0E0FDD0E0FC22740215
:1029C0008000CCC0E0EDC0E0E518C39CCCAD195050
:1029D000011D10AF068C188D1980068C188D19D228
:1029E000AF122A8CD0E0FDD0E0FC22C0E0C0F0881D
:1029F000F0E4936670080874019366187000A8F0FC
:102A0000A3A3700BD0F0D0E0D0E0D0E00227F5A374
:102A1000A3D0F0D0E022D083D082CCC0E0E493A356
:102A20006006122ACF1470FAE493A36006122BFEFC
:102A30001470FAD0E0FCE493A3C0E0E493C0E02279
:102A4000C0E074F2122652758900C2C590101DE0D4
:102A5000700E7A007B10900719E0F9123D01800397
:102A60001248B97F0102270EC0E0C0D0E8C0E0E9FB
:102A7000C0E0E5A8D2AFC2C7751A00A2E7A2E792EC
:102A8000AFD0E0F9D0E0F8D0D0D0E032CAC0E0E476
:102A900093A3C582CCC582C583CDC583F0A3C5826F
:102AA000CCC582C583CDC583DAE5D0E0CA22CAC0D1
:102AB000E0E0A3C582CCC582C583CDC583F0A3C5A4
:102AC00082CCC582C583CDC583DAE6D0E0CA22C0F8
:102AD000E0E493A3D39C5010E493A3C39C400AD09A
:102AE000E0D0E0D0E0022A33A3A3A3D0E022700913
:102AF000080808226016181818C6C333C608C6335B
:102B0000C608C633C608C633C6D5E0EA22C008C325
:102B1000E096F50808A3E096420808A3E09642086C
:102B200008A3E09645087001D3D00822C09FF59F06
:102B3000E473D09F22D083D082C09FE493C0E0741E
:102B40000193C0E0740293F59F227404800A740319
:102B50008006740280027401C0E0F404122B65D078
:102B6000E0122DCD222518F58210AF08F518400C83
:102B700015198008F51840021519D2AF851983225E
:102B800000C0D0251810AF08F518500C05198008A2
:102B9000F51850020519D2AFD0D022BB0102E722AE
:102BA000C082C08389828A83BB0003E08002E493F1
:102BB000D083D082226016080808C6C313C618C680
:102BC00013C618C613C618C613C6D5E0EA22C3E05A
:102BD000C696F608A3E0C696F608A3E0C696F608E1
:102BE000A3E0C696F6222518F8E43519F92225182F
:102BF000FAE43519FB222518FCE43519FD22C0E062
:102C0000E493A36C7009D0E0D0E0D0E0022A33A3B3
:102C1000A3D0E022BB000EC082C0838A838982F0E9
:102C2000D083D08222BB0101F722251810AF08F50E
:102C300018400C15198008F51840021519D2AF225A
:102C4000C3E09608A3E09608A3E09608A3E096A246
:102C5000D265D03322E066701008A3E066700A08DF
:102C6000A3E066700408A3E06622E7667010080916
:102C7000E766700A0809E76670040809E76622C378
:102C8000E697F60809E697F60809E697F60809E6D2
:102C900097F622C3E096F008A3E096F008A3E0962A
:102CA000F008A3E096F022E026F008A3E036F00852
:102CB000A3E036F008A3E036F022E657F60809E66E
:102CC00057F60809E657F60809E657F622E056F6E1
:102CD00008A3E056F608A3E056F608A3E056F6224D
:102CE000E056F008A3E056F008A3E056F008A3E091
:102CF00056F022E627F60809E637F60809E637F621
:102D00000809E637F622E026F608A3E036F608A31F
:102D1000E036F608A3E036F622E647F60809E6476D
:102D2000F60809E647F60809E647F622700422602D
:102D30000D18C6C333C608C633C6D5E0F41822E45E
:102D4000C396F608E496F608E496F608E496F622AA
:102D5000C6F4C608C6F4C608C6F4C608C6F4C62239
:102D6000600D08C6A2E713C618C613C6D5E0F32245
:102D7000C3E7960809E7960809E7960809E7962247
:102D8000C3E09608A3E09608A3E09608A3E0962285
:102D900075D00075813F7518D17519040002249B08
:102DA000600C08C6C313C618C613C6D5E0F422E6E5
:102DB000F008A3E6F008A3E6F008A3E6F022E0F6A8
:102DC00008A3E0F608A3E0F608A3E0F622CAC0E0F4
:102DD000E6F0A308DAFAD0E0FA22EAF0A3EBF0A3D7
:102DE000ECF0A3EDF022E0FAA3E0FBA3E0FCA3E00B
:102DF000FD22E0F8A3E0F9A3E0FAA3E0FB22E8F06B
:102E0000A3E9F0A3EAF0A3EBF022E5C754F84401EC
:102E1000F5C77901222518F582E43519F5832212C8
:102E20002B355CB303122B358DB303122B35CCB38A
:102E300003122B35CDB403122B357CB503122B3581
:102E400009B803122B3562B903122B35F5B90312F9
:102E50002B35CABA03122B3540BB03122B35A8BC45
:102E600003122B35C6BC03122B35008002122B3502
:102E70005A8002122B35C48002122B354D8102126A
:102E80002B35098202122B35518202122B358C828E
:102E900002122B35E28202122B354A8302122B35A5
:102EA000CE8302122B35E78302122B350C840212DB
:102EB0002B354A8402122B35998402122B35C28499
:102EC00002122B35118502122B35BD8502122B35CE
:102ED000858602122B35EA8602122B35B78702123D
:102EE0002B35FD8702122B35198802122B354B88A2
:102EF00002122B35F38902122B35CA8A02122B35A6
:102F0000F68A02122B352C8B02122B354D8B0212B6
:102F10002B355C8B02122B35678B02122B351B8CE9
:102F200002122B358E8C02122B35008D02122B359E
:102F3000088D02122B35838D02122B35DC8D021287
:102F40002B351F8E02122B35B19002122B35F791C3
:102F500002122B35879402122B356F9502122B35F6
:102F6000A29502122B35649602122B35139702128A
:102F70002B355B9702122B35BD9702122B35E2974A
:102F800002122B35F39702122B356B9802122B3558
:102F9000F39802122B35579902122B353C9A0212E4
:102FA0002B35619A02122B35829B02122B35A09B86
:102FB00002122B35B39B02122B35269C02122B35A5
:102FC000359C02122B35BD9C02122B350B9D021233
:102FD0002B35149D02122B35149F02122B3568A03D
:102FE00002122B3578A002122B3594A102122B3538
:102FF0000DA202122B3543A302122B3585A3021218
:103000002B35C1A302122B3595A502122B35FAA739
:1030100002122B350EA802122B3518A802122B35DE
:1030200022A802122B352CA802122B3536A8021228
:103030002B354FA802122B3559A802122B3563A845
:1030400002122B356DA802122B359CA802122B35CB
:10305000C4A802122B35CFA802122B3519A90212CF
:103060002B3523A902122B352EA902122B3552A97A
:1030700002122B3576A902122B35D7A902122B3555
:1030800022AA02122B353EAA02122B35A8AA02123E
:103090002B35F4AA02122B353CAB02122B35B7AB01
:1030A00002122B3551AC02122B3515AE02122B3504
:1030B00083AE02122B35B5AF02122B35DBAF0212F5
:1030C0002B354BB102122B35FFB402122B35FFB654
:1030D00002122B35D7B802122B3570B902122B35DC
:1030E00082BB02122B3544BC02122B3590BC02125B
:1030F0002B35F6BC02122B3508BD02122B3558BFFA
:1031000002122B3547C002122B3586C102122B3515
:10311000D8C102122B357DC202122B3538C40212DF
:103120002B3569C502122B3587C502122B35DCC53C
:1031300002122B35DAC602122B3502C702122B35CA
:1031400065C702122B3566C802122B35D9C8021288
:103150002B3507CA02122B3572CA02122B3562CBED
:1031600002122B35C8CD02122B35F6CD02122B35AB
:10317000F1CE02122B358FD002122B35DFD0021286
:103180002B3597D102122B354CD202122B35B0D2EF
:1031900002122B3569D302122B3509D402122B35BA
:1031A0006DD402122B35B7D402122B35F4D402128F
:1031B0002B355CD602122B35598101122B359B81A0
:1031C00001122B35968401122B35E98401122B351F
:1031D0002F8501122B35708601122B35D5860112F1
:1031E0002B35158701122B35588801122B359A8BF8
:1031F00001122B35C38C01122B35049801122B358B
:10320000A49801122B35979B01122B35CE9C0112ED
:103210002B35449D01122B356E9E01122B35BE9F1E
:1032200001122B35A5A001122B350EA301122B354F
:103230001CA501122B35ADA501122B3581A601125B
:103240002B350DA701122B3517A701122B353FA7E0
:1032500001122B35ECA701122B35D7A801122B3503
:10326000AAA901122B3537AA01122B354DAA01123A
:103270002B35B1AA01122B35DAAA01122B3507AB77
:1032800001122B354CAD01122B3527AE01122B3517
:103290006BAE01122B35DCAE01122B3595AF01124E
:1032A0002B35C7AF01122B350EB001122B3541B0B3
:1032B00001122B35A6B001122B35F5B001122B35BA
:1032C000FAB001122B354EB101122B3598B1011213
:1032D0002B3594B201122B35F9B201122B3557B3AD
:1032E00001122B35A1B601122B3575B701122B3502
:1032F00002B901122B35DCBB01122B358FBC011238
:103300002B35B6BE01122B355BBF01122B3599BF91
:1033100001122B3569C101122B357CC101122B35ED
:1033200085C101122B358EC101122B35A3C10112AB
:103330002B35C2C101122B35F7C301122B354AC4FC
:1033400001122B3554C401122B355EC401122B35EA
:10335000B9C401122B3515C501122B352DC601122A
:103360002B358EC601122B35DDC701122B3526C831
:1033700001122B35FEC801122B3529CA01122B353B
:10338000DFCA01122B35E1CB01122B35E3CC011240
:103390002B35C8CD01122B35DFCD01122B351CCEBC
:1033A00001122B3526CE01122B3530CE01122B35D2
:1033B0003BCE01122B3559CE01122B359BCE01127B
:1033C0002B35F9CE01122B351ECF01122B3538CFFC
:1033D00001122B35C5CF01122B35FECF01122B3533
:1033E0004ED101122B35A5D101122B35BFD20112BE
:1033F0002B35F5D201122B3591D301122B350DD47B
:1034000001122B357DD501122B3598D601122B35A3
:103410005ED701122B3508D801122B358DD8011239
:103420002B35F5D801122B35AAD901122B35FCD931
:1034300001122B3571DA01122B353ADB01122B35D3
:103440005DDB01122B3521DC01122B3545DC01122D
:103450002B3567DC01122B35C8DC01122B3513DF4D
:1034600001122B35EEDF01122B3598E001122B35BE
:10347000D9E201122B3527E301122B356AE3011241
:103480002B35C2E301122B3520E401122B354AE41F
:1034900001122B356EE401122B359FE401122B35FE
:1034A000C9E401122B3510E501122B356EE501122E
:1034B0002B35CAE501122B35CBE601122B3535E849
:1034C00001122B3573E801122B359CE801122B35C4
:1034D0002DE901122B3577E901122B359BE90112F9
:1034E0002B35F1E901122B350CEA01122B35C7EA15
:1034F00001122B35F1EA01122B3547EB01122B3566
:103500004CEE01122B357FEE01122B353CEF0112F0
:103510002B3517F001122B35A7F001122B35E8F0EF
:1035200001122B35DE8006122B351D8106122B353C
:1035300044BD03122B35EDBD03122B35CCBE031257
:103540002B35E7BF03122B3507C003122B3529C1DA
:1035500003122B35C6C203122B3533C303122B358E
:1035600009C403122B350FC503122B3574C5031282
:103570002B35B0C503122B3509C603122B3542C6B5
:1035800003122B358BC603122B351DC703122B35A7
:10359000BAC703122B358FC803122B355CC903122F
:1035A0002B35E9C903122B350FCA03122B353CCA40
:1035B00003122B356DCA03122B3542CB03122B3568
:1035C00052CB03122B35A5CB03122B35B2CB0312F2
:1035D0002B35BFCB03122B35C8CB03122B352CCC8C
:1035E00003122B358ACC03122B35D5CC03122B3585
:1035F000F0CC03122B3517CD03122B3534CD03122B
:103600002B3540CD03122B35E4CE03122B35FDCEE6
:1036100003122B3579CF03122B358CCF03122B35A8
:103620009CCF03122B3542D003122B35B2D103129B
:103630002B35C5D203122B3565D303122B356FD32F
:1036400003122B35DDD303122B35EED303122B35AA
:103650002DD403122B355BD403122B3528D503123E
:103660002B357FD503122B35C4D503122B351AD633
:1036700003122B3538D603122B3586D603122B3581
:1036800054D703122B35A2D703122B35E4D70312DC
:103690002B3567D803122B3591D803122B35C7D899
:1036A00003122B35D6D803122B3534D903122B3500
:1036B000ACD903122B35EDD903122B353CDA0312AA
:1036C0002B3567DA03122B3581DA03122B359BDA9F
:1036D00003122B3570DB03122B357ADB03122B35EB
:1036E000B5DB03122B35C5DB03122B35CEDB031202
:1036F0002B351FDC03122B3533DC03122B3551DD48
:1037000003122B3564DD03122B357BDD03122B35C1
:1037100090DD03122B352ADE03122B35A9DE0312AE
:103720002B354CDF03122B3557DF03122B35A4E06A
:1037300003122B35C0E003122B3518E103122B3591
:1037400086E103122B35D2E103122B35ECE1031293
:103750002B354CE203122B35EAE203122B3535E30D
:1037600003122B3598E503122B3530E603122B3567
:10377000A7E603122B35EDE803122B3505E90312FA
:103780002B3508E903122B3514E903122B3528E9F0
:1037900003122B3530E903122B3567E903122B3561
:1037A0005BEA03122B35E5EA03122B3567EB0312B4
:1037B0002B35DCEB03122B35B4EC03122B35D6EC96
:1037C00003122B356DED03122B3579ED03122B35DA
:1037D000D6ED03122B35D9ED03122B3506EE03126D
:1037E0002B351BEE03122B358AEE03122B35D6EF49
:1037F00003122B35E9F003122B3574F103122B352C
:1038000087F203122B3551F303122B3582F3031287
:103810002B35A8F303122B35B1F303122B35E0F34C
:1038200003122B3590F403122B3540F503122B3580
:10383000B3F503122B3565F603122B35D8F60312B8
:103840002B3517F703122B3560F703122B3595F73D
:1038500003122B35D2E404122B353DE504122B352F
:1038600084E504122B35FAE504122B354AE60412DE
:103870002B35CEE604122B3512E904122B353DEB25
:1038800004122B351AEF04122B3597EF04122B3547
:10389000D2EF04122B35F0EF04122B3550F0041246
:1038A0002B3578F004122B35A8F004122B35D9F003
:1038B00004122B3506F104122B355FF104122B355F
:1038C000AAF104122B35A4D704122B3520D80412E8
:1038D0002B3546D804122B357DD804122B35D6D97A
:1038E00004122B35F2D904122B3537DA04122B359A
:1038F000C7DA04122B351FDB04122B35F4DB04125C
:103900002B35D2DC04122B351CDD04122B357DDD6A
:1039100004122B3501DE04122B352ADE04122B355E
:103920006BDE04122B3519E004122B35E9E004128A
:103930002B35B0E104122B3583E204122B35BDE2A6
:1039400004122B3515E304122B3537E304122B3503
:10395000CBE304122B357EE404122B351AC9051271
:103960002B357FC905122B3526CA05122B355ECAA9
:1039700005122B35A9F101122B3554F201122B350A
:10398000F1F301122B356DF401122B35A5F4011260
:103990002B3590F701122B3522F901122B358CF9BA
:1039A00001122B35C4FC01122B3565FE01122B359B
:1039B000DFF405122B3507F505122B35F3F505124B
:1039C0002B3578A105122B35FBA105122B3512A240
:1039D00005122B3585A205122B35EBA205122B35CE
:1039E00014A305122B3599A305122B353BA4051200
:1039F0002B359EA405122B3503A505122B3523A5C7
:103A000005122B3553A505122B356FA505122B3545
:103A10009EA505122B35CEA505122B3504A6051241
:103A20002B3564A605122B35E1F104122B35B1F2CA
:103A300004122B35D6F204122B35F6F204122B3574
:103A40000AF304122B3572F304122B3596F3041289
:103A50002B3514F504122B353AF604122B351BF7CF
:103A600004122B357FF704122B35ABF704122B35DC
:103A70002FF804122B3580F804122B35A1F804120C
:103A80002B3519F904122B353EF904122B35A1F907
:103A900004122B3531FB04122B35FEFB04122B359F
:103AA00035FC04122B355AFC04122B357AFC041217
:103AB0002B35A0FC04122B35B4FC04122B351DFD54
:103AC00004122B3571FD04122B358DFD04122B359C
:103AD00097FD04122B35B8FD04122B350FC80412C4
:103AE0002B3529CB04122B3556CC04122B3531CE75
:103AF00004122B35BBCE04122B356FCF04122B359D
:103B000098CF04122B35CDCF04122B357BD0041265
:103B10002B350BD104122B357ED104122B3500D25C
:103B200004122B3503D204122B3506D204122B3586
:103B300009D204122B3529D204122B352CD20412AF
:103B40002B3545D204122B35A9D204122B359BD329
:103B500004122B35D0D404122B351DD504122B356D
:103B600024D604122B35F6D604122B357BAA031269
:103B70002B3507D702122B356ADB02122B353CDCC2
:103B800002122B35C3DC02122B35F4DC02122B356A
:103B900022DD02122B3576DD02122B35A4DD021256
:103BA0002B35C5DE02122B35F3DE02122B3521DF59
:103BB00002122B3557DF02122B3504E002122B358F
:103BC0002AE002122B3589E002122B3503E20212A1
:103BD0002B3540B303122B358EE302122B356BE4E9
:103BE00002122B35B5E402122B3504E502122B35F7
:103BF00070E502122B35D8E502122B3525E60212AC
:103C00002B3595E602122B35A6E702122B359AE8E2
:103C100002122B354BE902122B3580E902122B35AB
:103C2000D5E902122B3580EA02122B35AEEA0212D8
:103C30002B3533EC02122B35B8EC02122B35F8EC95
:103C400002122B3537ED02122B3550ED02122B35B7
:103C5000FFED02122B35B7EE02122B355EEF02128A
:103C60002B35F2EF02122B3598F002122B3502F1B0
:103C700002122B358DF102122B3520F202122B3558
:103C80003EF202122B3511F302122B35CFF3021242
:103C90002B3585F402122B3523F502122B35389B78
:103CA00005122B35799B05122B35E29B05122B351E
:103CB000039C05122B351C9C05122B35D69C051236
:103CC0002B35DF9C05122B35309D05122B35599D68
:103CD00005122B35709D05122B35D49D05122B3501
:103CE000669E05122B35979E05122B35F39E051205
:103CF0002B35599F05122B358D9F05122B3500A0B2
:103D000005122B3542A005122B3582A005122B354A
:103D1000BAA005122B35CCA005122B35DEA005125A
:103D20002B350FA105122B354FA105122B35C6B12E
:103D300005122B3509B305122B352FB305122B3580
:103D400040B305122B3558B505122B3577B5051242
:103D50002B35C8E805122B35FEE805122B3549E94D
:103D600005122B3595EA05122B35E3B304122B35DA
:103D700021B504122B355DB504122B3522B7041280
:103D80002B354CB704122B35D2B904122B3512BA8D
:103D900004122B35A7BB04122B353CBC04122B3567
:103DA0009ABC04122B352BBD04122B3563BD0412B3
:103DB0002B35A5BD04122B351FBF04122B35A8C00F
:103DC00004122B35DEC204122B350CC304122B3522
:103DD00038C304122B3541C304122B3597C3041288
:103DE0002B3527C404122B352EC704122B35B2C72E
:103DF00004122B3572FE05122B3588FE05122B3569
:103E000092FE05122B35E2FE05122B359EC00512DF
:103E10002B35B7C005122B355CC105122B359CC163
:103E200005122B35B5C105122B35E9C105122B350D
:103E300036C205122B356AC205122B35ACC20512EB
:103E40002B3582C405122B35EDC405122B355CF7DA
:103E500005122B35B1F705122B350AF805122B3553
:103E600010FF05122B3552FF05122B3594FF05125A
:103E70002B35A4FF05122B35069A04122B35619AB7
:103E800004122B35759B04122B35429C04122B35E2
:103E9000579C04122B35A19C04122B350F9D041244
:103EA0002B35229D04122B35669D04122B35D59D92
:103EB00004122B35ED9D04122B3549A004122B352D
:103EC0004FA104122B35AAA104122B359BA3041277
:103ED0002B351CA404122B3555A404122B35A0A499
:103EE00004122B35B6A404122B35C3A404122B35AF
:103EF000FCA404122B350EA504122B35ECA50412DC
:103F00002B35F7A504122B357CA604122B35D4A62D
:103F100004122B3520A704122B3559A804122B3577
:103F20008AA804122B3502AB04122B3533AB0412D2
:103F30002B3555AC04122B3584AC04122B35F6AC62
:103F400004122B3502AD04122B3536AD04122B357D
:103F5000A6AD04122B3583AE04122B35BCAE041271
:103F60002B35C6AE04122B35C9AE04122B35D3AE99
:103F700004122B35EFAE04122B356BAF04122B3528
:103F8000A4AF04122B35C0AF04122B35ECAF0412D2
:103F90002B3527B004122B3542B004122B354CB010
:103FA00004122B357BB004122B3591B004122B3543
:103FB000ADB004122B35DCB004122B35FCB004126A
:103FC0002B3545B104122B358EB104122B3598B226
:103FD00004122B3595FA05122B35A6FA05122B354E
:103FE0002FFB05122B35FDF703122B354CF803126E
:103FF0002B350AFA03122B35DDFB03122B351BFC84
:1040000003122B35F1FC03122B35F6FD03122B3571
:1040100018FE03122B3574FE03122B35F5FE031226
:104020002B35E84F00122B350A5000122B355C510E
:1040300000122B35A55100122B351E5200122B35C4
:10404000995200122B35025300122B35495300129E
:104050002B35BB5300122B355C5400122B35DB542F
:1040600000122B35175500122B356B5900122B35CA
:10407000795B00122B35AC5B00122B35F15B001223
:104080002B35FB5C00122B35E45F00122B357A6078
:1040900000122B35466200122B35796300122B3546
:1040A0008F6400122B35036500122B35CF6500128B
:1040B0002B35436600122B35466600122B35FD6604
:1040C00000122B35426800122B35866A00122B3500
:1040D000206D00122B35FE6D00122B353B6F001248
:1040E0002B35807200122B35907200122B35C7735E
:1040F00000122B35787400122B35C47500122B3545
:10410000327600122B35657700122B35BA77001204
:104110002B35008004122B35A78004122B35198112
:1041200004122B35298104122B35AB8104122B3557
:10413000028204122B35F78204122B351E830412DF
:104140002B35C38304122B35128404122B35708453
:1041500004122B35CB8404122B35A68704122B3581
:104160005F8804122B35C48804122B35578A041239
:104170002B35F78A04122B35908B04122B35ED8BDF
:1041800004122B35638C04122B355F8D04122B35F2
:10419000528E04122B35AB8E04122B35C18E0412B5
:1041A0002B35E28E04122B35218F04122B35B18F63
:1041B00004122B35F49004122B35B19204122B35D6
:1041C000FB9304122B35359504122B3540960412BF
:1041D0002B35E09604122B354F9704122B356C9833
:1041E00004122B35008005122B356B8005122B3500
:1041F000B38005122B351A8105122B3576810512F5
:104200002B35B18105122B354D8205122B35A78236
:1042100005122B35138405122B359A8405122B3584
:10422000D38405122B35028505122B357C850512AA
:104230002B35C48505122B35EA8505122B354187B0
:1042400005122B35468705122B35BD8705122B35F8
:10425000298805122B35248905122B35118A051260
:104260002B35A0AC05122B35DDAC05122B3576AD08
:1042700005122B3581AE05122B35C9B005122B3531
:1042800045B105122B3510DB05122B35C1DB0512AC
:104290002B3589DC05122B35DEDC05122B3561DD73
:1042A00005122B3584ED05122B3525FF03122B3516
:1042B00036FF03122B35D6FF03122B35EC7F00128D
:1042C0002B35EBFF02122B3588FB05122B3598FBA3
:1042D00005122B35B0FB05122B3564FC05122B356E
:1042E00091F905122B3516FA05122B357CFA0512B9
:1042F0002B3525FD05122B3528FD05122B3561FDCB
:1043000005122B35B4FD05122B35C6FD05122B35D4
:10431000C9FD05122B3518CD05122B3526CD0512FA
:104320002B359FCD05122B3574CE05122B3533D08E
:1043300005122B3598D005122B35FBD005122B35E5
:10434000F87F00122B35F8EA05122B3530EB0512F9
:104350002B3581EC05122B3505ED05122B3523E6A7
:1043600005122B35C4E605122B35F5E605122B3563
:1043700040E705122B3504E805122B3537E8051206
:104380002B355DE805122B356FE805122B3583E8D8
:1043900005122B3591E805122B3518A705122B3580
:1043A00044A705122B35EBA905122B3540AA05129F
:1043B0002B357CAA05122B3590AA05122B35A9AAFC
:1043C00005122B359CAB05122B3578AC05122B351D
:1043D0008CAC05122B350FF205122B3533F205127A
:1043E0002B354CF205122B358BF205122B35BEF214
:1043F00005122B35EEF205122B35F8F205122B358E
:1044000060F305122B3563F305122B356DF305129E
:104410002B357AF305122B357DE305122B35A5E3F9
:1044200005122B35E6E305122B3504E405122B3576
:104430001FE405122B3587E405122B3593E4051292
:104440002B35F2E405122B3516E505122B35D7E591
:1044500005122B35E4E505122B35F5E505122B3554
:10446000008006122B35188006122B353E8006126E
:104470002B350FB705122B3558B805122B355EB802
:1044800005122B3575B805122B3596B805122B354C
:10449000ACB805122B35C0B805122B353FB9051243
:1044A0002B35A4B905122B352CBA05122B35A5BA1C
:1044B00005122B357EBB05122B358EBB05122B3515
:1044C0009DBB05122B35D9FD05122B35FDFD0512BF
:1044D0002B3525FE05122B354DFE05122B35BEE082
:1044E00005122B352AE105122B3549E105122B3532
:1044F000AFE105122B35F5DD05122B350EDE051269
:104500002B3525DE05122B352EDE05122B354CDE24
:1045100005122B3556DE05122B3560DE05122B35C4
:1045200073DE05122B3500DF05122B356FDF051208
:104530002B359DDF05122B35EEDF05122B353AE0CA
:1045400005122B3555E005122B355FE005122B3592
:1045500070E005122B35B3E005122B35878006126B
:104560002B35D28006122B35E8F502122B3514F6C6
:1045700002122B3532F602122B3545F602122B357C
:1045800060F602122B35BFF602122B35EDF6021241
:104590002B35F9FA02122B353BFC02122B356DFC40
:1045A00002122B35D8FC02122B355CFE02122B3581
:1045B00084FE02122B3599FE02122B35A9FE02123F
:1045C0002B35E9FE02122B352BFF02122B353BFF58
:1045D00002122B3524F605122B3534F605122B3535
:1045E00052F605122B356DF605122B3594F6051291
:1045F0002B35B5F605122B35CFF605122B3507F7FF
:1046000005122B352AF705122B3571FC05122B35B7
:10461000B7FC05122B350FD105122B351FD1051212
:104620002B353DD205122B356FD205122B3591D289
:1046300005122B35B9D205122B35D2D205122B35E6
:104640000ED305122B3577D305122B35B3D30512B4
:104650002B35FAD305122B3527D405122B3553D41D
:1046600005122B3582F005122B35B9F005122B35CA
:10467000DFF105122B35E2F105122B357EF805121C
:104680002B35F0F805122B352EF905122B356FF965
:1046900005122B352F9305122B35359305122B352B
:1046A0007C9305122B35889505122B35B89505128C
:1046B0002B35229605122B35DD9605122B352497C6
:1046C00005122B35579705122B35E19705122B351F
:1046D000F89705122B35059805122B350F98051202
:1046E0002B35AF9905122B35A19A05122B35FF9A60
:1046F00005122B35B28A05122B35C88A05122B35C7
:104700007A8B05122B35A48C05122B35998D051249
:104710002B35308E05122B356B8E05122B35DD8E29
:1047200005122B353B8F05122B354B8F05122B3580
:10473000728F05122B35C48F05122B35339105125C
:104740002B35389105122B355A9105122B356BFFFD
:1047500002122B3599FF02122B35CEFF02122B3598
:10476000D0FF02122B35D2FF02122B35E3FF0212CB
:104770002B35E5FF02122B35E8FF02122B35F9EE3F
:1047800005122B3567EF05122B3589EF05122B35F6
:10479000C1EF05122B35F7EF05122B35E7D70512C0
:1047A0002B352AD805122B3548D805122B357BDA44
:1047B00005122B35AFDA05122B35DADA05122B3557
:1047C000AEFF05122B35697800122B354C7900129B
:1047D0002B35347A00122B35457A00122B35567A58
:1047E00000122B35A27A00122B35917C00122B354A
:1047F000EC7D00122B351C7E00122B35E77E00125B
:104800002B35447F00122B35FAC405122B3518C501
:1048100005122B355CC505122B3582C505122B35CB
:10482000A4C505122B35BCC505122B35D4C5051200
:104830002B35ECC505122B3592C605122B35D4C687
:1048400005122B35DEC605122B35F3C605122B35A6
:10485000FAC705122B3515C805122B351EC80512CF
:104860002B3527C805122B3530C805122B353AC811
:1048700005122B35B7C805122B35CEBB05122B35CB
:1048800013C005122B352FC005122B3534C005126D
:104890002B35A7D405122B35BDD405122B353ED6AA
:1048A00005122B3568D605122B35AFD605122B35E0
:1048B000B8D705122B3584F305122B35DBFF011217
:1048C0002B35C07F00122B3542A903122B3563A86C
:1048D00003122B358FA603122B3550A403122B3550
:1048E000EFA303122B3596A303122B351DA303123E
:1048F0002B35F3A203122B35E8A003122B35B8A0F9
:1049000003122B357CA003122B3568A003122B3524
:10491000D49F03122B35F29E03122B35249E0312D3
:104920002B35D39B03122B35A89B03122B35499BA8
:1049300003122B35BA9903122B35489903122B35E4
:10494000459903122B358D9703122B35449703128B
:104950002B351E9703122B355A9603122B35D4B2E2
:1049600003122B355EB203122B3522B203122B3504
:10497000D9B103122B3592B103122B35DCB00312DF
:104980002B3550B003122B35A49403122B354494CD
:1049900003122B35159403122B35129403122B3569
:1049A00041B003122B35FD9303122B35BD93031237
:1049B0002B35A49303122B35AE9203122B359DE2B7
:1049C00002122B356D9203122B352EAD03122B35AF
:1049D000FA9103122B35C79103122B356C910312F8
:1049E0002B353B9103122B35048E03122B35168D7C
:1049F00003122B35D08B03122B357E8B03122B35F4
:104A0000728B03122B35D98A03122B35A789031217
:104A10002B35F88603122B359B8403122B354F84DC
:104A200003122B35348303122B35C98203122B3525
:104A3000F38103122B35008003122B35AF81031253
:104A40002B356B8003122B35328003122B35CFD6DA
:104A50000200000080FB8F000100030987000100B5
:104A60000209240002007C10250002007E102600AE
:104A7000020080102700020082102800010084102C
:104A800029000100851084000400861086000100C2
:104A90008A102A0001008B102B0001008C102C00C2
:104AA00001008F102D000800EA082E000100901070
:104AB0002F00010091103000010092103100010020
:104AC000931032000100F20833000100F3083400B3
:104AD0000100941036000100F40838000100951020
:104AE000390001008E1083000200A710630001004E
:104AF000FF0864000100E108650001008D106D00F1
:104B00000100000971000800E20866000100A6101B
:104B10004300010097104400020098104500010076
:104B20009A10460002009B1047000800F708480052
:104B300001009D104B0001009E1004000100A9100F
:104B4000A1000100AB1037000100AA10880001008D
:104B500004093C000100F5083D00010096104900E1
:104B600002009F106700010001094D000200A11022
:104B70004E000100A3104F000200A4103E000100EF
:104B8000F6080000000000000001363601010001B7
:104B900002010001030100010401060605020000F4
:104BA000070100340801000F090401010D0100FF95
:104BB0000E08000017020000190100FF1A01000191
:104BC0001B0100FE1C0100081D0200001F01000166
:104BD00020010001210200002301000F2402000037
:104BE0002601000127010008280200FF2A01000712
:104BF0002B0102402C0100002D0100012E010001BB
:104C00002F0100FF30010B1C310800003A010008A1
:104C10003B01000F3C0100013D0100FF3E0400008C
:104C200042040000460400004A0400004E04000054
:104C300052040000560400005A0400005E20FFFFEA
:104C400036000100060000000F0000000000000018
:104C500000000000000003FFFF00000403FFFF004E
:104C600000FFFF0FF4010005C40403200001000051
:104C70000B000000000000000003010F0000000016
:104C80000000000000000000000000000000000024
:104C90000000000000000000000000000000000014
:104CA0000000000000000000000000000000000004
:104CB00000000000000000000000000000000103F0
:104CC0007103010301030103010301032203020332
:104CD00001031003000300030003000300030003AB
:104CE000000342030003240306030003000304033C
:104CF00012032503230325032303040304030003F2
:104D000000030003440300030003230300036503BF
:104D100021003503810300030503000300030003A2
:104D2000000325032303030071003001600011001C
:104D30007000310220035004800010006100000068
:104D4000140063007300720062004300000013004F
:104D50000600000000000400120000000000000037
:104D6000000004000400370037003C02440000004B
:104D70000000000000006500000035008100000018
:104D80000500000083000000010171010101010123
:104D900011010101310101010101800110016101D5
:104DA0003B001400630173017201620143010001C1
:104DB000130106013D01350004011201000100014B
:104DC0000001000104010401330133013C014401ED
:104DD000320136000001000165010001350081014A
:104DE000000105018201830100010302710230010B
:104DF000600211027002010202020202800210022D
:104E000061023A00410063027302720262024302CD
:104E10000002130238000002000204021202000223
:104E200000020002000204020402370037003C02C4
:104E3000440200023900000200026502000235024D
:104E4000810200020502820283020002030471044F
:104E50000204600411047004020402040104020448
:104E600010046104000414046304730472046204F3
:104E700043040004130406040004000404041204A0
:104E80000004000400040004510464000004000451
:104E90000004440400040004000400046504000449
:104EA0003504810464000504000483040004000048
:104EB00051411300C1400100514102004340030031
:104EC000494004004F400500554006006140300055
:104ED000854031007F4032009140330097403500DB
:104EE0009D403400A3403600A9401100B540140095
:104EF000BB40150073401F007940FFFF000001FD1B
:104F000031063332082D320B4B321067310A5D32D5
:104F10000203320521320709320CE5310DF131640B
:104F20006F2FFF000007ECFDFDFDECDCDCCCBCAC22
:104F3000AC9C9C8C7C7C6C6C5C5C5C4C4C3C3C2CE1
:104F40002C1C1C03EAF5E5D5D5C5B5A59595858539
:104F50007575656555554545353525251515050086
:104F6000160F00000B150B020002220F3300000E7B
:104F70000C0E020B040B0A0708000F00011916188B
:104F800016161823030000034A49434E181A250534
:104F900002303017181921301B1D1F303030161801
:104FA0001920231A1C1E3000393D3F373C3C362C5B
:104FB000442D02040201010101090200BE040A3C61
:104FC000003C007F00E803000000000E0009280CF0
:104FD00008100C030303080900040001FF1E1E0C47
:104FE000050508040415100AC082C083900816E461
:104FF000F0A3F07CD57D047A897B0712468B122FB3
:1050000075124A33122F7B026DA174F3122580743E
:10501000F5122C2A89098A088B0AE9705F740265E7
:1050200008703E9007A87408F0750C00780C122BDD
:1050300056ECF50C780C122B56EBF50C780C122B69
:105040005690108612298990108AE0F97CF77D0825
:105050009010A7126DB2122F9F7407122B8002516D
:105060001C74016508600302511F9007A87408F0C2
:105070007B00AA0AA90A122FDB02511C74016509E0
:10508000600974026509600302511FEA6006740337
:10509000650870409007A87402125140122DE61264
:1050A0002F8D9007AEE0A2E34010E9700D90081A32
:1050B000E004F06404700312514A74036508705CE4
:1050C00090081BE0F8740128F0E8C39405404D12E5
:1050D000514A80487401650870457401650990075C
:1050E000A8702E740AF07401122E15E4F0740212E6
:1050F0002E157403F004122E15E4F0A3F0A3F0A310
:10510000F07408122E15E4F0AA18AB1912320F80B1
:1051100025740A125140122DE6122FC3E960179030
:1051200080F01229897A017B009007A5E0F9123EF0
:10513000217404122B80740B122B807F050228052A
:10514000F090108AE0F990108622901086E4F0A387
:1051500074F8F0A374FFF0A37407F02274F612251C
:1051600080E9FFEAFE7AD1F9123CDD8A828B83E581
:10517000824583702A7A027B00123CBFEA4B700E94
:105180007A107B009007A5E0F9123D0180148A8215
:105190008B8374D1F0EFA3F0EEF9123CCB8003EFD8
:1051A000A3F00253B674F712258089089007021203
:1051B000746CFF901078E0F47003A3E0F470369004
:1051C0000719E0901078F0A3E4F080298E828F8395
:1051D000A3A312663560168E828F83A3A3A3E0F586
:1051E000838882A3126635FAA90812402B8E828F1B
:1051F00083127799FFEE4F70D3901078E0F470032C
:10520000A3E0F4600A901078E0FAA90812402B128B
:10521000331790077312591C1233110275A874F1D9
:10522000122580890A8C08750900750B00740F120D
:105230002E151262337411122E151259438049AE85
:105240000E1252EAF50CA3E0F50DAE0BEE2EFEE4C5
:1052500033FFEA2EF582EB126628650C7004A3E09A
:10526000650D7019AE09EE2EFEE433FFEC2EF582CB
:10527000ED3FF583E50CF0A3E50DF00509050EE51E
:105280000EC3950840B9050BE50BC3950A5005758B
:105290000E0080EBA909026CC774F4122580890BFB
:1052A0007D00740C122E1512623380010DEDC39532
:1052B0000B5032750A008002050AE50AC39C50ECC7
:1052C000ED25E0FEE433FFEA2EF582EB3F1252FAC1
:1052D000F509AE0A1252EA65087004A3E065097088
:1052E000D7790180027900026A6EEE2EFEE433FF68
:1052F000E82EF582E93FF583E022F583E0F508A387
:10530000E02274F612258012539D7003A3E06D70A5
:10531000177508AC7509077808122B52EEFA12417E
:10532000577402122B80801F750802750980780857
:10533000122B528C088D097808122B52125390129E
:10534000417B7404122B80806D74F61225801253F9
:105350009D7003A3E06D70177508B975090778088B
:10536000122B52EEFA12415D7402122B80801F75CF
:1053700008037509807808122B528C088D0978086B
:10538000122B5212539012417B7404122B808026F0
:10539000125CE7F583E0FD7C801266E122EAFEEB19
:1053A000FF1275AD1277AAFCE439FD900773E06C2B
:1053B000227402122B807F0202280574F6122580C7
:1053C00074FE122C2AEAFEEBFF851882851983E40D
:1053D000F0A3125B7312682BFBECFA88828983A31B
:1053E000A3E0F9750900750800600574FF69700590
:1053F000750882803D900773E06A7003A3E06B70CC
:105400001AAA18AB19123893E9F50985188285197B
:1054100083126A79701C7508838017900902E06016
:1054200004640170057508818008E06402700375EA
:105430000880851882851983125943A908EEFAEF6E
:10544000FB124163E5096011851882851983126A90
:10545000796006126DAC123D610253B174F21225EF
:1054600080EAFEEBFF750A00750B001254CE123372
:1054700017EA65087003EB650970121238A5E91484
:10548000F50A79017AE27B071238AB8003750B804D
:10549000126622F50C780C122B56750CE2750D076E
:1054A000780C122B52780A122B567808122B52E5E0
:1054B0000BF5087808122B561264F8126625F97A53
:1054C000057B801241697407122B800262411275BC
:1054D000AD1277AAF508E439F5092274F612258091
:1054E000E9FE7F0080298A828B831252FCF8E4C88F
:1054F000F9E50828E439F509EF25E0F8E433F9EC9B
:1055000028F582ED125CF0EA2402FA50010B0FEF4D
:10551000C39E40D20253B674E812258074FB122C4D
:105520002A8A168B17851882851983E4F074031272
:105530002E15E4F0A3F004122E15E4F0A3F012608F
:10554000693517125B45F50B850A82F5831277A63C
:10555000FEE439FF850A82850B83A3A3E0FA850A5E
:1055600082850B83A3A3A3E0F9EAF508E439F509E2
:10557000E50A2404F50A5002050BEEFAEFFB12339C
:10558000B3E964016016EEFAEFFB1233B3E9703D44
:10559000900773E06E7003A3E06F603112683312FE
:1055A0002B56E4F508F5097808122B527808122BCF
:1055B000569007731229917508807808122B56129D
:1055C00059221241697407122B800259121259494B
:1055D0008810602B1273AB123D5B7403122E1512F0
:1055E000591C7403122E15126A7960137403122E5B
:1055F0001512593BA91012405B8A0A8B0B80037568
:105600001000125949880F60271273AB123D5B746A
:1056100001122E1512591C7401122E15126A79608E
:105620000F7401122E1512593BA90F12405B800313
:10563000750F00900702805D850A82850B83A3A306
:10564000A3A3A3A3A3A3E4F0A3F0AA0AAB0B85141E
:1056500082851583A3A3125959126635F9123CCBE2
:10566000851282851383E0C0E0851882851983E066
:10567000F874E228F582E43407F583D0E0126A7DFD
:1056800004F0E511A2E05007AA12AB13123D6185A8
:105690001482851583E0F514A3E0F515E51445158E
:1056A000700302587F851482851583A3A312663583
:1056B00060DD851482851583A3A3A3A3A3A3A3A35D
:1056C000E0A2E050CA851482851583A3A3A3A31288
:1056D0006A79851482851583A3A3601F126635FA43
:1056E0007901851482851583A3A3A3A312663A12B8
:1056F00027668A128B13751101800F125959A3A3C3
:10570000E0F512A3E0F513751100E51245137003DF
:10571000025682851282851383A3E065087004A374
:10572000E06509600F74FF6508700474FF65096027
:1057300003025682851282851383A3A3A3A3A3A386
:10574000A3122991851282851383A3A3A3A3A3A3E4
:10575000E0FC7405122E15126DB2A91012403D74B2
:1057600002122B80E9703C851282851383A3A3A3C8
:10577000A3A3A3A3A3A3A3122991851282851383B4
:10578000A3A3A3A3A3A3A3A3A3E0FC7403122E15B6
:10579000126DB2A90F12403D7402122B80E9700302
:1057A000025682E50F2510C333240AFA7B00123C0F
:1057B000BF8A0A8B0BEA450B70030256608A828B04
:1057C0008374D2F0851682851783A3A31262338A6D
:1057D000828B83A3A3E8F0A3E91276B0A3E51012AD
:1057E00077B2E50FF0E510603CEA2405FAE4350BEA
:1057F000FBE50A240AF8E4350BF98A828B831260F0
:105800006E7403122E1512595E122B4EAC10EC2C36
:10581000FCE433FD8A828B83126DB2123C9B7403CD
:10582000122B80800D8A828B83A3A3A3A3A3E4F011
:10583000A3F0E50F7003025638A810E828F8E43307
:10584000F9E50A28F8E50B39F9E8240AFAE439FB06
:10585000850A82850B83A3A3A3A3A3A3A3A31259A1
:105860001C7401122E1512595E122B4EAC0FEC2C2B
:10587000FCE433FD123C9B7403122B8002564A85D4
:105880001882851983E06027126833122B56750839
:10589000E27509077808122B527403122E1512684C
:1058A0003C122B569007731229917508008029EE3F
:1058B000FAEFFB1233B3E9702F126833122B5675CF
:1058C00008E27509077808122B527508007808124B
:1058D0002B569007731229917808122B56125922D1
:1058E0001241697407122B807403122E15126A7903
:1058F000600B7403122E15126DB2123D6174011209
:105900002E15126A79600B7401122E15126DB212E7
:105910003D617405122B807F10022805EAF0A3EB8D
:10592000F022E5162402FCE43517FDE51612648921
:105930003517F583E0F97A067B8022125943AA0ACB
:10594000AB0B22E0FCA3E0FD22850A82850B83E0FD
:10595000F8A385820A85830B2212663AA322E0F51A
:105960000CA3E0F50D750E00780C2274F112258061
:1059700074F4122C2A8A088B09ECFEEDFF740B12CA
:105980002E157403F0122BEE12468B123311EAFC23
:10599000EBFD7403122BEE124685E9600FEE241323
:1059A00012662564036010E06401600B851882852F
:1059B00019837484025AFD8E828F83A3A3A3A3A3A9
:1059C000A3A3A3E06018F46015EE24131266256407
:1059D000037016EE24141266256003F4700B85180C
:1059E000828519837482025AFD127558E064217011
:1059F00002A3E06003025AD4851882851983748C4F
:105A0000125B7364036003025ABE7401122BF61218
:105A1000620D1249C1E96003025ABE123FBF8A0AF1
:105A20008B0BEA450B7003025AFE8E0C8F0D750E20
:105A300000780C122B4E7C157D00123C9B740312D7
:105A40002B80850882850983A3A3E50A2415FCE43D
:105A5000350BFD7409122AAE1271B9C0E0E50A24B3
:105A60001EF582E4350BF583D0E0126074C0E0E5EA
:105A70000A241FF582E4350BF583D0E0F0E50A2413
:105A800020F582E4350BF5837405F0EE240BFE500F
:105A9000010FFAEFFB12394D7D007C007900EEFA20
:105AA000EFFB1241219080F01229897A007B10903F
:105AB00007A5E0F9123E217404122B808078125B56
:105AC0003B122B56125B4D1249D97401122B80E9FF
:105AD000702C8014125B3B122B56125B4D1249D373
:105AE0007401122B80E9700D851882851983E4F00A
:105AF000123F8F80098518828519837488F012718E
:105B0000B9F50A780A122B567401122BE6880A8915
:105B10000B780A122B52E508240CF582E4350912A1
:105B20005B454480F50B780A122B521265BA12417C
:105B3000157405122B80740C026CC4EE126220E006
:105B4000F50A780A22F583E0F50AA3E022EE240B99
:105B5000FCE43FFD8E828F83A3A3A3A3A3A3A3A3EF
:105B6000A3126DEF8E828F83A3A3A3A3A3A3A3A3EA
:105B7000E0F922F01276F3E022C082C08374F312BF
:105B80002C2A851882851983E4F004122E151259E7
:105B90001C7403122E15AA82AB83122E9DAA18AB79
:105BA00019122ED3740D122B80026DA174F61225DA
:105BB00080EAFEEBFF12622D88828983127560F8FD
:105BC0009007B4E058F508A3E059F509E508450940
:105BD000601C7808122B52900773122991126622CA
:105BE000FD7C001266DD1241757404122B80025395
:105BF000B674F412258074FF122C2AEAFEEBFF859E
:105C00001882851983E4F09008F6E06021EE240BF9
:105C1000126625640160178E828F83A3A3126233FC
:105C2000EE2415126625687003A3E0696003025C28
:105C3000E212622DE8FAE9FB88828983A3A3A3A379
:105C4000A3A3A3A3E0FC88828983A3A3A3A3A3A304
:105C5000A3A312774BEC28F508E439F509EC4509C4
:105C60006010EC9471E994085008900902E0640215
:105C7000700A85188285198374808038122F0F8AE4
:105C80000A8B0BA80AA90BE849602188828983A3A3
:105C9000A3A3A3E06016C394035011E82412125C7E
:105CA000EDE82414125CED123F8F8009851882857F
:105CB00019837481F0125CE712683A122B56740152
:105CC000122BE6880889097808122B5275081F756F
:105CD00009807808122B521264EE124115740512D5
:105CE0002B807401026A6BEE1275833F22F582E409
:105CF00039F583E508F0A3E509F02274EA1225805E
:105D000074DB122C2A8A148B15751200751300127D
:105D1000662DF50EAC18AD197A007B00799C122F18
:105D2000ED7A047900122EE5EAF50C8518828519C2
:105D300083E02AF0F8E50EC3984003025F1AE0C33F
:105D4000950EF509C394044003750903E50975F040
:105D50001AA4FAABF0123D5B8A128B13EA4513705A
:105D600003025F1D750D00AE12AF13850E08807E15
:105D7000125F85123CA7850A82850B83A3A3A3A388
:105D8000E0702D850A82850B83126A79700C126E81
:105D9000FCF0EE2418126EFF8010125F93F0900555
:105DA00064E014C0E0125F6DD0E0125FBEE48034A6
:105DB000900564E004C0E0125F6DD0E0125FB6C3EE
:105DC0009403EE4003025E8112621C7402125FB6FD
:105DD00064017003025E8EEE2415125F96F0EE24CD
:105DE00016125F96F0EE241AFE50010F050DE50D18
:105DF000C395094003025EB9E508C3950C40030250
:105E00005E9785080AAA0A7B00122F578A0A8B0B15
:105E10000508900551125F9F12468B850A82850BFB
:105E200083126233125F7BE8F0A3E9125FD0850A28
:105E300082850B83A3A3A3A3A3A3A3A3A3A3E0C0CF
:105E4000E0125F63D0E0F07401122E15E4F0850AD1
:105E500082850B831262337402122E1512606E74E7
:105E600001122BEE122EC1E964016003025D707411
:105E700004122E15AC82AD83125F8B12468B025D2D
:105E800076125F94125FB664036003025DD7EE245E
:105E900015126EFF025DDDE50CC3950E4005750819
:105EA00000801DE50EC3950CF5088014125F93F079
:105EB000EE241AFE50010F050DE50DC39509505D46
:105EC000740E122BF685080AAA0A7B007987122F16
:105ED000ED05087418122E15125F9F12468B125F83
:105EE00085123CA7EE2412F8E43FF9740E122E1529
:105EF000126DB288828983EAF0A3EB125FBE74034D
:105F0000125FD0741D122E15E0C0E0125F63D0E066
:105F1000126D197097126EFC8095750900750A0054
:105F2000780A122B567812122B527809122B56E54A
:105F30000EF5097809122B567405122E15E0FD7C1A
:105F4000001264751241B17405122B80E5124513DD
:105F50006007AA12AB13123D617425122B807F0ECD
:105F6000022805EE2419F582E43FF58322125F71C1
:105F700022EE2418F582E43FF58322EE2412F58206
:105F8000E43FF583227C087D0079FFEE240AFAE4E1
:105F90003FFB22EE2414F582E43FF58374012212C4
:105FA00062378E828F83E8F0A3E9F07C657D05EE91
:105FB0001266F83FFB22127706A3A3A3E022F0EEBD
:105FC000126EF37402F0EE2416F582E43FF583229C
:105FD000F0EE2417F582E43FF5837402F0125F714E
:105FE00074FFF02274F612258074F9122C2A8A08A4
:105FF0008B091260693509127833123CB3EAF8EB69
:10600000F9ECFAEDFB851882851983122DFEEE243A
:1060100004FE50010F8E828F83E0C0E07404122EC4
:1060200015D0E0126CF0FA7405122E157401F0749C
:1060300006122E157401F090077DF0900786041269
:10604000771DA312623390077E12606EEA90078775
:1060500012607490077CF0AA18AB19122F93E960B4
:1060600003122F9974070253B3EA12745F22E8F007
:10607000A3E9F022F012768AE02274F212258074ED
:10608000FF122C2A7508007E007F0012323F8A0A18
:106090008B0B12323F8A0C8B0DA80CA90D800805C2
:1060A00008126215126231E84970F4900902E0604A
:1060B000076401600302618A12323F8A0C8B0DA8CB
:1060C0000CA90D8006126215126231E8496035880C
:1060D000828983126DB2900551E06A7003A3E06B70
:1060E000600C126215F583126DB2EA4B70D788828C
:1060F0008983126233900551E0687003A3E06970F0
:106100000302618A7A167B00123D5B8A0C8B0DAE0E
:106110000CAF0DEE4F60739005511262338E828F7B
:106120008312606E900546E08E828F83A3A3F012E7
:10613000339BE98E828F83A3A3A3A3A3F090108B3C
:106140001276FAF07C657D0512620D12468BAA1854
:10615000AB197941124811851882851983E06008CE
:10616000900773126233800478FE79FF8E828F83EA
:10617000A3A3A3A3A3A3A312606E12621BE50AF05C
:10618000A3E50BF08E0A8F0B0508900787E0F8E572
:1061900008C39850047A008022E508C398FAC39493
:1061A0000640027A057900800DE50A126227350B58
:1061B000125B45F50B09E9C39840EE7509007809B3
:1061C000122B56780A122B52EAF5097809122B562F
:1061D000900787E0F5097809122B56AD087C007A04
:1061E0007E7B0790077CE0F91241AB7405122B808F
:1061F000900902E060046401700BEE4F6007EEFA54
:10620000EFFB123D61122F9974010254C8EE240B6A
:10621000FAE43FFB22E81262273922EE12622022C2
:106220001262273FF583222414F582E42212745E61
:106230003FF58312623722E0F8A3E0F922EEFAEF8D
:10624000FB7F0602280574EC12258074FF122C2AAD
:106250008A0A8B0B7E008E0E8E0F126069350B1230
:106260006633FFAC18AD197A007B00799D122FEDD3
:10627000851882851983E0F8EFC3984003026321F3
:10628000E0C39FFEC3940B40027E0AEE75F007A4A4
:10629000FAABF0123D5B8A088B098A0E8B0FEA4538
:1062A0000F607C750C00801A850882850983A3A382
:1062B000A3A3A37403F0E5082407F5085002050919
:1062C000050CE50CC39E5059AC08AD09850C10E5D2
:1062D000102FFAE43400FB798B122FED85088285AC
:1062E0000983A3A3A3A3A3E014600814601314609C
:1062F0001F80B5850882850983A3A3A3A3A3E48097
:10630000B4850882850983A3A3A3A3A3740180A5F0
:10631000850882850983A3A3A3A3A3740280967E24
:10632000007508007808122B56780E122B52EEF5E5
:10633000087808122B56EFF5087808122B567405CA
:10634000122E15E0FD7C00E50A1266F8350BFBE520
:106350000A126489350BF583E0F91241B77405120E
:106360002B80E50E450F6007AA0EAB0F123D61743E
:1063700001122B807F0C02280574EA12258074FE1E
:10638000122C2A8A148B15750A00750B0012662DC3
:10639000F508AC18AD197A007B0079A31249CD85B8
:1063A000080C851882851983126233C3E50C98E4C2
:1063B00099507D851882851983E0C3950CFEA3E072
:1063C0009400FFC3EE9404EF940040067E037F0028
:1063D0008004EE4F605AEEFAEFFBEA75F015A4FA6E
:1063E000A8F075F015EBA428FB123D5B8A0C8B0D11
:1063F0008A0A8B0BEA450B6037750900750E00851C
:106400000E10C3E5109EE49F502BAC0CAD0D850E15
:1064100012850810E5122510FAE43400FB79A21267
:1064200049CDE50C2415F50C5002050D050E80CF65
:1064300075098B7E00750C00780C122B56780A12A9
:106440002B52EEF50C780C122B567808122B567442
:1064500005122E15E0FDAC091264751241BD7405DC
:10646000122B80E50A450B6007AA0AAB0B123D61AF
:106470007402025F5BE5141266F83515FBE5141231
:1064800064893515F583E0F922240FF582E422743E
:10649000F612258074FF122C2A1264E51275A0A34F
:1064A000A3A3A3A3A3A3A3E0F9122FB7E98518829E
:1064B000851983F07508007808122B567401122B89
:1064C000E6880889097808122B5275083575098005
:1064D0007808122B521264EE1241157405122B80AB
:1064E00074010253B3EAFEEBFF12745E3F2279019E
:1064F0001264F8FAE43FFB22EE2402FCE43FFDEED6
:10650000240F2274F412258074FA122C2A8A088B24
:1065100009EA12745712746CFFEEFAEFFB122EA305
:10652000E96013123311EAFCEBFDEEFAEFFB1246C1
:1065300085E96401700A7401122E15E4F0A3800944
:106540007401122E15EEF0A3EF127739A3A3A3A3C3
:10655000A3E0F8A2E650087403122E157401F0E8C7
:10656000A2E750087404122E157401F07405122E5F
:1065700015E4F004122BEE122FE1E985188285193B
:1065800083F07A007B00123335750A00780A122BEB
:10659000567401122BE6880A890B780A122B527561
:1065A0000A34750B80780A122B521265BA12411503
:1065B0007405122B807406026A6B7901E5082402C7
:1065C000FCE43509FDE508240FFAE43509FB2274E3
:1065D000F612258074FF122C2A1264E5126633F934
:1065E000122FA5E9851882851983F0EE240B126617
:1065F00025702C7508007808122B567401122BE6B2
:10660000880889097808122B527508367509807830
:1066100008122B521264EE1241157405122B8002DF
:1066200064E0EE240EF582E43FF583E022EA127482
:106630005F3515F58312663AE022E0F8A3E0F583B2
:10664000888222022B3274F412258074EF122C2AD5
:10665000EAFEEBFF1254CE900773E065087004A3C6
:10666000E065097052A818A919880A890B780A12DE
:106670002B52750A11750B00780A122B527C007D83
:10668000007A817B00123DE57404122B80E97027AB
:10669000750A00780A122B567401122BE6880A89B3
:1066A0000B780A122B52AC08AD091266DD12416F4D
:1066B0007403122B808021750A11750B80780A12E1
:1066C0002B527808122B52126622FD7C841266DD52
:1066D00012417B7404122B807411026A6B1266E102
:1066E00022EE1266F83FFBEE240FF582E43FF583BD
:1066F000E0F922FCEFFDE5082402FAE42274F1122D
:10670000258074EB122C2AEAFEEBFFEE24131266AE
:106710002512682BFAE4CAFBEC2AF508E43BF509DC
:10672000900773E065087004A3E0650960030267E1
:10673000D388828983A3A3E09410500F8882898331
:10674000A3A3E0851882851983800885188285199E
:10675000837410F0E0C0E07404122E15D0E01275BE
:1067600091A3A3A982AA83890C8A0D750E00780CC7
:10677000122B4E7407122E15E0FC7D007408122EA9
:1067800015AA82AB83123C9B7403122B80740412F3
:106790002BE6880A890B780A122B52750A11750BA1
:1067A00000780A122B527C007D007A817B00123D1A
:1067B000DF7404122B807404122E15E09007AC6075
:1067C00005E0D2E48003E0C2E4F0851882851983F5
:1067D000E480088518828519837484F0E0C0E07431
:1067E00001122E15D0E0F07402122E15E508F07497
:1067F00003122E15E508F0125CE712683A122B56C8
:106800007402122BE6880889097808122B52750841
:10681000147509807808122B5279031264F0124122
:10682000157405122B807415026CC41275B4E0FC4B
:10683000A3E022E5161275833517F583E0F5087895
:10684000082274F412258074E0122C2A8A088B091D
:10685000AC18AD19124103900902E0640270337460
:1068600002122E15AE82AF83123311EEFCEFFD1231
:106870004685E9601D1233178A0A8B0BA80AA90BFB
:10688000851882851983E0687003A3E069700302AC
:106890006A691234CD7402122E15126DA81233E3F8
:1068A000E964017003026A697418122BEE12332333
:1068B0007402122E15AC82AD837418122BEE1246A0
:1068C00085E9603212331D8A0A8B0BA80AA90B8551
:1068D0001882851983E0687003A3E0696018851841
:1068E0008285198312623390054712606E7A477B66
:1068F00005794B124817900902E0600764016003B4
:106900000269A712737DC082C0831233178A088B75
:1069100009D083D082E065087004A3E06509605C5B
:106920007402122E15AA82AB83122F0F8A088B09CC
:10693000A808A909E849602688828983A3A3A3A39C
:10694000E06401600D88828983A3A3A3A3E06402AD
:10695000700C7402122E15AA82AB83122F1B9005A5
:10696000E5126A7960169008F6E06401700E126D07
:10697000AC9005E6E0F58388821227661233178A09
:10698000088B09A808A909851882851983E0687011
:1069900003A3E06960117402122E15126DA8122E65
:1069A000F1E96003123F8F7402122E15126DA812C6
:1069B00034BB7900126DAC123131740B122E15E418
:1069C000126A7DF8A3E0F9740C122E1512606E7431
:1069D0000B122BEE122EC1E9603F7C087D0079007E
:1069E0007418122BEE123CA7740E122E15AC82AD49
:1069F000837418122BEE124685E9601D7402122E64
:106A000015AC82AD83740E122E15AA82AB83122EA2
:106A10009D740B122BEE122ED37402122E15AC8223
:106A2000AD83740E122E15AA82AB83122E9D740BA9
:106A3000122BEE122EC7E96030740C122E15126262
:106A400033851882851983E0687003A3E0696019B3
:106A5000851882851983126233740C122E15126008
:106A60006E740B122BEE122ED37420122B807F0427
:106A7000022805F582E438F583126F3322F0851879
:106A800082851983E02274F112258074F6122C2A73
:106A9000EAFEEBFF750800900818126A7970507AC8
:106AA000377B00123D5B900818EAF0A3EB12726886
:106AB00060197C377D007900123CA7EEFCEFFD9059
:106AC0000818126DB21240D3E9700B85188285192F
:106AD000837488026C2D127564126CCC7401F07C86
:106AE000DF7D409004D3126DB2124A39026CC2E0CD
:106AF000C8126CCC7402F0EEFCEFFD1271BE1240B5
:106B0000D3E9700C8518828519837488F0750801A3
:106B1000750AE2750B07780A122B52126DC2122900
:106B20009112756424281271B1FC126DF51275640E
:106B300024141271B1F91240377404122B80126CB4
:106B4000D9126CF624311271B16043127252FAE418
:106B500033FB123D5B900818E02432126D0B60226B
:106B6000750CE2750D07750E00780C122B4E127223
:106B700052FCE433FD126DE0123C9B7403122B8037
:106B8000800C8518828519837488F0750801780A4D
:106B9000122B52126DB612299112756424111271C2
:106BA000B1FC126DD7127564242B1271B1F9124029
:106BB000377404122B801275642434126CF624345A
:106BC0001271B16035127249FAE433FB123D5B90E9
:106BD0000818E02435126D0B6042750CE2750D0744
:106BE000750E00780C122B4E127249FCE433FD1224
:106BF0006DCE123C9B7403122B80E508A2E0402569
:106C0000126CD91271B170089008181272156015C3
:106C10007B007A0079001240D9026CC28518828507
:106C200019837488F08518828519837486F0740935
:106C3000122E1574021273C1126CE8122E15E8F0B0
:106C4000A3E9126CF0F5087808122B567401122B88
:106C5000E6880889097808122B5275082075098082
:106C60007808122B5279017406122BF6EEFAEFFB1C
:106C70001241157405122B801272047042740912AD
:106C80002E157402F0126CE2122E1512726F122B76
:106C9000567401122BE6880889097808122B527560
:106CA00008207509807808122B5279017406122B7E
:106CB000F6900818126DB21241157405122B80124D
:106CC00040CD740A122B807F07022805126CD02257
:106CD000242EF582E438F583229008181271DA2404
:106CE000312290081812663AA3A312623774012267
:106CF0001273C1A3E022F582E438F583126D01C856
:106D000022E9F0900818E0F8A3E022F8A3E03400AC
:106D1000F988828983EAF0A3EB12759A126F332205
:106D2000C082C083900818126A796075E0C8243563
:106D3000126A736006126DCE123D611275642432C0
:106D4000126A736006126DE0123D611275642412BE
:106D5000126A736009126DB6126DB2123D6112753E
:106D6000642415126A736006126DF5123D61127586
:106D7000642429126A736009126DC2126DB2123D49
:106D800061127564242C126A736006126DD7123D6D
:106D900061900818126DB2123D61900818E4F0A3DA
:106DA000F0D083D082022B32AC82AD8385188285ED
:106DB0001983126DEF221271D72412F582E438F58F
:106DC00083221271D72429F582E438F583221271C7
:106DD000D72435126DE9221271D7242C126DE922C5
:106DE0001271D72432126DE922F582E438F583E07E
:106DF000FAA3E0FB221271D72415126DE92274F177
:106E0000122580EAFEEBFF8C088D09750A018C0CB7
:106E10008D0D750E00780C122B4E7C177D00123CE8
:106E20009B7403122B80EE2412126EFFF0A3F0EE7F
:106E30002415126EFFF0A3F012737DE0603AEE2489
:106E400012F8E43FF9880C890D1273A6123D5B120B
:106E50006F206021E5082412126F13122B4EE508F3
:106E60002411126F07125F7C126DB2123C9B7403E7
:106E7000122B808003750A00E50812738B6035EED3
:106E80002415F8E43FF9880C890D1273A6123D5BB6
:106E9000126F206055E5082415126F13122B4EE572
:106EA000082414126F07126EEF126DB2123C9B741D
:106EB00003122B80E50AA2E0402BEE2412F582E4B7
:106EC0003F126A776009125F7B126DB2123D61EE6C
:106ED0002415F582E43F126A77600AEE126EEF1213
:106EE0006DB2123D61A90A026CC7750A0080CB120F
:106EF0006EF3222415F582E43FF58322EE2414F587
:106F000082E43FF583E422127550E025E0FCE4338F
:106F1000FDEE22127550E0F50CA3E0F50D780C2281
:106F2000850C82850D8312591C850C82850D831278
:106F30006F3322E0F8A3E0F9E8492274EE122580CD
:106F400074ED122C2A890A8A0E8B0F750C00750DB0
:106F500000750BFF7510FF7511FF750800750900AE
:106F6000851882851983E412726860177403650AB4
:106F700060067402650A7010E0C824301271B165B1
:106F80000F600579000271A77CDF7D407A007B00ED
:106F9000124A397401650A700A851882851983744A
:106FA00085803DE50A60067403650A70199008182B
:106FB0001271E4F07403650A7029E50E60298518E2
:106FC00082851983801A7402650A701BE50E900889
:106FD0001870051271E480081275671271FB740253
:106FE000F08004E50A601E1271EA701912720E60D8
:106FF00005126CDC800A127215600A127564243462
:107000001271B114F012720E60221252FCF50912C4
:107010007252F8E433F9900818E0FAA3E0CA243277
:10702000127226241D1271CB2425802E1272156037
:107030002E900818E02417F508A3E03400F5091293
:107040007249F8E433F9900818E0FAA3E0CA24354D
:1070500012722624061271CB240E1271B1F50B7434
:1070600009122E157402126A7D6003027115E5087B
:10707000450970030271151271EA70047E228002C4
:107080007E21850882850983126CE8122E15126014
:107090006E90081CE0C0E01275642430F582E4387C
:1070A000F583D0E0F07412122E157403F0AC0CAD21
:1070B0000D740A122BEE12468B850882850983A374
:1070C000E0F50C780C122B56780B122B56740C1220
:1070D0002BE6880C890D780C122B527810122B524B
:1070E000E5082406F50CE43509F50D780C122B5251
:1070F0001271B9F97409122BF6EEFA7B001241876E
:107100007408122B807CDF7D409004D3126DB21284
:107110004A390271A5126CE2122E1512726F122BEF
:10712000567401122BE6880889097808122B5275CB
:1071300008207509807808122B5279017406122BE9
:10714000F6900818126DB21241157405122B8012B8
:107150007204704E1275642419F582E438F58312B6
:107160006CEA122E15E8F0A3126CFC2418F582E4E8
:107170003812683A122B567401122BE688088909D6
:107180007808122B527508207509807808122B5246
:1071900079017406122BF61271BE12411574051294
:1071A0002B801240CD79017413122B807F0A0228A4
:1071B00005F582E438F583E02212769AE022900801
:1071C00018E02417FAA3E03400FB22F50CA3E03406
:1071D00000F50D1271D7229008181271DE22E0F826
:1071E000A3E0C8221271F47401229008181271F4FD
:1071F000E06401221271DE1271FB22242FF582E479
:1072000038F583221271D7126CD0E0640222127218
:107210005890081822127219221271DE2434F58255
:10722000E438F583E022F582E43AF583E028F8A318
:10723000E039F9E824FEF582E934FFF583E0F51042
:10724000A3E0F511900818E0229008181272192591
:10725000E02212725825E0229008181271DE2431C3
:10726000F582E438F583E022126D02F9E84922E85C
:10727000F0A3126D01F5838882A3E0F50878082257
:10728000C082C0837B007A8579011240D9026DA14A
:1072900074F41225808C088D09EA240F12773F12AE
:1072A00076A41262338C828D83A3A312606EEA24CB
:1072B0000E12773FA3F01274631273B212757650F8
:1072C000010FFCEFFDE5082406FAE43509FB124640
:1072D0008BEE2408FE50010F8E828F83E0C0E012F7
:1072E0007696D0E0127471F8127686E812757A50AC
:1072F000010FE5082412127385A3F0E50824151286
:1073000073851273BBA30EAF83C0E012737DD0E010
:10731000F06028E508241212739D123D5B1277522B
:107320006019E508241212739012737FE0F912407D
:107330005B8A0A8B0BAE0AAF0B8007E5082411129B
:1073400073858E828F83E0A3AE82AF83C0E0127418
:1073500049D0E0F0601FE508241512739D123D5BD3
:107360001277526010E508241512739012738BF98E
:1073700012405B8005127449E4F0026A6EE508244D
:107380001112755022127550E4F02212744FE0224F
:10739000127550125943EEFAEFFBE50822F8E43576
:1073A00009F9880A890BE01273AB2225E0FAE4336D
:1073B000FB22FF1276768C828D8322A31273C1E0AA
:1073C00022F08E828F832274F61225808C088D091C
:1073D000127463FFEEFCEFFDAA08AB0912468BEEB8
:1073E0002408FE50010F8E828F831277A0127471D1
:1073F000850882850983A3A3A3A3A31275765001F0
:107400000F8E828F83E0F8E508127457E812756BCF
:107410007403687026EEFCEFFDE508240BFAE435F2
:1074200009FB12468B8E828F83A3A3A3A3A3A3A3DE
:10743000A3E0C0E0127449D0E0800A12766F1275A2
:107440004AE8F0A3E9F00253B6E50812744F22129D
:1074500062273509F5832212745F12755322EE12EA
:1074600075BE2212771712746A22F583E0FEA3E03C
:10747000221276C512767A2274F2122580EAFEEB89
:10748000FF750A00EE2410126625C3940C400D12FD
:1074900076EF127567240B1271B1F50AA80AE82875
:1074A000F8E433F9E8240DFAE439FB123D5B8A086D
:1074B0008B09EA450970030275411264E91276DE10
:1074C0008A828B831276C17078EEFCEFFDEA24038A
:1074D000FAE43509FB12468BEE2408FE50010F8EAC
:1074E000828F8312756085088285098312757950B1
:1074F000010F127548E4F0E50A6046E508240DF82E
:10750000E43509F98E828F83E0C0E0127548D0E03F
:10751000127681C0E0127558D0E012756B850A0BA7
:107520008E828F83E0FCA3E0FBEC88828983127556
:1075300089500109EE2402FE50010F150BE50B7076
:10754000DFAA08AB09026241E508240B127550223C
:10755000F582E43509F58322E508240C12755022E2
:1075600012767A229008181271DA2212756F22129E
:1075700076CD0EAF8322A3A3A3A3F0A3E9F0EE245C
:1075800002FE22240EF582E42212591DE82402F89C
:10759000221275952212759AA322F088828983227D
:1075A000126DED8A828B83227F010228051275BD40
:1075B0003FF583E0F8A3E0F98882898322EE241363
:1075C000F582E42274F21225801277131252FA85A2
:1075D0000882F583E0F50DA3858208858309A3A3BE
:1075E000E0F50C1276D93400FB123D5B8A0A8B0B56
:1075F000AE0AAF0BEE4F60378E828F83E50DF085BC
:107600000882850983E0FA12772685088285098336
:10761000A3A3A3A982AA8389088A09880A780812E1
:107620002B4E1276D43FFB123C9B7403122B80022C
:10763000623D74F7122580EA2413F8E43BF988824E
:107640008983E0FAA3E0F5838A8212774512766A8D
:107650001275B4A3E0FA88828983A3A3E0F9EA8CC7
:10766000828D83A312606F0275A812759AE02212B0
:10767000767AF8E508228E828F83E0FAA3E0F9EAB1
:107680002212756FE02212768A22E508240FF58215
:10769000E43509F5832212769A22E50812758335BE
:1076A00009F583221276A9A322F08A828B83A32272
:1076B0001276B422F08A828B83A3A3A322A3A3A36E
:1076C000A31276C5221276CDAE82AF8322F08E82CF
:1076D0008F83A322AC0C7D00EE2404FAE422127600
:1076E000E222F583E0FEA3E0FF8E828F83E0221288
:1076F00076F3221275BD3FF58322E08E828F83A33D
:10770000A3A3A3A3A322F0850A82850B83A3228CC3
:10771000088D0912771722EA1275BE3B22F0850800
:1077200082850983A32212774BEA8E828F83A3F08E
:10773000A3E9127739E50CF0221276CDA3A322F546
:1077400082E43BF583E08C828D8322A3E0F8E4C8D9
:10775000F922850A82850B8312591C850A82850BC2
:1077600083126F332274F612258012770FF583127D
:1077700077991273B212757A50010F1266F33509B8
:10778000FB12468B8E828F83A3A3A3A3A3A3A3A3E1
:107790001277A0A3A3F00253B6126237E8FEE922E3
:1077A000127846A3A3221277AA22E0FA12774BEAB4
:1077B00028221276B4A3A3A3A32274F61225801262
:1077C000770F127833123CB3EAF8EBF9ECFAEDFBE1
:1077D000850882850983122DFEEE2404FE50010FD8
:1077E0008E828F83E08508828509831276BDC394DB
:1077F00006500512784B8037850882850983A3A33C
:10780000A3A3E064FE600E850882850983A3A3A379
:10781000A3E0F4701B12783E12756B85088285090F
:1078200083A3A3A3A3E0F47007127858F0A3E9F0B0
:107830000253B612746AFF7904EEFAEFFB228E82CD
:107840008F831278462212784BA322E08508828526
:107850000983A3A3A3A3A3221276768508828509B0
:1078600083A3A3A3A3A3A3A32274F6122580127E4D
:10787000DC6003027945A3A3E06003027945A3E03D
:1078800064027002A3E06003027945901008E024CE
:1078900080600914605214605F02794590100CE01A
:1078A0006003027945901002E0600478018002785C
:1078B00000901010E8F0A3E4F0901001E0600A904E
:1078C0001010E04402F0A3E4F0900FF6E0640460CE
:1078D000149010037410F0A37410F0A3E4F0A374D8
:1078E00002127F3BF0027FBB900FEFE06404705503
:1078F000901010E4F0A380D090100CE0547FF508B5
:10790000900FEFE06404703DE508C3940650369094
:10791000100CE05480601C74F62508F582E4340FE6
:10792000F583E06403700478018002780090101001
:10793000E8809274FB2508F582E4340FF583E06457
:107940000370E880E2900FF67404809874F61225B4
:1079500080E9FE90100E127EDF6003027A29900FFC
:10796000EFE06404600B90100C127EDF6003027A7B
:1079700029901008E0541F60091460301460200240
:107980007A2990100AE064017022EE901001F060F4
:10799000047905800279067A0012476F027A2F90E7
:1079A000100CE0547FFA90100AE060057900027A2A
:1079B00031EAC394065072EA90620EF090100CE027
:1079C0005480602FEE600474108002744090621145
:1079D000F0EE600474038001E4C0E074F62AF582DE
:1079E000E4340FF583D0E0F0EE600479088031795B
:1079F00007802DEE6004742080027480906214F081
:107A0000EE600474038001E4C0E074FB2AF582E4B4
:107A1000340FF583D0E0F0EE6004790A8002790932
:107A200012476F90620EE48005900FF67404F079AF
:107A300001027FBBC082C08379001247C9E970038D
:107A40001247638056C082C08379011247C9E9702A
:107A5000031247698045C082C08390100C127EDFFC
:107A60007014A3127EDF700E90100AE05480F8A309
:107A7000E0F9E8496007900FF67404801D90100A41
:107A8000E0906200F0900FEF6009E06402700C7407
:107A9000038007E0640370037402F0D083D0820295
:107AA0002B3274F412258090100BE01460081460DF
:107AB0001014603E805F124781127C5AA37B808045
:107AC0004990100AE0FA7900124787127C5A7B80AD
:107AD000E92402F9E43AFA122B9BFC1919E0FAA303
:107AE000E92403F9E43AFA122B9BF9ECA3F0A3E999
:107AF000801F90100AE0F9124793901003EAF0A358
:107B0000EBF0A3E4127C69A37B00122B9BA3F0A3F0
:107B1000E4F0027C11901003E4F0A3F0A3F0FA0269
:107B20007BE575090074037808122D2C127C73E430
:107B300093C0E090100BE0F8D0E0686003027BE4B3
:107B40008A0875090074037808122D2C127C73A31F
:107B5000E493C0E090100AE0F8D0E0686003027B94
:107B6000E48A0875090074037808122D2C127C8BA6
:107B7000E493C0E090100DE0F8D0E06870668A08E9
:107B800075090074037808122D2C127C8BA3E493E2
:107B9000C0E090100CE0F8D0E06870488A087509E1
:107BA0000074037808122D2C127C7FF98882898357
:107BB000A3A3A3A3E493F508740193F5099010031C
:107BC000E508F0A3E509F0A37480F088828983A317
:107BD000A3A3A3A3A3E493F8740193F9901006E878
:107BE000F0A3E9F00A8A089010E2127DE67583108E
:107BF0007582E4E0C398F50AA3E099F50B74037865
:107C00000A122DA0C3E508950AE4950B5003027BE8
:107C100022901003E0FCA3E0FDA3E0FEEC4D4E90AB
:107C20000FF670047404802CE06404602890100641
:107C3000127DE675831075820EC3E098A3E099501B
:107C40000E90100E127DE6901006E8F0A3E9F09079
:107C50000FF67401F07F04022805901003EAF0A3E8
:107C6000EBF0A37480127C6922F0901003E0F9A37A
:107C7000E0FA22127C7722127C7F8882F5832290A0
:107C800010E2E02508F8A3E0350922127C77A3A3CF
:107C90002274EE122580EAFEEBFF8E828F83A3A36F
:107CA000A3A3E493602B9010E6127DE6880889096F
:107CB000800AE5082404F508500205098508828534
:107CC0000983E493F8740193F9EE687002EF697028
:107CD000E1750C00804B9062147490F07410127D6A
:107CE000D670027940750A01750B00E50E780A120C
:107CF0002D2C850882850983A3A3A393550A6004CC
:107D0000E9D2E0F9E9906215F0EA906213F074FBB1
:107D1000250EF582E4340FF583E4F090620EF00551
:107D20000C8E828F83A3A3A3A3E493F8E50CC398DE
:107D30004003027DD17A00790512477B8A0A8B0BBA
:107D4000EA450B60DAEA2402F8E4350BF9E8FCE9CD
:107D5000FD8C828D83E493540FF50E90620EF079C2
:107D6000008A828B83A3A3A3A3E4932407F510A323
:107D7000E4933400F51174037810122DA0AA108C2E
:107D8000828D8393A2E74003027CD69062117448EF
:107D9000F07408127DD670027940750A01750B00E7
:107DA000E50E780A122D2C850882850983A3A393FA
:107DB000550A6004E9D2E0F9E9906212F0EA9062B3
:107DC00010F0850E0A74F6250AF582E4340F027D60
:107DD000177F0A022805F0850A828B83A3A3A3E4F8
:107DE000935403640122E0F8A3E0F922C082C08327
:107DF000127EDC7010A3127EDF700AA3E0640170B3
:107E000002A3E06007900FF67404800C90100374D6
:107E1000F0F0A3740F127F31F0027A9B74F51225F3
:107E200080900FEFE06402601490100C127EDF70FF
:107E30000CA3127EDF700690100BE06009900FF625
:107E40007404F0027ECB7A00790112476F90100A19
:107E5000E060637A00F91247878A088B09AE08AFA1
:107E600009EE4F6049900FEF7404F090100AE09013
:107E70000FF0F0750A008E828F83A3A3A3A3E4936F
:107E8000F8E50AC398503D850A08127ED0E4F07ADE
:107E900000790412477B8A828B83A3A3A3E493F81F
:107EA000127ED0E06870E81247E7050A80C8900F9C
:107EB000F67404F0800E900FF0F0900FEF7403F062
:107EC000F91247AB7A00790212476F7F0302280547
:107ED00074F12508F582E4340FF5832290100AE04E
:107EE000F8A3E0F9E8492274F5122580900FEFE03D
:107EF00064047019901008E064817011127EDC70C7
:107F00000C90100EE064017002A3E06007900FF681
:107F10007404801A90100CE024F1F508A3E0340FEB
:107F2000F509901003E508F0A3E509127F31F08010
:107F30009AF0A3E4F0A304127F3B22F0A3E4F090B4
:107F40000FF6042274F6122580900FEFE06404709F
:107F500064901008E06401705C90100E127EDF7077
:107F60005490100AE0FB90100CE0FA900FF0E0F94A
:107F700012478D8A088B09AE08AF09EE4F60369024
:107F8000100CE0FA790312476F90100AE0C0E090FD
:107F9000100CE024F1F8A3E0340FF988828983D033
:107FA000E0F0EEFAEFFB1247E790100CE0FA7904EC
:107FB00012476F8006900FF67404F07F02022805C6
:107FC000C082C083851882851983E0F8A3E0F9E8B0
:107FD0004960128A828B83ECF0A3E824FF18E9340D
:107FE000FFF94870F2D083D082022B32C2AF75C93C
:107FF000AB75C95B80FEFFFF851A87C2AF022B32CB
:10800000240354004900200043004300320035009F
:10801000330031002000550053004200200043008F
:10802000440043002403540065007800610073009D
:10803000200049006E0073007400720075006D002E
:1080400065006E007400730095482537BB313F4AC8
:108050007F497B3EE93FF746D946D1420000000008
:108060000000000000000000000000000000000010
:108070000000000000000000000000000000000000
:108080000030313233343536373839414243444594
:10809000460000000000000000000000000000009A
:1080A00000000008000400020001FFFFFFFFFFFFC7
:1080B000FFFFFFFFFFFFFFFFFFFF020502000801B8
:1080C0007400000000000082003A003B0000000045
:1080D0000000000200020602F8FF0000E71F030094
:1080E000805101003C000000100E00000400000060
:1080F000E8030000300000000943388664000000F7
:10810000BC02000019E0FCFF00F8FF0760EA000075
:10811000000000000100000002000000975118005C
:10812000FEFFFFFF1F000000080000006AAEE7FF2F
:10813000965118009F020000E9FFFFFF0000FF00BA
:1081400032000000000000FFFA00000004030904F0
:1081500000000000000000000A74F7122580E9907A
:10816000059EF0900553E4F01246619005B2E4F0EC
:10817000A3F090059FF0A3F0123473900902E06021
:108180000464017006122EDF12309B1246679005C0
:1081900014E4F0A3F012485302B19374F012258056
:1081A000EAFEEBFF5480606890059EE0F9123CD730
:1081B0008A088B09EA4509604F7C0080010CEC7548
:1081C000F003A4F8A9F074FE28F582744E39F58303
:1081D000E493F4602CE493F88508828B83E0687064
:1081E000DCAA08EC75F003A4F874FF28F582744E3D
:1081F00039F583E493C0E0740193F583D0821227AC
:1082000066AA08AB09123CC5EEFAEF648002848CC2
:10821000EF5420601E1232D58A088B09EA450960A6
:108220000A1231F1AA08AB09123CC5EEFAEF64203C
:1082300002848C900902E064027024EEA2E0501FD8
:10824000900558E0640F701179001231C1E960099E
:1082500090107C12D3771231D9EE6401028392EE32
:1082600054207003028363750C007A207B00900514
:108270009EE0F9123E33EA4B4C4D70179081181274
:1082800029897A207B0090059EE0F9123E2774042C
:10829000122B807C0079047A007B0012329F8A08BE
:1082A0008B098018850882850983A3A3A3A3A3A3B0
:1082B000A3A3A37401F0850A08850B09E508450905
:1082C00060777C007904AA08AB0912329F8A0A8B76
:1082D0000B750C01E5082404F8E43509F988828956
:1082E0008312EF2512EABD70CD850882850983A32C
:1082F000A3A3A3A3A3A3A3A3A3E0640170A68508DB
:1083000082850983A3A3A3A3A3A3E0540470958546
:108310000882850983A3A3A3A3A3A3A3A3A374068D
:10832000128B8E700374B7F0E0FA8508828509839A
:1083300012866A1231D30282B612326F7C00790142
:108340007A007B0012329F8B09EA45097010E50C18
:10835000700C7A207B0090059EE0F9123E2DEE64B1
:1083600020802FE0600764016003028462EE5410F5
:1083700060081230D7EE64108018EE544060081286
:10838000314FEE6440800BEE5480600B122FABEE49
:108390006480FAEF02848CEF540160169005D112CC
:1083A000CBBD600612C627122766EEFAEF64010203
:1083B000848CEF540860471230A79008F2E0640103
:1083C00070349008F3E0602EF508E4F509F50AF53D
:1083D0000B9080F0780C122DBE7808790C12241BBB
:1083E0007808122B4A7A007B0890059EE0F9123E2D
:1083F000277404122B80EEFAEF640802848CEF5489
:108400001060129005B0E06005E4F01230A7EEFABB
:10841000EF64108077EF544060489005DB12CBBDCD
:1084200060399005E112CBBD60319008F6E064013F
:1084300070299005DB12C6241227669005E112C64A
:108440002412276690810C1229897A007B409005BE
:108450009EE0F9123E277404122B80EEFAEF64407E
:10846000802AEF5402600A12343DEEFAEF64028073
:108470001BEF5404601912CAC712C8D979019005BC
:108480005112D377123023EEFAEF6404FB80047AA2
:10849000007B0002C164C082C08374EA122C2A7C73
:1084A000167D007900AA18AB19123CA77408122E89
:1084B000157402F09005471297B41284D57409120E
:1084C0002E1512C8D97413122E15E412CA2312489D
:1084D000417416800EE8F0A3E9F090055112D138EE
:1084E000227408122B8002C19C74F712258074DF5D
:1084F000122C2AEAFEEBFFEE4F602DAC18AD1912DC
:1085000032F97406122E15E0601E7417122E15E053
:10851000FD7401122E15E0FCEEFAEFFB7900122E2D
:108520005BE9600479A480027900742102B190743F
:10853000F4122580EAFEEBFF8E828F83A3A3A3A310
:10854000A3A3E054406016128B821233B3E9600794
:108550007AFF7BFF02863112C62002862490090230
:10856000E060076401600302860A90053EE0A2E134
:10857000400302860A8E828F8312866412C9E9A3A1
:10858000A3A3A3E0FA88828983A3A312D54A8E828B
:108590008F83A3A3A3A3A3A3A3E0541060047940F3
:1085A00080027900750AFE750BFF780A122B5212B1
:1085B000B658122991AC08AD09128B821230AD74F5
:1085C00004122B80E5086A7003E5096B600B12B694
:1085D0005D6A7003A3E06B704E750A00780A122B77
:1085E0005679028E828F8312B248AA08AB091233E1
:1085F000F57401122B807508CDAA088E828F831224
:10860000866A1231D3E9604C8057900902E0640217
:10861000600FE06004640170DD90053EE0A2E1407F
:10862000D590054712D37774FE6A700374FF6B60B0
:10863000C512C62012DA6B1233B3E98E828F8360C3
:108640000512AA7E800312AA9312AA9C124847E937
:10865000F50870A5EE4F60097901EEFAEFFB1232D2
:108660007B02BF31E0F812B28A2212EDF0E0F9226B
:1086700074F6122580E9FEEAFF7A0F7B00123CBFF8
:10868000EA4B601F8A828B83740CF0EEA3A3F0EF99
:108690008A828B8312AED190059EE0F9123CCB7991
:1086A00000802FEEF91232A58A088B09A808A909C3
:1086B000E849601C88828983A3A3A3A3A3A3A3A3DF
:1086C000A3740612E6ADE0F9123161EEF9123281BF
:1086D000791002C51074F4122580900558E0640FDB
:1086E0007030EA4B602C900553E064086005E0644C
:1086F00004701F8A088B09E4F50AF50B7808122B21
:108700004A7A017B0090059EE0F9123E2174041222
:108710002B8002989F74F2122580EAFEEBFF8C08F2
:108720008D09890A740E122E151297CE850C82F5CA
:1087300083E4F0A312C8DFE0F912338FE960261258
:10874000D36A1233B3E96402701B8E828F83A3A3B2
:10875000A3A3A3A3A3A3A312B8F0850C82850D83C2
:1087600012C8D98003750A0012B082146025146003
:108770003A14605B14606314603F14607D24FE70E3
:108780000302881414700302882814700302883BC3
:10879000028849780C122B52AC08AD09EEFAEFFBB7
:1087A0001230BF7402122B80028844AC08AD09EE6F
:1087B000FAEFFB1230C502885312D36A1233B3E9C1
:1087C0006003028849EEFAEFFB123113028853A9C5
:1087D0000AEEFAEFFB1233FB806A12BB9864027058
:1087E00068E50A700A12DB247003A3E0697064EE86
:1087F000FAEFFBA90A123383804A12DB247003A329
:10880000E069704512BB986402703EEEFAEFFB120D
:10881000336B803F9005D312CBBD6037EEFAEFFB90
:1088200012C627122766802B12DB247003A3E0698F
:108830007017EEFAEFFB1234078018EEFAEFFBA97F
:108840000A123413E9F50A800A750A007AD37B000C
:1088500012426BA90A02D14974F412258074DB120A
:108860002C2A8A088B098A828B83A3A3E0F912320F
:10887000A58A0A8B0BAE0AAF0BEE4F7003028989F3
:10888000850882850983A3A882A983E0C0E012C875
:10889000A7D0E012E6C464F16033850882850983BD
:1088A000A3E064CD6027850882850983A3E0641A6C
:1088B000601B850882850983A3E064E9600F850851
:1088C00082850983A3E064E16003028A7390090250
:1088D000E06007640160030289A28E828F83A3A3F4
:1088E000A3A3A3A3A3E0540870030289A28E828FDE
:1088F00083A3A3A3A3A3A3A3A3A37405F090090236
:10890000E0600464017053850882850983A3E064F4
:10891000E960479005D712CBBD600612C627122723
:10892000669005D912CBBD603190053EE0A2E150C2
:108930002912CD95A3A3A312B0988882898312D35C
:10894000771234A3EA4B6012850882850983A3E07D
:10895000F99005D912C6241227668E828F83A3A3AD
:10896000A3A3A3A3A3A3A3E0640270108E828F83AA
:10897000A3A3A3A3A3A3A3A3A37406F0850882853E
:108980000983A3A3E0F912328112326F900902E049
:108990006402700990108012D3771231D9742502C5
:1089A000989C790012327BE97003028A7390090265
:1089B000E0600764016003028A4890053EE0A2E19E
:1089C0004003028A4812CBB8607E8E828F8312D316
:1089D000777404122BF612CDB21232F98508828513
:1089E0000983A3E064E97020128B71122B5685086D
:1089F00082850983A3E0F50A780A122B5612D55B0B
:108A000012332F7402122B80740D122E1512CBAE5E
:108A100012E9E912C8D97409122E15E060047940F0
:108A200080027900740F122E1512B098740D122E58
:108A30001512D3771230B9E9600E8E828F83A3A30B
:108A4000A3A3A3A3E04420F0EE2404F50AE43FF539
:108A50000B8E828F8312AD2AE0F9850A82850B8303
:108A600012D377124673850A82850B83EAF0A3EB53
:108A70000288FC850882850983A3E0C0E0740212A5
:108A80002E15D0E012A510EEF0A3EF128B8EC0E0F1
:108A90007403122E15D0E012E2BEE0AA18AB1970D2
:108AA0002E122FFF900902E060046401702474020A
:108AB000122E15E0701C128B821233B3E9703690BF
:108AC00005D712CBBD602E12C6271227668003126F
:108AD00033897402122E15E064E97019128B711239
:108AE0002B56750AE9780A122B5612D55B12332FD2
:108AF0007402122B80900902E06007640160030297
:108B0000895A90053EE0A2E1400302895A8E828F85
:108B100083A3A3A3A3A3A3A3A3A3E0640270398E9A
:108B2000828F83A3A3A3A3A3A3E05404602A128B80
:108B3000821233B3E98E828F83700F12C62474FFC2
:108B4000F0A312AD45740502897BA3A3A3A3A3A33D
:108B5000A3A3A3740302897B850882850983A3E00C
:108B600064E9600302895AEEFAEFFB1234190289B4
:108B70005A8E828F8312D138E8FAE9FB750A0178A0
:108B80000A228E828F8312B263FAA3E0FB22F0E501
:108B90000812EDE63509F583E02274F4122580EA27
:108BA000FEEBFF7508007509008E828F83A3A3A3D7
:108BB000A3A3E0603B75080812D36A79FF124973DA
:108BC0008B0BEA450B601075082C8E828F83A3A354
:108BD000A3A3A3E0D2E0F08E828F83A3A3A3A3A3D9
:108BE000E0540364016003028CA4430811028CA4C6
:108BF000EE241812BB9B6049EE241A12BB9B600343
:108C0000F4701D12DB247003A3E06970067508225E
:108C1000028CA4900553E064046003028CA4801CC1
:108C2000EE241BF582E43F12B680241A12BB9BFA95
:108C3000EE2419129874123125E9706875090180C3
:108C40006312D36A1233B3E9640270037508011228
:108C5000DB247003A3E0697006E508D2E1F508E5BE
:108C60000860158E828F83A3A3E07006E508D2E525
:108C70008004E508D2E6F50812D36A1233B3E9643A
:108C8000017006E508D2E0F5088E828F83A3A3E089
:108C9000601212B082F912338FE964016006E508B0
:108CA000C2E0F508900902E0600464017012E50872
:108CB000A2E1400CE509A2E04006E508D2E7F5088C
:108CC00002BF3174EC12258074CD122C2AEAFEEB1F
:108CD000FF851882851983129B907510007511000D
:108CE000750900900902E06402701C8E828F83A3D4
:108CF000A3A3A3E0601190107E12CBBD6009901079
:108D00007E12D3771231D97405122BF68E828F839F
:108D1000A3A3A312CBB012D3751232F9E9700302E8
:108D20008E4679017407122E15E0C3940240011992
:108D30007409122E15E0C3940240027900740E12D9
:108D40002E15E064F87003A3E0F47003028E4674FD
:108D50000E122E15E064F97003A3E0F47003028E86
:108D600046740E122E15E064FA7003A3E0F470034B
:108D7000028E46740E122E15E064FB7003A3E0F41D
:108D80007003028E467408122E15E0F8900541E03B
:108D9000686003028E46E9A2E04003028E4612B8E4
:108DA000E77424122E1512CA12241C12B8EA741287
:108DB000122E1512C8D9740B122E15E0601D741CEA
:108DC000122E15E0FD7406122E15E0FC8E828F83A4
:108DD00012D3757901122E5BE9703D7405122BEEEA
:108DE0001231EBE9F508740B122E15E0702E900588
:108DF0003BE06028742255086422602074425508C4
:108E0000644270147422122E1512978B600E742215
:108E1000122E1512979160047ACF802CE9A2E650A9
:108E20006E900902E060046401702590053EE0A2A6
:108E3000E1501D7422122E1512B08B122A16010158
:108E40000A678E00468E7AD37B0012426B02976FC0
:108E50007422122E1512B08B24FD600B14600824AE
:108E6000FD600424FD70DF7422122E151297D67057
:108E70000E7422122E1512C626A3E0640D60107423
:108E800005122BEE1233EFE96401700302976FEEC7
:108E9000242DF582E43FF583129E687003A3E069F8
:108EA000701E750A00780A122B56780A122B56EE9D
:108EB000242F1298741297A212332F7402122B804F
:108EC000740B122E15E07003028F6D1297A21234EC
:108ED000A38A0A8B0BEA450B7003029016740612E4
:108EE0002E15E0F88E828F83A3A3E028F8A3E03448
:108EF00000F9E8240D129779F88A828B83A3A3A343
:108F0000E068600FE88A828B83A3A3A312DC0812B7
:108F100097DCF079047406122E1512A2FFE02AF8ED
:108F2000A3E034008882F583A3AA82AB83123CB30A
:108F30008A0C8B0D8C0E8D0F850A82850B83A3A363
:108F4000A3A3780C122B0D400302976F9081147825
:108F50000C122D06850A82850B83A3A3A3A3E50C1F
:108F6000F0A3E50DF0A3E50EF0A3E50FF0900902E4
:108F7000E064026015E06007640160030290B09055
:108F8000053EE0A2E150030290AA900553E064047C
:108F90006008E06409600302976FE508A2E54003FA
:108FA000029051EE242F12BB9BC0E07402122E15CA
:108FB000D0E01297FCC0E07403122E15D0E0129797
:108FC000F4C0E07404122E15D0E0F07416122E15C1
:108FD000E0640170267410122E151297977003A387
:108FE000E0697017740E122E1512D3771233B3E99D
:108FF000640270077416122E15E4F01297EA122913
:10900000897406122BF67409122BEE1230057404C3
:10901000122B8002976F900598E064016003028F25
:109020006D7422122E1512978B7009E508A2E65076
:1090300003028F6D7412122E15E0F47003A3E0F496
:10904000600CEEFCEFFD7405122BEE1231F7029767
:109050006FA2E650527422122E1512CDAC70167407
:109060001C122E15E06402703E7405122BEE79007E
:1090700012338380327422122E1512979170147459
:109080001C122E15E06404701E7405122BEE1233B0
:109090007780147422122E151297D6700A790074F4
:1090A00005122BEE1233FB02976F900902E060135A
:1090B000E06401600302976F90053EE0A2E1400387
:1090C00002976F7416122E15E0601CEE240212B681
:1090D00047129D311412AEC7129D31C0E0741612B2
:1090E0002E15D0E0F07006E508C2E7F508E508A205
:1090F000E35061751110A2E25018740A122E15E0A7
:1091000054E3F0740A122E15E0131313541FF8E001
:10911000802CA2E4502A740A122E15E01313543F37
:109120005407F86009740768600B18E87007C3E516
:1091300008C2E7F508E8333354FCF8E054E348F09C
:10914000740A122E15E0C0E08E828F83A3A312AEA4
:1091500017D0E0F0900553E064046008E064096013
:1091600003029230740E122E1512DB317003A3E04D
:1091700069601F740E122E1512D3771233B3E9648F
:1091800002600F740A122E15E0540364016003029A
:10919000976F7407122E15E07041EE242F12BB9BBF
:1091A000C0E07402122E15D0E01297FCC0E07403E8
:1091B000122E15D0E01297F4C0E07404122E15D0D0
:1091C000E01297E51229897406122BF67409122B06
:1091D000EE1230057404122B8080527422122E1568
:1091E00012CDAC7016741C122E15E06402703E7421
:1091F00005122BEE790012338380327422122E1561
:109200001297917014741C122E15E06404701E7471
:1092100005122BEE12337780147422122E1512973A
:10922000D6700A79007405122BEE1233FB02976F89
:10923000746155087003029337E508A2E0506D127F
:10924000B08F7405122BEE123155E9705C12332980
:10925000E9F5097416122E15E0700F7410122E1510
:109260001297977003A3E0696042A90912B08F7446
:1092700005122BEE12315BE96024E508A2E3500CE5
:1092800085188285198374FFF0A3800C740E122E4A
:10929000151297B4E8F0A3E9F0751004800EE50804
:1092A000C2E5F508750900800353089FE508A2E5AB
:1092B000503FEE242F12BB9BC0E07402122E15D03B
:1092C000E01297FCC0E07403122E15D0E01297F460
:1092D000C0E07404122E15D0E01297E512298974AB
:1092E00006122BF67409122BEE1230057404122BA1
:1092F00080E508A2E6400302960AA818A919880A80
:10930000890B780A122B52A909129782122BEE129E
:1093100031DF7402122B80E9F509700302960A749A
:1093200022122E1512B08B6401600302960A74108B
:109330004510F51002960A7407122E15E0640170AC
:109340005D7422122E1512B08B6405701EA818A928
:1093500019880889097808122B52129780122BEE6F
:109360001231DF7402122B8002976F7422122E15B5
:109370001297D67029740E122E1512D377122EFD65
:10938000E9601BA818A919880A890B780A122B52C0
:10939000129780122BEE1231DF7402122B8074169A
:1093A000122E15E070257407122E15E06401700C62
:1093B0007422122E15E0F81297D6600CEEFCEFFD29
:1093C0007405122BEE1231F702976F123275E960B5
:1093D0000302976F741D122E15E0700302948574BA
:1093E00020122E1512B098741F122E15E0FA741E5A
:1093F000122E15E0F9123125E9607D741F122E1529
:10940000E0701E740E122E151297B412BC7EFAA3D1
:10941000E0FB122F098B0BEA450B600302960480D8
:10942000517420122E1512D377741F122E15E0F9E5
:1094300012311F85188285198312DA6B7808740D32
:10944000122E15E060027810740C122E15E06004E4
:10945000740828F8740A122E15E0600108088E823C
:109460008F83A3A3E028FAA3E034008A82F583E087
:1094700014F07510400296047508007808122B56F7
:10948000790B0295BD740E122E1512C8D5740912EF
:109490002E15E060030295D8E508A2E3500302957B
:1094A000D87407122E15E06401607A79008518825D
:1094B00085198312D3771231798A0A8B0BA80AA9EE
:1094C0000BE849601C88828983A3A3A3A3A3E0645B
:1094D00001605288828983A3A3A3A3A3E0640260EE
:1094E00044EE242D12B09285188285198312D37709
:1094F0001234A38A828B83E5824583600FA3A3E0A5
:10950000F91234C1E96005C3940840197410122E91
:109510001512D377122EFDE970030295B374091268
:109520002E157404F0E4F5097809122B56741E12F6
:109530002E15AC82AD83740F122E1512D377740AD8
:10954000122E15E0F912318B7401122B80E9600F95
:109550007510208E828F83A3A312B08B543FF074BA
:109560001D122E15E06023740E122E1512B0987481
:109570001E122E15AA82AB831232F385188285192A
:109580008312DA6B74404510F5107407122E15E043
:109590006401601579007410122E1512B098740EC3
:1095A000122E1512D37712312BE508A2E35037792A
:1095B0004080357508007808122B567902740F1216
:1095C0002E1512B0987411122E1512D3771233F58E
:1095D0007401122B8002976FE508A2E34003029505
:1095E00025744002952679007410122E1512B09839
:1095F000740E122E1512D3771230B9E9600674205A
:109600004510F510123329E9F5098518828519836B
:10961000E064FE7003A3E0F470037509009008F5A0
:10962000E0640160030296BDEE241312BB9BF4704C
:1096300003A3E0F470030296BD740E122E15C3E06E
:1096400094F9A3E094FF507512B8E77410122E1528
:10965000E0687003A3E06960647410122E1512D3E1
:1096600077122F098A0A8B0BA80AA90BE849604DCB
:1096700088828983A3A3A3A3E06401600D88828903
:1096800083A3A3A3A3E0640270337426122E15747F
:109690000112DFE1F8A3E0F97431122E1512C8D9D6
:1096A0007426122BEE122ECDE960127429122E159B
:1096B000AA82AB83122F1BE96003123F8FE508A239
:1096C000E7400302976FE509700302976F8E828F60
:1096D00083A3A3A3A3E0FA7B00123D5B8A0A8B0B52
:1096E000EA450B700302976FEE2404F512E43FF590
:1096F000138E828F83A31297C4122B4E85128285FC
:109700001383E0FC7D00123C9B7403122B807407D2
:10971000122E15E0C0E07402122E15D0E0F0740392
:10972000122E15E4F0A3F07402122BE6880C890DBA
:10973000780C122B527810122B52E509F508780894
:10974000122B5612CAB9122991851282851383E011
:10975000F97407122E1512B098AA0AAB0B1232E751
:109760007407122B80E96007AA0AAB0B123D6174E3
:1097700033122B807F0C022805F582E412E80E22BA
:10978000790012CABD12B09C74072212B26364063B
:109790002212B26964072212D138EE241312B66481
:1097A0006822EE242BF582E43FF58312B68624135B
:1097B00012988F22E01297B922F8A3E0F985188257
:1097C00085198322A31297CE750E00780C22E0F53E
:1097D0000CA3E0F50D2212B269640322A3E4F0A306
:1097E000F0A3F0A322F01297EA22EE2425F582E4FA
:1097F0003FF58322F0EE243112B66422F0EE2430DD
:1098000012B6642274F4122580EAFEEBFF8C088DF8
:10981000099008F2E0600F12DB247003A3E0697086
:10982000051230A7804C790012D36A1231798A82EE
:109830008B83E58245836032A3A3A3A3A3A3E05453
:10984000186027E508241C12C8BC122991E50824D9
:109850001312C8BC122991EE241812987412987928
:109860001231917404122B808008790012987912B9
:1098700030D1802B12B664F9228E828F83A3A3A3EA
:10988000A3A3A3A3A3A312B686240B12988F22F539
:1098900082E43FF58312E9E4FB227418122B807FE7
:1098A0000402280574F012258074EA122C2A8A0A10
:1098B0008B0BEA2402F50EE4350BF50F0A0AFB12B6
:1098C0002F0F8A088B09AE08AF09750801850A8237
:1098D000850B83A3E0F509750C01AC0EAD0F740B7D
:1098E000122E15AA82AB8312468B7413122E1512F8
:1098F0009B907415122E157402F07408122E15E444
:10990000F0901027E0700EEE4F700AE509700675B2
:1099100008C3029AE4900553E0640860067508C223
:10992000029AE0850A82850B83A3A3A3A3A3A3A322
:10993000A3A3A3E0A2E1500EA2E35005750C04809E
:109940000C750C038007A2E35003750C02EE4F70F8
:10995000030299F08E828F83A3A3A3A3E064046023
:109960000D8E828F83A3A3A3A3E06403700C740401
:10997000650C602C7403650C60268E828F83A3A314
:10998000A3A3E06402600D8E828F83A3A3A3A3E050
:10999000640170357402650C60067401650C701CFE
:1099A0008E828F8312D3771233D1E970438E828FE8
:1099B0008312A67B122E1512C8D980348E828F8313
:1099C000A3A3A3A3E06402600D8E828F83A3A3A34D
:1099D000A3E06401700A8E828F8312A7E2122766C9
:1099E000E50A2402FAE4350BFB122F1B7E007F00F0
:1099F0007413122E15E064FE7003A3E0F4704E128F
:109A00002ED9E97048E5096023900590E064027062
:109A10001B90102E12D3771233D1E9700F90102EB5
:109A200012A67B122E15E8F0A3E98020850A828514
:109A30000B83A3A3A3A3A3A3A3A3A3A3E05402F90B
:109A40001230E37413122E15EAF0A3EBF074131224
:109A50002E15E064FE7003A3E0F470057508C7805E
:109A60007FE509F50D780D122B56850A82850B834B
:109A7000A3A3A3A3A3A3A3A3A3A3E0F9E50A24029A
:109A8000FCE4350BFD7414122E1512D37712302915
:109A90007401122B80E97048A90CE50A2402FCE449
:109AA000350BFD7413122E1512D377122EEB8A0E7E
:109AB0008B0FAE0EAF0FEE4F601E74026509700D76
:109AC0008E828F83A3A3A3A3A3E0D2E3F074151225
:109AD0002E15E4F0F50880087413122E15129B90D1
:109AE000E5097009AA18AB19124823800AFCA90CD1
:109AF000AA18AB19123371E9F8EE4F6053E509600B
:109B0000208E828F83A3A3A3A3A3E0D2E6F07402E6
:109B10006509700D8E828F83A3A3A3A3A3E0D2E572
:109B2000F0850A82850B83A3A3A3A3A3A3A3A3A366
:109B3000A3E0A2E6500D8E828F83A3A3A3A3A3E08C
:109B4000D2E7F08E828F83A3A3A3A3A3A3E004F0A4
:109B5000E5087003E86034FC7D007A017B10124652
:109B60006DEE4F600CE50A2402FAE4350BFB122F70
:109B70001B7413122E15E064FE7003A3E0F4600B57
:109B80007413122E1512A7E2122766741602C16111
:109B900074FEF0A304F02274F712258074F7122CDF
:109BA0002AEAFEEBFF900553E06403600DE06401D8
:109BB0006008E064096003029CC18E828F83A3E089
:109BC0006003029C977C007D007A027B0012466D48
:109BD000129CC68A828B8312B8F090054412C8D9B1
:109BE0007953124817790090055112D37712302318
:109BF000900553E06409600990055112D37712343F
:109C00009D851882851983740112CA2379421248EE
:109C1000179005537404F07401122BEE794A124820
:109C2000117401122BF67A497B0512468B900902BA
:109C3000E060046401701F900547E064FE7003A3B8
:109C4000E0F4602A79007401122BF690054712D3D4
:109C500077122EEB8018E06402701390054412B066
:109C6000987A037B0012466D12A5A212466D9005EC
:109C70003EE0A2E35004D2F08002C2F012CA197989
:109C800052124817900902E06402703290107C1260
:109C9000D3771231D980278E828F83A3AE82AF8390
:109CA000FC7D007A037B1012466D8E828F83E0F973
:109CB00090055112D377123023900553E4F01232FD
:109CC00045740902B190EE2402FAE43FFB22C082FF
:109CD000C08390051412CBBD701F900553E0146033
:109CE0000924FC600A14600C800F90051D803490DC
:109CF0000519802F90051B802AE8496008900515FA
:109D000012A308700C8A828B83A3E0F912300B80B7
:109D10001D900514129D3164027005123431800EBD
:109D20009005D512CBBD600612C62712276602C168
:109D30009CE0F8129D3722A3E0C82406F582E4389F
:109D4000F583E02274F412258074FB122C2A8A0811
:109D50008B097A0F7B00123CBF8A0A8B0BAE0AAFCD
:109D60000BEE4F7003029E638E828F83740212CAC1
:109D7000237950124811850882850983A3E0600386
:109D8000029E46900551E0F47003A3E0F460449015
:109D90000551E064FE7003A3E0F460378518828506
:109DA0001983129E687003A3E06960278508828585
:109DB0000983A374EAF07A447B0579531248177A31
:109DC000477B05794B1248177A517B057950124829
:109DD00017807385188285198312DBF512C8D97A2A
:109DE000447B05795312481190054412AD3B12C8CB
:109DF000D97A477B05794B1248117A467B0579E180
:109E0000124811900558E0C3940F501D900546E08C
:109E1000C0E07402122E15D0E0F07404122E1574F6
:109E200001F004122BEE12483B750A00780A122B3F
:109E300056780A122B569010B1E0F912AA2A123362
:109E40002F7402122B8085088285098312D68AA37B
:109E5000F09005537403F0EEFAEFFB90059EE0F9E5
:109E6000123CCB740502989C12DBF9E0682274F472
:109E700012258074E8122C2AEAFCEBFD8C828D837B
:109E8000A3A3A3A37808122DBE7808122D50900525
:109E9000547808122CE07F7F7E7F790090055478FB
:109EA00008122DBEE97808122BB5E508A2E050296A
:109EB000780090059F8014850882850983A3A3E01C
:109EC00069700108E508241412C8BC12A70570E7E0
:109ED000E8C39F5004E8FFE9FE09E9C3941B40BCB6
:109EE0008C828D83A3A3A3A3122DF2E8494A4B6071
:109EF0007DEC2404F508E43DF509850882F583121C
:109F00002DF2900554122DFE7C187D007900AA18C0
:109F1000AB19123CA7850882850983122DF285189A
:109F200082851983122DFE7404122E157401F0908F
:109F3000055AE0C0E07405122E15D0E0F074071247
:109F40002E15E412CA2312482F807090055112D3A7
:109F5000771230598A0A8B0BA80AA90B900551E891
:109F6000F0A3E912CBCA687003A3E069602D9005E5
:109F70009F12A7056025850882850983129E687057
:109F800003A3E069700C850882850983A3A3E06EB2
:109F900060B9E508241412C8BC80D6EE900546F0DE
:109FA000123227E96015900553E4F090051F12CB9B
:109FB000BD600879C412C62712276602989A74F405
:109FC00012258074E8122C2A8A828B83A3A3A3A370
:109FD000A3A3A3A3A312B8F0E8FAE9FB79009005C4
:109FE000547808122DBEE97808122BB5E508A2E0D6
:109FF0005031EA29F582E43BF583E0F890102DE03A
:10A00000C398501F750801750900750A00750B008B
:10A01000E97808122AEE7808122D50900554780835
:10A02000122CE009E9C3941B40B4900554122DF2A0
:10A03000E8494A4B604E7C187D007900AA18AB199C
:10A04000123CA7900554122DF285188285198312AF
:10A050002DFE7404122E157401F07407122E15745F
:10A0600001F090055AE0C0E07405122E15D0E0F022
:10A070007407122E15E412CA2312482F9005537448
:10A0800006F0801E900553E4F0FCFD7A047B10126C
:10A09000466D90051F12CBBD600879C412C6271209
:10A0A000276602989A74F512258074D1122C2A8A98
:10A0B000088B098A828B8312B8F4741C122BF68ADF
:10A0C000828B83A3A3A3A3A3A3A312B23F12D37231
:10A0D000123257741C122E15E0702C8508828509E7
:10A0E00083A3A3A3A3A3A3A3A3E0C3940B40188EAD
:10A0F000828F83A3A3A3A3A3A3A3A3E064027007F7
:10A1000012C8A7E0F4600302A2FA900553E06402CB
:10A11000700302A1DCE06406700302A1DC90051468
:10A1200012CBBD600812A308700302A21190055360
:10A13000E064086008E06404600302A2FA741E127E
:10A140002E1512A2FFA3A3A3A312B8F4900514E046
:10A15000F8496007129D3764026077900551E06E00
:10A160007003A3E06F600302A2FA74016A601674C0
:10A1700023122E15AC82AD837A657B05124685E9E4
:10A18000600302A2FA7A007B0290059EE0F9123E7B
:10A1900033EA4B4C4D600302A2FA900554122DF2A3
:10A1A000851882851983122DFE90055AE0C0E0744F
:10A1B00004122E15D0E0F07405122E157401F074FF
:10A1C00006122E15740212CA23122F93E96003029D
:10A1D000A2F7EEFAEFFB12342B02A2FA900514124A
:10A1E000CBBD702D7508007808122B567808122BFD
:10A1F00056EE2410F582E43FF58312CBB1A3A3A35E
:10A20000A3A3A3A3A3A312AE0C12332F7402122B89
:10A21000808E828F8312B8F07407122E15E8F0A397
:10A22000E912AD4512B8F07409122E1512CA1224A3
:10A230000D12BB9BC0E0740B122E15D0E0F012C8BB
:10A24000A712AD1E740F7808122DA0740C122E15D3
:10A25000E508F07420122E15E0C0E0740D122E15E2
:10A26000D0E0F07422122E15E0C0E0740E122E150C
:10A27000D0E0F0741D122E15E0C0E07410122E15FF
:10A28000D0E0F0741E122E15E0C0E0740F122E15EF
:10A29000D0E0F0EE241012BB9BC0E07411122E151A
:10A2A000D0E0F07421122E15E0C0E07412122E15C9
:10A2B000D0E0F0742E122E15E0C0E07413122E15AB
:10A2C000D0E0F07423122E15A982AA8389088A0986
:10A2D000750A007808122B4E7C087D007417122E28
:10A2E00015AA82AB83123C9B7403122B8074071255
:10A2F0002BEE12301D8003122F99742F02EF34E0E1
:10A30000FA8E828F83A3A322129D3864012274F6F1
:10A3100012258074C9122C2A9005CF12CBBD60067D
:10A3200012C627122766900553E06408700302A343
:10A33000CB900590E064027023904FE5E493900584
:10A3400035F0904FE5E493900533F090055C74018F
:10A35000F01297DC04F0A3E4F0A3806C900564E0B5
:10A36000F8742128F582E4340AF583E0FA90053583
:10A37000F0742228F582E4340AF583E0F99005337D
:10A38000F07508FF7509FFEA7808122D2CE508F42E
:10A39000FCE509F4FD3395E0FE90055CECF0A3EDDF
:10A3A000F0A3EEF0A3F07508FF7509FFE9C39A78F2
:10A3B00008122D2CE508F4FCE509F4FD3395E0FEC8
:10A3C000A3ECF0A3EDF0A3EEF0A3F07C237D0079E5
:10A3D000007414122BEE123CA7900564E07009740F
:10A3E0001E122E1574018006741E122E15E412A57D
:10A3F00010740FF090102C12CA237946124817746B
:10A4000001122E15E4F090108BE0C0E07402122EC1
:10A4100015D0E0F0900541E0C0E07403122E15D095
:10A42000E0F07404122E15E4F07405122E15E4F019
:10A430007407122E15E4F0900564E0C3940F500CDD
:10A44000E0C0E07406122E15D0E080077406122ECC
:10A4500015740FF07C657D057408122E15AA82AB69
:10A460008312468B7C037D0079FF7410122E15AA8F
:10A4700082AB83123CA790059DE0C0E07413122EBE
:10A4800015D0E012C81B7401122BEE1232517AA1C2
:10A490007B05794512481712335F900558E0C0E0FC
:10A4A000741C122E15D0E0F0900559E0C0E0741D28
:10A4B000122E15D0E0F0900546E0C0E0741A122E7E
:10A4C00015D0E01284D97418122E1512C8D9742030
:10A4D000122E15E4F090055BE0C0E0741F122E15FB
:10A4E000D0E0F07434122E15E4F07429122E15E425
:10A4F000F07A447B0579531248177A477B05794BEC
:10A500001248177414122BEE124835743702C50D19
:10A5100012A51422F085188285198322C082C08377
:10A520008A828B83A3E09005536004E4F08070740A
:10A5300008F0900564E0702890051F12CBBD6008FC
:10A54000790012C62712276690055112B0987A0535
:10A550007B0012466D90055112D37712349D8018FE
:10A56000790012301790054412B0987A067B0012D9
:10A57000466D12A5A212466D9005DB12CBBD601F81
:10A580009008F6E06401701790810C1229897A0016
:10A590007B4090059EE0F9123E217404122B80024C
:10A5A000C19C90054712B09C7A047B002274F4127F
:10A5B000258074EA122C2AEAFEEBFF129CC6122FA9
:10A5C0000F8A088B09EA4509700302A6768A828BF6
:10A5D00083A3A3A3A3E0640160278A828B83A3A340
:10A5E000A3A3E06402601A8A828B83A3A3A3A3E0DF
:10A5F0006403600D8A828B83A3A3A3A3E064047029
:10A6000075EE2402FCE43FFD740B122E15AA82ABFA
:10A610008312468B85088285098312A67B122E152C
:10A6200012C8D97415122E157401F07408122E1563
:10A63000E412CA23124829890AAC0A7D007A077BF2
:10A640000012466D850882850983A3A3A3A3A3E016
:10A65000C2E012C108A3A3740112E2CD5001097A2D
:10A66000027B00122323E8850882850983A3A3A324
:10A67000A3A3A3A3A3F0741602989C12D138741359
:10A680002274F212258074F8122C2AEAFEEBFF8C59
:10A690000A8D0B890C9080B2AC18AD197408122A7F
:10A6A000AEF50DEEFCEFFDAA18AB19124685E97068
:10A6B00003750D0190059F801AEEFCEFFDE508245F
:10A6C0000BFAE43509FB124685E97023E5082414EA
:10A6D00012C8BC12A7056024E50DA2E040DB850886
:10A6E00082850983E0650A7004A3E0650B70DD854F
:10A6F0000882850983A3A3E0650C70D0AA08AB0982
:10A70000740802D14612AD22E508450922C082C074
:10A710008390059F02C19974F712258090059F12BE
:10A72000E9E4800C12D40312B8F7123D61EEFAEF9F
:10A73000FBEA4B70EF90059FE4F0A3F002B1937435
:10A74000F4122580EAFEEBFFEE241312BB9B640398
:10A75000700CEE240BFAE43FFB122F0F800EE06426
:10A7600002707C12C8A712D377122F098A088B09AE
:10A77000E508450960698E828F83A3E0700F850824
:10A7800082850983A3A3A3A3A3A3E4805164F160FA
:10A790000A8E828F83A3E064E17027850882850991
:10A7A00083A3A3A3A3A3A3E06401701685088285F5
:10A7B000098312A7E2122766EE240BFAE43FFB128C
:10A7C0002F1B850882850983A3A3A3A3A3A3E0600D
:10A7D0000E850882850983A3A3A3A3A3A314F00273
:10A7E000989F12989590052D12C8ED2274F11225AC
:10A7F000808A088B09ECFEEDFF890A12D677EEF805
:10A80000EFF9A30EAF838A828B83A3A3E0C454F035
:10A81000FA88828983E04A12A8CD12D68B12A8C882
:10A82000E0333354FCF88E828F83E04812A8C8A32B
:10A83000E033333354F8F88E828F83E048F0EEF83B
:10A84000EFF9A30EAF838508828B83A3A3A3A3A3F1
:10A85000A3E0A2E0E4331313FA88828983E04AF08C
:10A86000E5082407F50CE43509F50D750E00780CA4
:10A87000122B4E7C087D00EEFAEFFB123C9B74031A
:10A88000122B80EE2408FE50010FE508240FF50C72
:10A89000E43509F50D780C122B4E7C037D00EEFAA1
:10A8A000EFFB123C9B7403122B80E50AC3940F400C
:10A8B00012E5082412F582E412DF018E828F83A351
:10A8C000A3A3F07F0702280512A8CDA322F08508D4
:10A8D000828B83A3A3A32274F1122580EAFEEBFFEF
:10A8E000890A8C088D098E828F83E08C828D831279
:10A8F000B696AE82AF83E012BF3612C124C412BF37
:10A900003612A9A1E054038C828D8312C122A2E2E7
:10A91000E4338C828D8312C121131313541F12BF91
:10A920003612C120A2E7E4338C828D83A3A3A3A3B4
:10A9300012A9A18E0C8F0D750E00780C122B4E7C77
:10A94000087D00E5082407FAE43509FB123C9B74F6
:10A9500003122B80EE2408FE50010F8E0C8F0D7811
:10A960000C122B4E7C037D00E508240FFAE4350918
:10A97000FB123C9B7403122B80E50AC3940F401515
:10A980008E828F83A3A3A3E0C0E0E508241212C83F
:10A99000BCD0E08008E508241212C8BCE4F002A88C
:10A9A000C3A3A312B69A0EAF832274F51225808A30
:10A9B000088B098A828B83A3AE82AF83E0F91230C1
:10A9C000418E828F83E064EB602485088285098351
:10A9D000A3E064E16018850882850983A3E064F13F
:10A9E000600C850882850983A3E0641A70098508D4
:10A9F00082850983A3E4F090107C12D3771231D9B9
:10AA0000750A01780A122B56850882850983A3E00E
:10AA1000F5087808122B56790012AA2A12332F74DF
:10AA200002122B8012326F02EF3790055112B09C48
:10AA300090054712989522C082C083E99005B170B5
:10AA400003E4800274018065E0F902C19C74F7128E
:10AA50002580EAFEEBFF8E828F8312C9EB12DA505B
:10AA600012DA6B1233B3E98E828F83600512AA7EED
:10AA7000800312AA9312AA9C12484702B19312AA09
:10AA800085E4F0A322E0F8A3E0C8240DF582E438C1
:10AA9000F5832212AA857401F0A3E422F07CC77D1D
:10AAA000318E828F8312989522EAF0A3EBF002C1D7
:10AAB0009C74F61225809005B1E0701B7C00790132
:10AAC0007A007B0012329FEA4B600C8A828B8312E1
:10AAD000CBBD60031231CD02C510C082C0837904A2
:10AAE000123299E9F8904FE1E493C398401079FF4E
:10AAF000123299E9F8904FDFE493C398500479013A
:10AB00008002790002C19C74F01225808A088B09AA
:10AB1000890B750C008A828B83A3A3A3A3A3A3A391
:10AB2000A3E0F91232A58A0E8B0FAE0EAF0F750A95
:10AB300001EE4F600302ABD785088285098312AD11
:10AB40002AA3A3A3A3A3A312BC7012D37712328D9E
:10AB50008A0C8B0DAE0CAF0DEE4F700302AD108E54
:10AB6000828F83A3A3A3A3E4F0A3F0E508240CFA47
:10AB7000E43509FB8A828B83E0C0E012E2C3D0E0B7
:10AB8000F01233BFEE240D12DA65E50812DEF3355C
:10AB90000912B8EE12B65812C8D9750C01EE240687
:10ABA00012BB9F547FF0A3E054FC12E6C45404602F
:10ABB0000302AC4E901084E0F50875090074077824
:10ABC00008122D2C8E828F83A3A3A3A3A3A3E045F9
:10ABD00008F0A3E04509F08E828F83A3A3A3A312FC
:10ABE000AD1C74077808122DA0E5085407F508E598
:10ABF0000B606B8E828F83A3A3A3A3A3A3A3A3A3A2
:10AC0000740212C12512B007600B90053F12AD3BD4
:10AC1000A3A312C8D9E508700302ACDCEE24061227
:10AC2000EDB9547FFCA3E054FCFDE50824FFF508D2
:10AC3000E434FFF50974077808122D2CEC4508F868
:10AC4000ED4509F98A828B8312C8D902ACDC8E8269
:10AC50008F83A3A3A3A3A3A3E0448002ABD6E508FC
:10AC60007005750A0080758E828F83A3A3A3A3A3AA
:10AC7000A3E05420600C123CB9EA547F7900245FB1
:10AC800080198E828F83A3A3A3A3A3A3E054106093
:10AC90001A123CB9EA540F7900240A5001098E8235
:10ACA0008F83A3A3A3A3F0A3E9800D8E828F83A338
:10ACB000A3A3A37401F0A3E412AD457404F07A20B9
:10ACC0007B0090059EE0F9123E33EA4B4C4D700C30
:10ACD0007A207B0090059EE0F9123D01E50CA2E090
:10ACE00050318E828F83A3A3A3A312D37BF9EEFAF4
:10ACF000EFFB123293E9601B12B18812CBBB6009E3
:10AD000012B27712D377123D61EEFAEFFB123D617A
:10AD1000750A00A90A02C1648E828F83A3A312ADB3
:10AD20002222E0F508A3E0F50922A3A3A3A3A3A38D
:10AD300012B09C850882850983A32212D1388E82A5
:10AD40008F83A3A32212C8C9A3A3A32274F412253C
:10AD50008074F7122C2A7E001232A5EA4B7003028F
:10AD6000AE058A828B83A3A3A3A3A3A3A3A3A3E07B
:10AD70006406600302AE058A828B83A3A3A3A3A308
:10AD8000A3A3E0FF8A828B8312AE17E0C0E07408B1
:10AD9000122E15D0E012B25C12C8D61232C3EF5494
:10ADA00008606085188285198312B0987A007B004C
:10ADB0001232878B0BEA450B704912EF2E12485F57
:10ADC0007C007D007A007B0080258E828F8312B00C
:10ADD0008BF47003A3E0F4602A90055112AE0C12BC
:10ADE0004859E9641A601C7C007D00EEFAEFFB1202
:10ADF00032878A0A8B0BAE0AAF0BEE4F70CC79000C
:10AE00001248657E01EEF9740902989C12B09C8E7E
:10AE1000828F831298952212B8E212AE1E22240865
:10AE2000F582E438F58322C082C083EA4B70059036
:10AE300005B280068A828B83A3A312B03B60258A69
:10AE4000828B83A3A3A3A3A3A3A3E0540860E5EC90
:10AE50004D60158A828B8312B08B6C7003A3E06DFA
:10AE600070D280047A007B0002C19C74F2122580AB
:10AE7000EAFEEBFF890A8C088D097A117B00123DEE
:10AE80005BEA4B603E8A828B83A3A3A3A3A3A3A305
:10AE9000A3A3E412B250A3E50A12DC08A3A3A312F1
:10AEA000F00F8A828B83A3A3A3A3E4F0A312B27151
:10AEB00012AED112DA5812B766E4F012AEC6A3A3EE
:10AEC000F0A3F002D149A312AECB22F08A828B8389
:10AED00022A3F012EDE53BF583E4F02274F4122591
:10AEE00080EAFEEBFF89088C0A8D0BEE4F7003029F
:10AEF000AF907401650870127901123299E9F890E7
:10AF00004FE2E493C39850228016740465087014CD
:10AF10007904123299E9F8904FE1E493C398500A0A
:10AF20007911806E7402650870668E828F83A3A388
:10AF3000A3A3A3A3A3A3A3E50812BEA112D66F8E59
:10AF4000828F83A3A3E4F0A3F09005B212CBBD607F
:10AF5000178003E0F8A312C9F2A3A312B03B8882C2
:10AF60008983A3A370ED80039005B212DA5C7A2086
:10AF70007B0090059EE0F9123E33EA4B4C4D700C7D
:10AF80007A207B0090059EE0F9123D017900800255
:10AF900079C102989FC082C083E9F879009005B218
:10AFA000801D8A828B83A3A3A3A3A3A3A3A3A3E04F
:10AFB00068600574FF687001098A828B83A3A312FD
:10AFC000B03B70DE02C19C74F7122580EA4B70051D
:10AFD0009005B280068A828B83A3A312B03B6020C7
:10AFE0008A828B83A3A3A3A3A3A3A3A3A3E06970D3
:10AFF000E4EC60108A828B83E012B00770D7800483
:10B000007A007B0002B19312AA86E0540422C08227
:10B01000C0839005B280068A828B83A3A312B03BC3
:10B0200060128A828B83A3A3A3A3A3A3A3A3E06933
:10B0300070E580047A007B0002C19C129895EA4B6F
:10B040002274F7122580EAFCEBFD9005B280068A97
:10B05000828B83A3A312B03B60218A828B8312B0C0
:10B060008B6C7003A3E06D70E68A828B8312866618
:10B0700012CAD8A2E0E43370D680047A007B0002C2
:10B08000B193EE241DF582E43FF58312B26322EE04
:10B090002413F582E43FF58312B09C2212B0A02263
:10B0A000E0FCA3E0FD2274F21225808A0A8B0B8C4F
:10B0B0000C8D0D750800750900EA450B6030900590
:10B0C000B280068E828F83A3A312B8F7EE4F601E64
:10B0D000AC0CAD0DEEFAEFFB850A82850B831227CF
:10B0E00066E9640170DDEEF8EFF988088909AA08BD
:10B0F000AB0902D1497900022B3274F712258090F6
:10B1000005B212B8F07C007D00800DE8FCE9FD88F6
:10B11000828983A3A312B8F0E8496030EA6870021C
:10B12000EB6970E79005B212D377E86A7002E96BB9
:10B1300088828983A3A3700812B8F09005B28009B1
:10B1400012B8F08C828D83A3A312C8D9804574F7FE
:10B15000122580EAFEEBFFEE4F602B1232BD12B2D9
:10B160007D123D618E828F8312D377123D6112B1C1
:10B170008812CBBB600912B27712D377123D61EE11
:10B18000FAEFFB123D61800BEE240DF582E43F22C5
:10B19000122B807F0102280574F71225808A828B8A
:10B1A0008312B2489005B212B8F07508007E008094
:10B1B0003388828983A3A3A3A3A3A3A3A3A3E06447
:10B1C0000570180E88828983E0FFA3E0F5838F82E3
:10B1D000E06C7003A3E06D7002050888828983A388
:10B1E000A312B8F0E84970C9904FD312E418500880
:10B1F000904FCD12D2B8400F8A828B83A3A3A3A312
:10B200007401F0A3E4800C90053FE0F812B23FE82F
:10B21000F0A3E912B271740512B250E0440812B200
:10B220005CF47003A3E0F4600E90055112D5721225
:10B230004859E9641A7005790112486502B193A36F
:10B2400012B640A3A3A3A32212B263FCA3E0FD2283
:10B2500012B2542212DC10A3A3A3A32212AECB126B
:10B26000B26322E0F812B26922A3E0F5838882E09B
:10B270002212B254A3A32212B188F5832212B284FF
:10B28000129893228E828F83E0F8A3E0C8241FF5E2
:10B2900082E43822C082C083EAFCEBFDEC4D6017EB
:10B2A000EC24FBF582ED34FF12CBBB700712B2EE3B
:10B2B000E0F46007123CC57905803090059EE0C03F
:10B2C000E012B2EED0E0F0904FE7E493F97AB47B6D
:10B2D00005123CFBE9640170107A007B2090059E0A
:10B2E000E0F9123D0179008002790402C19CEC244E
:10B2F000FFF582ED34FFF5832274F4122580A2AFAE
:10B30000E433F508C2AF9005B412B8F7EE4F603AD7
:10B31000EE24FBF582EF34FF12CBBB7A007B20904A
:10B32000059E6007E0F9123D018005E0F9123D0736
:10B33000E4F50AF50B780A122B52EEFCEFFD7AB415
:10B340007B05123CF57402122B80E508A2E092AF57
:10B35000EEFAEFFB02989F74F012258074DB122C3A
:10B360002AEAFEEBFF750B00750A007508FE7509E9
:10B37000FF123275E9600302B633EE241512BB9B4F
:10B38000604690109EE0C43354E0F8E0333354FC40
:10B3900048C0E012D35CD0E012B69612D37679FFA3
:10B3A0001249738B0DEA450D6011750B017508FF8D
:10B3B00012B65D440412C8F6D2E0F0900902E060D3
:10B3C0000464017003750A408E828F8312D3751254
:10B3D00033B3E9600312C9C9EE241312BB9B700D8D
:10B3E000904FDEE493C0E012CAB9D0E0F08E828FB5
:10B3F00083E0A2E7500454038019EE241412BB9B8F
:10B400007012900530E0C0E012ED97D0E0F09005AA
:10B4100030E004F012EDB070199008E1E0600D909A
:10B42000053BE0700D8E828F83E07006EE241112D2
:10B43000C9CC900902E060046401704890053EE0C8
:10B44000A2E15040E50BA2E040218E828F8312D30F
:10B45000751233B3E9602D8E828F83E0600DEE2488
:10B460000B12B085F912338FE9601912B66C7003B4
:10B4700002B5E4EE241312EDB3600302B5E412B694
:10B480005D54FBF08E828F83E06401700DEE240B1F
:10B4900012B0856402700312B67912B66C600302B2
:10B4A000B55DE50BA2E0500302B55D900902E060D6
:10B4B000076401600302B55D90053EE0A2E1400330
:10B4C00002B55DE50AF50B780B122B56EE2406FC4F
:10B4D000E43FFD8E828F8312D375EE24121298748E
:10B4E00012318B7401122B80E9600612C9C912B6A1
:10B4F000728E828F83A3A3A3A3A3A3E0603CEE2458
:10B5000002F50CE43FF50D850C8212B6802407FA93
:10B51000E43FFB1232F38A088B09850C82850D8388
:10B52000E065087004A3E06509700C8E828F83A328
:10B53000A3A3A3A3A3E4F012B6798E828F83E06461
:10B54000016008A90A12B68B12312BA90A8E828FCC
:10B550008312B68B1230B9E9600312B672AC18AD23
:10B5600019EEFAEFFB1232ED8A0A8B0B74FE6508B6
:10B57000700474FF6509700312AD18EA450B70037F
:10B5800002B6378E828F83E0C0E07401122E15D090
:10B59000E0F07402122E1512DA5C7401122BE688A8
:10B5A0000C890D780C122B5212B658122991EE24E8
:10B5B0000E12BB9BF50C780C122B569005441229E9
:10B5C000917407122E15E0F9AC08AD091232E77438
:10B5D00007122B80E9FE74106E705EAA0AAB0B1284
:10B5E0003D618055EE241312BB9BC0E07415122EF2
:10B5F00015D0E012EE14740D122E1512CA12240486
:10B6000012B64712B8F0740F122E1512CA12241473
:10B6100012BB9BC0E07416122E15D0E012E2B912D4
:10B62000B64012B0987404122BEE12315BE960033D
:10B6300002B484791180047E10EEF9742502C16190
:10B64000E0F98A828B832212B64B22F8E43FF9E8B4
:10B65000FAE9FB8A828B8322EE12C9DE2212B661DE
:10B6600022EE240FF582E43FF583E02212B6615406
:10B67000402212B6614420F02212B6614440F0220A
:10B68000F58312B6862212B0A0EE22A3A3A3A312C2
:10B69000D3871298952212B69A22F08E828F83A3B6
:10B6A00022C082C08374DC122C2A8A828B83A3A3DB
:10B6B000A3A312B8F0740E122E15E8F0A3E912D16C
:10B6C0002F740C122E1512C8D912B766E0C0E074A0
:10B6D0001A122E15D0E0F012B7703B12B8EE74209B
:10B6E000122E1512C8D9EA12D3643BF583E0C0E0EC
:10B6F0007408122E15D0E0F0EA241CF582E43B1207
:10B70000B8EE7412122E1512C8D9EA2411F582E48B
:10B710003BF583E0C0E07409122E15D0E0F0EA2476
:10B7200012F582E43BF583E0C0E07407122E15D0D9
:10B73000E012A51074FFF07401122E1574FFF0745E
:10B7400002122E1574FFF0908110122989740412D0
:10B750002BF67407122BEE1230057404122B80792D
:10B760000074240284E3EA240DF582E43BF583228D
:10B77000EA12EDE62274EE12258074EF122C2A8A6A
:10B780000E8B0F8C088D09890C750A107A217B00AD
:10B79000123D5B12D18FE849700302B8DB750B00D4
:10B7A0007C217D007900851882851983E0FA123C9E
:10B7B000A77426122E1512B8F7900902E0600464EF
:10B7C00001703EAA08AB09122F098A108B11A8102C
:10B7D000A911E849602388828983A3A3A3A3E06415
:10B7E00001600D88828983A3A3A3A3E06403700989
:10B7F000EE5440700474044FFFEF54046003750B63
:10B800000190055112D37785188285198312B8E209
:10B810002409F582E43812DA697423122E1512B85D
:10B82000F0740F122E15E8F0A3E912B8FD12EDDC4A
:10B8300012B8FD12AE1E740212BC7A12C625E508BB
:10B84000F0A3E50912B8FD12EDA7E50CF07425127E
:10B850002E15E0F50885188285198312EDECE508B0
:10B8600012B8FD241FF582E438F583E50EF0A3E558
:10B870000FF07406122E1512DA5C7408122E15E5FC
:10B8800008F07428122E1512C624C082C083740CCE
:10B89000122E15AC82AD83D083D0827403122AAEEF
:10B8A000A90BAA18AB1912327BE964017021900927
:10B8B00002E0600464017012E50BA2E0500CA908DC
:10B8C0001232A5EA4B60031232C9750A00800C855A
:10B8D000188285198312D377123D61A90A74110267
:10B8E000BEAE12D13DC822EE2413F582E43FF583AB
:10B8F00012D13822A3A3A3E0FEA3E0FF2212D19E1F
:10B90000C82274EE122580EAFEEBFF8C088D098EAA
:10B91000828F83A3740812CA05E060088E828F8329
:10B92000A37410F012BB9860098E828F83A3E02469
:10B9300008F0EE241512BB9B60088E828F83A3E073
:10B9400004F08E828F83A3A3A3A3A3A3E060198E28
:10B95000828F83A3A3A3A3A3A3A3E0C3332402F8EA
:10B960008E828F83A3E028F0EE241112BB9B60052A
:10B97000750B0E8003750B008E828F83A3E0F8EEAB
:10B98000240D12BB9B28250B8C828D83F0EE241195
:10B9900012BB9B601190053CE0F9122E6185088274
:10B9A000850983E029F0850882850983E0C39475C1
:10B9B000400975080075090002BB91E0FA7B00128E
:10B9C0003D5B8A088B09EA4509700302BB918E82B0
:10B9D0008F83E0FA90054112BBA97402780C122DF6
:10B9E0002CEA450CFAAB0DEE241212BB9B5403F566
:10B9F0000C750D007406780C122D2CEA450CFCEB2E
:10BA0000FDEE241512BB9B6004780180027800EEE5
:10BA10002416FAE43FFBE8F9ED49FDEE241112BBD0
:10BA20009BF50C7409780C122D2CED450DFD8A82C6
:10BA30008B8312BBA9740B780C122D2CED450DFDD8
:10BA400012BE7E12BBA9740C780C122D2CED450D84
:10BA5000FD8E828F83A3A3A3A3A3A312BBA9740A01
:10BA6000780C122D2CECF8ED450DF9E8850882854F
:10BA70000983F0E9A3F0EE240212BB9F85088285BA
:10BA8000098312BBCDF0EE2404F8E43FF9888289E3
:10BA90008312C0CFA312BBCDA3A3F0EE241312BB1D
:10BAA000B0F0EE241412BBB0A3F0750A088A828BA2
:10BAB00083E06015EE241812B092E5082408FAE439
:10BAC0003509FB12468B750A1012BB98601BEE24D9
:10BAD0001A12B092850A0CE508250CFAE43509FB28
:10BAE00012468B7408250AF50A8E828F83A3A3A3BE
:10BAF000A3A3A3E06058EE2407F510E43FF51185F9
:10BB00001082F583E0C0E012C8B5D0E012BBBDE002
:10BB1000C0E012C8B5D0E012BBBD1297C4122B4EC4
:10BB2000851082851183E025E0FCE433FD850A0C55
:10BB3000E508250CFAE43509FB123C9B7403122B33
:10BB400080851082851183E0C333250AF50AEE242F
:10BB50001512BB9B6008C0E012C8B5D0E0F012C857
:10BB6000A71297C5122B4EEE240D12BB9BFC7D0035
:10BB7000850B0A8E828F83A3E0F8E50828F8E43568
:10BB800009F9E8250AFAE439FB123C9B7403122BED
:10BB900080AA08AB0902BEB1EE241712B66422F8DF
:10BBA000E43FF988828983E022E0F50C750D0022DC
:10BBB000F582E43FF58312BBD6A3A3A322F0050AC6
:10BBC0008E828F83A3A3A3A3A3A3A3A322A3A312C1
:10BBD000DFE712BBD62212C0D3A3A32274F412252E
:10BBE0008074FD122C2A8A088B09ECFEEDFF74018B
:10BBF000122BE6880A890B780A122B527402122B38
:10BC0000F6EEFAEFFB1231077402122B80E970573F
:10BC1000851882851983E0850882850983F074017F
:10BC2000122E15E0F812BC70A3A312BC7E6029147A
:10BC3000850882850983A312BC7A12D75074011239
:10BC40002E15E028F8A3E039F9E824FEF582E9345E
:10BC5000FFF58312E9E4800C850882850983A3E45B
:10BC6000F0EEFAEFFB80047AFE7BFF740302989CEF
:10BC7000A3E0F98508828509832212BC8622E8F0B8
:10BC8000A3E912BC862212BC8A2212A514E02274F7
:10BC9000EE1225808A0A8B0BECFEEDFF750F01E991
:10BCA000C39408500302BE168E828F83E912AEC77A
:10BCB00012C0FA1232FFE96003750F0012C0DC8E69
:10BCC000828F8312C12CEE12B7713F12C116C0E0F1
:10BCD000EE2411F582E43FF583D0E012C10EC0E0FE
:10BCE000EE2412F582E43FF583D0E012B696740894
:10BCF00012BEA1A3A3A3E06018E50A2408F8E43566
:10BD00000BF912CAB912C8D98E828F83A3E0240816
:10BD1000F08E828F83A3A3A3A3A3A3A3A3E0601C9D
:10BD20008E828F83A385820885830912C0EFEE245B
:10BD30001512E29BA3E912CBCA2408F08E828F83EE
:10BD4000A3A3A3A3A3E0600F12BE888E828F83A358
:10BD5000A3A3A3A312BEA8EE241912C9CCEE241BE0
:10BD600012C9CCA3F0EE241812BB9B700302BE06CE
:10BD700012BE88FAEE2419F582E43FF583EA12BE7A
:10BD8000A8F8E50A28F582E412E292F812CBCEE890
:10BD900012BEA8E8C39AEE5068241912BB9BF89013
:10BDA0004FD2E493C398500575110C8008EE241906
:10BDB00012BB9BF5118E828F83A3E0F8E50A28F56C
:10BDC0000CE4350BF50D750E00780C122B4EAC11F2
:10BDD000EC2CFCE433FD7AC17B0E123C9B74031205
:10BDE0002B80EE241BF582E43FF58374C1F0A3742D
:10BDF0000EF0E511C333F8850882850983E02880B9
:10BE00000412C9C5E4F08E828F83A3E0F88E828F7E
:10BE100083E0C398500479008062A3E0FAE50A2821
:10BE2000F8E4350BF9EE241D12E29BA3E912C125BB
:10BE3000C39AC0E012BE7ED0E012C8C4603CEE24BB
:10BE400017F8E43FF9880889098882F583E024F22D
:10BE5000F0EE241D12BB9F240EFAA3E03400FB88F1
:10BE600082898312DA6B90053CE0F9122E61E9F8C1
:10BE7000850882850983E0C398F0A90F8033EE24FA
:10BE800017F582E43FF583228E828F83A385820893
:10BE9000858309E0F8E50A28F582E4350BF583E0AF
:10BEA0002212B69AA3A3A32212CBD804F022122BFB
:10BEB000807F0A02280574F41225808A088B09EA1B
:10BEC00012BF3DF0EA1313543F12BF36A3A3A3F0F1
:10BED000EAC4131312BF3DA3A3F0EB12BF4812BF75
:10BEE000507409780A122DA012BF4612BF4F740A6F
:10BEF000780A122DA0E50A5401C0E0EC2418F5825E
:10BF0000E43DF583D0E012BF55740B780A122DA0E2
:10BF100012BF46A312BF4F740C780A122DA012BF95
:10BF200046A3A3A3A3A3A3A3A3F0740D7808122D83
:10BF3000A0A90802989F540F8C828D832254038CF1
:10BF4000828D83A3A322E50A54018C828D8322A3D0
:10BF5000A3A3A3A3A3F08A0A8B0B22C082C0837978
:10BF6000008A828B83A3A3A3A3A3A3E090053B60D5
:10BF70000EE070228A828B83A3A3E070198016E002
:10BF800060148A828B8312D36E900544E06A70033A
:10BF9000A3E06B60010902C19C74F01225808A0A3B
:10BFA0008B0B890C8C088D098A828B8312C0FA1244
:10BFB00032FF12C0DC85088285098312C12CE50896
:10BFC00012B771350912C116C0E0E508241112C874
:10BFD000BCD0E012C10EC0E0E508241212C8BCD0EB
:10BFE000E012EE3F740812C108E0601EE50A240862
:10BFF000F8E4350BF9E508241312C8BC12C8D9853A
:10C000000882850983A3E02408F0850882850983D6
:10C01000A3A3A3A3A3A3A3A3E0601B850882850910
:10C0200083A312C0EBE508241512C8BCE8F0A3E90D
:10C0300012C1252408F0850882850983A3A3A3A340
:10C04000A3E06019850882850983A3AE82AF8312BD
:10C05000BE9385088285098312C12004F0AA08AB2B
:10C0600009123305E9F50D7061850882850983A3FE
:10C07000A3A3A3A3A312C0CF701AE0FAE50A2AF87B
:10C08000E4350BF9E508241D12C8BC12C8D9E50C2B
:10C09000C39A802A12C0EBE8240EF8500109E50883
:10C0A000241D12C8BC12C8D990053CE0F9122E61BB
:10C0B0008E828F83E0F8E50CC39824F2C399C0E028
:10C0C000E508241712C8BCD0E0F0A90D02C1641223
:10C0D000C0D322E0850882850983A322850A828550
:10C0E0000B83A3A312C142E0F9EA22AE82AF83E040
:10C0F000F8E50A28F8E4350BF922E0FAA3E0F8E4C1
:10C10000C8F9EA28E439FB2212EE22A3A32212C1C5
:10C1100055A3A3A3E022F583E812C14EA3A3E02216
:10C12000A3A3A3A3A3F08E828F83E022A3A3A3A340
:10C13000A3A3A3A3A312C14E12C142A3A3E0F9EA91
:10C14000F822E0FA850A82850B83A3A3A322F0A339
:10C15000E912C15522F0850A82850B83A3A3A3A30C
:10C1600022122B807F08022805C082C0837AC27BFE
:10C170000579E21248117AC27B058020C082C08313
:10C180009005448014C082C083900547800BC08214
:10C19000C083794A124811800312D377D083D082AA
:10C1A000022B3274F61225809005CAE0FE04F0EEF0
:10C1B000F91232A58B09EA450970EDEE60EAF90241
:10C1C000C51074EE122580EAFEEBFF8C0E8D0F89F0
:10C1D0000A750B00750C001234A38A088B097412BF
:10C1E000122E15E0F5107413122E15E0F50DEA4528
:10C1F000097017E50D600302C2E6A90AAC0EAD0F87
:10C20000EEFAEFFB1234C702C3F4E50D700302C26D
:10C21000AC900902E060046401700E9005D712CB67
:10C22000BD600612C627122766E510700B850882CE
:10C23000850983E4F002C2E1900902E0600764012D
:10C24000600302C30990053EE0A2E1400302C30976
:10C250009005D912CBBD600CA910AA08AB0912C673
:10C2600027122766850882850983E0FA12E2AE501C
:10C270000109C3EA98E499A2D265D0335009850830
:10C2800082850983E004F0850882850983E0F890BF
:10C290004FD4E493687072750B01EEFAEFFB123124
:10C2A00097850882850983A3E4F0805DE5107021FD
:10C2B000EA2402F582E412DF01850A0E250EF8E475
:10C2C000340013E813F070098A828B83A3A37401EE
:10C2D000F08A828B83A3A3E0F89010B1E0C398505A
:10C2E00028750C0180237401650D701DE51060191F
:10C2F000900902E060046401700F90053EE0A2E145
:10C300005007EEFAEFFB123197900902E0640260E9
:10C310000FE060046401702A90053EE0A2E1402233
:10C320007401650D701CE5109005E96013E004F0E0
:10C33000901085E0F89005E9E0C3984005750B0181
:10C34000E4F0E50CA2E092F0E50BA2E072F040030D
:10C3500002C3F4900902E060046401704190053E5C
:10C36000E0A2E15039EEFAEFFB122F098A088B099F
:10C37000A808A909E8496026E50CA2E0500D8882CA
:10C380008983A3A3A3A3A3E0C2E0F0E50BA2E0503E
:10C390006388828983A3A3A3A3A3E0D2E0F0E50B83
:10C3A000A2E05050900902E060046401701D900505
:10C3B0003EE0A2E15015EEFAEFFB122EF7E9600B1A
:10C3C000EEFAEFFB790012303B8029900547E06ED2
:10C3D0007003A3E06F701DEEFAEFFB790112303BA2
:10C3E000900902E06402700C7A017B0090059EE0E7
:10C3F000F9123E2D02BEB174F412258074016A4B0D
:10C40000700E7A017B0090059EE0F9123D018037A5
:10C4100090107C12DA6BEA4B60218A088B09E4F5F4
:10C420000AF50B7808122B4A7A017B0090059EE0F2
:10C43000F9123E217404122B80800C7A017B00904B
:10C44000059EE0F9123E2D02989FC082C083901095
:10C450007E02AAA9C082C08390108002AAA974F6A5
:10C460001225807508307509057808122B527C6EEC
:10C470007D007A217B00123DD37402122B80E9F5F6
:10C4800008122E85E94208900902E06004640170F8
:10C4900006122F33E9420890070B12CBBD60091238
:10C4A000C627122766E94208122E1FE9FE124247EC
:10C4B000E9F8E5084E48F9805774F61225801246CF
:10C4C000677508307509057808122B5275086E7566
:10C4D00009007808122B527C007D007A217B001223
:10C4E0003DDF7404122B80122E8B900902E0600451
:10C4F00064017003122F3990070D12CBBD60061234
:10C50000C627122766122E251242538003122B8053
:10C510007F0202280574F612258074FF122C2A7EF1
:10C52000007508307509057808122B527C6E7D0065
:10C530007A217B00123DD37402122B80E960030242
:10C54000C5F87808122B5275086E8E097808122BE0
:10C55000527C007D007A217B00123DE57404122B91
:10C5600080E9600302C5F8900544E064FE7003A30F
:10C57000E0F4700302C5F80E900553E0640860050E
:10C58000E06404706F851882851983EE12CA2379DE
:10C59000421248177A5B7B0579431248177A587B19
:10C5A0000579471248177A497B05794A1248177A64
:10C5B000477B05794B1248177A517B057950124811
:10C5C000177A447B0579531248177A597B057954B9
:10C5D0001248177A467B0579E112481790053EE02C
:10C5E000A2E35004D2F08002C2F012CA19795212AA
:10C5F000481780041246671E122E91900902E060CF
:10C600000464017003122F4B90070F12CBBD60061C
:10C6100012C627122766122E31EEF9740102C50DDB
:10C620008E828F83E0F8A3E0F58388822274F6126D
:10C630002580E9FEA2E050267508307509057808C6
:10C64000122B5275086E7509007808122B527C0067
:10C650007D007A217B00123DDF7404122B80EEA254
:10C66000E35003122E97900902E060046401700801
:10C67000EEA2E15003122F51EEA2E2500E900711EC
:10C6800012CBBD600612C62712276602C51074F6CB
:10C6900012258074EC122C2A7401122BF690102CA7
:10C6A000E0F97AA17B05123257900590E0640270A0
:10C6B0007C7405122E15E4F07407122E15E4F07A3E
:10C6C00004F9122EE58A08904FE5E493FAC3E508D1
:10C6D0009AEB9400400302C763122ED9E96003026B
:10C6E000C763904FC912C7BF60157A047903122E31
:10C6F000E5904FE5E493FC904FC912C7C950087408
:10C7000005122E157401F0904FC712C7BF60157A3D
:10C71000027901122EE5904FE5E493FC904FC71289
:10C72000C7C9503F7407122E157401803590055CFF
:10C73000122DF2E8494A4B600474018001E4C0E024
:10C740007405122E15D0E0F0900560122DF2E84924
:10C750004A4B600474018001E4C0E07407122E1596
:10C76000D0E0F090102CE0F97CA17D057401122B33
:10C77000EE1232517AA17B057945124817740712DF
:10C780002E15E070117405122E15E07009851882BF
:10C79000851983E480088518828519837401F090D7
:10C7A0001028E0F8901027E058F885188285198342
:10C7B000E05812CA237941124817741402C50DE4D7
:10C7C00093F8740193F9E84922E493F8740193F91A
:10C7D000ECC398F8E499F9C3EA98EB992274F7123C
:10C7E000258074ED122C2AE9FE90059DF0AC18AD61
:10C7F0001990102CE0F97AA17B05123257741212AD
:10C800002E15EE12C81BAA18AB191232517AA17B51
:10C81000057945124817741302B190F090102CE07E
:10C82000F97CA17D052274F4122580EAFEEBFF90CD
:10C83000102EE064FE7003A3E0F470687A167B00AB
:10C84000123CBF8A088B09EA450960588A828B83AB
:10C85000740112C8C48A828B83A3600474028002AC
:10C86000740112C8DFA3E08A828B83A3A3A3A3A3CE
:10C87000A3A3A3A312C8F5FCA3E0FDEA2402FAE4F3
:10C880003509FB12468BE508241312C8BCE4F0AA54
:10C8900008AB0990059EE0F9123CCB12C8A712D153
:10C8A0002812C8D902989F12C8AB22EE240BF58239
:10C8B000E43FF58322850A0CE508250CF582E43572
:10C8C00009F5832212C8C9E022F08E828F83A3A3C8
:10C8D000A3A3A3A322E01297B9E8F0A3E9F022F002
:10C8E000EE241DF582E43FF58312C8ED2212D13DFE
:10C8F000F583888222A3F0EE241512B6642274F226
:10C9000012258074FD122C2A8A088B09890A8C0B47
:10C910007401122E15740412CA231233958A0C8BDB
:10C920000DAE0CAF0DEE4F700302C9BAEE12B77127
:10C930003F12C9E97407F0A3A882A983E50824136C
:10C94000FAE43509FB8A828B8312C9FA8A828B83C7
:10C9500012C9F9E50812D36412DF018882898312B3
:10C96000CA057401F0E508240BF8E43509F9EE1264
:10C97000C9C512CA1212EDBF12331112DA62EE24C7
:10C980001312EDC17403650A60067401650A70072D
:10C9900012C9D57404800412C9D5E4F090102E1287
:10C9A000AD3B12C8D97401650B7006EE241112C993
:10C9B000CCEEFAEFFB122F818002791090102E122C
:10C9C0009B9002D14412EE0B22EE2412F582E43F3A
:10C9D000F583E4F02212C9DD7440F0A322EE12DEEA
:10C9E000F33FF5832212EDE53BF58312C9EF22E018
:10C9F000F8A3E0F98882898322A3E088828983F002
:10CA0000A308A98322F0EE2416F582E43FF58322E1
:10CA1000A3A3E8F0A3E9F0EE22A2F0E433851882A4
:10CA2000851983F0AA18AB192274F4122580EAFE46
:10CA3000EBFF7A007B0490059EE0F9123E2D12CAAE
:10CA4000C712C8D99005537409F01233118A088BA4
:10CA500009AC08AD0912CAB912D377124685E96448
:10CA60000170537A0F7B00123CBF8A088B09EA459C
:10CA70000960438A828B837402F012CAD1FC8882D7
:10CA80008983A3A3E0FBEC8A82850983A3A312DA3E
:10CA90006C88828983A3A3A3E08A8285098312C854
:10CAA000F5FAA3E0FB794A124817AA08AB099005EA
:10CAB0009EE0F9123CCB02989F12CABD22EE2413CD
:10CAC000F582E43FF5832290051612D1389010804C
:10CAD00022EE241DF582E43FF58312CDA2E02274FC
:10CAE000F412258074FD122C2A8A088B0974011215
:10CAF0002E15740212CA231233958A0A8B0BAE0AC2
:10CB0000AF0BEE4F700302CBA912EE2A7008888299
:10CB10008983A37420F0850882850983A3A3A3A336
:10CB2000A3E06401700988828983A3E0D2E6F085DE
:10CB30000882850983A3A3A3A3A3A3E06401700AC9
:10CB400088828983A3E0D2E7800312EDA112EE1B55
:10CB50007019850882850983A3A312CBBD6006EEF8
:10CB6000241612EDC112EDFD12C8D985088285097F
:10CB700083A3A3A3A3A3A3A3E06401700312EDD234
:10CB800085088285098312D3771233B3E9600312D3
:10CB9000EDCB12EDBE12331112CBC312CBAF12CAC2
:10CBA00010FAEFFB122F818002791002BC6BE0F8C3
:10CBB000A3E0F98E828F832212B284F58312D138DA
:10CBC000E8492212CBCEEAF0A3EB12CBD822EE2416
:10CBD0001AF582E43FF58322F0850882850983E017
:10CBE0002274F512258074F3122C2A890AEAFEEBCE
:10CBF000FF7508007509007C0D7D007900AA18AB4F
:10CC000019123CA7EE12D7583FF58312CD8E741F30
:10CC100058600C7AD37B0012426B790002CCE0E8BA
:10CC2000A2E55008740C122E157401F0E8A2E7502A
:10CC300008740B122E157401F0E8A2E6740A50086D
:10CC4000122E157401F08008122E15E06401701385
:10CC50008E828F83A3A3A3A3A3A3A3E06032EE24B9
:10CC60001380128E828F83A3A3A3A3A3A3A3A3E005
:10CC7000601EEE2415F582E43FF58312A7056010CF
:10CC8000AC08AD097402122E15AA82AB8312468B32
:10CC900012C8A712C8D5740A122E15E064017037A5
:10CCA00012D36A1233B3E97035EE240B12B8EA904E
:10CCB0000547E0687003A3E0697023E50845096053
:10CCC00016123311EAFCEBFD7402122E15AA82AB88
:10CCD00083124685E96007AA18AB19123035A90AF4
:10CCE00002EF3274F712258074D2122C2AEAFEEB7E
:10CCF000FF8E828F83129D31A2E0400302CD891204
:10CD0000CD95E054FE12E6BC740D122BF612CDB296
:10CD100012330BE97073742A122E1512CDAC7069A0
:10CD20007C0D7D007900AA18AB19123CA77416126D
:10CD30002E1512C8D5742A122E1512CD8EA2E550CA
:10CD400008740B122E157401F0E8A2E75008740A5B
:10CD5000122E157401F0E8A2E650047420800274CB
:10CD600022122E1512B0987402122E15AA82AB83CD
:10CD700012468B8E828F83A3A3E0C0E0740C122E28
:10CD800015D0E012CA2312302F742E02B19012C8AF
:10CD9000EDA3E0F8228E828F8312CDA2A3A3A3A3DA
:10CDA000A32212D13DF988828983A32212B263643F
:10CDB0000422EA241EF582E43BF583E0F9EA241F0D
:10CDC000F582E43B12989322E9F8790074046860D4
:10CDD0000A740A686005740368700109022B3274D2
:10CDE000F61225808A828B837420F0A3A37401F04D
:10CDF000122F878A088B09AE08AF09EE4F60168E96
:10CE0000828F837401F0900591E0700912EDBE12DB
:10CE1000331112DA62EEFAEFFB02C510C082C08352
:10CE200090054102AA48C082C08390102D02AA48F2
:10CE3000C082C083E990102D02AAADC082C0839049
:10CE400005B67401F0E9A2E350037403F0E9A2E12E
:10CE50005004E0D2E2F002C19C74F6122580790001
:10CE60007C008A088B09780812284BF8FF078ACEC5
:10CE700088CE88CE88CE88CE80CE84CE8ACE85CE0F
:10CE80007C0480060C0C80027C089005B6E05C6097
:10CE900003098003EC60010902C51074F4122580B7
:10CEA000EAFEEBFF8908122F0F8A0A8B0BA80AA94A
:10CEB0000BE849604188828983A3A3A3A3E060367D
:10CEC000C39405503174016508601A88828983A370
:10CED000A3A3A3E06401600D88828983A3A3A3A315
:10CEE000E06402700A8882898312A7E2122766EE44
:10CEF000FAEFFB122F1B02989F74F61225808A828C
:10CF00008B83E07012A312CBBD600C8A828B8312DC
:10CF1000D3761249B580047A007B0002C510C08226
:10CF2000C083900590E06402700B900553E06408A4
:10CF300070031233D702C19CC082C0837C00EC1204
:10CF4000CFEB7003A3E06B7011904FD9E493C0E076
:10CF500012CFBAD0E0F079C580510CECC3940340F5
:10CF6000DD7C00EC75F003A4F8A9F074BA28F58212
:10CF7000740512977C64FE7003A3E0F4600F0CEC60
:10CF8000C3940340DE7C00EC12CFAE7015EC12E3CC
:10CF90005512DA6B904FD9E49388828983F0790037
:10CFA00080090CECC3940340DE79C702C19C75F084
:10CFB00003A4F8A9F012CFBAE02274B928F582745C
:10CFC0000539F58322C082C0837D00ED12CFEB705E
:10CFD00003A3E06B700912CFB56004790180090DDD
:10CFE000EDC3940340E5790002C19C75F003A4F8F9
:10CFF000A9F074BA28F582740512E80E6A2274F258
:10D0000012258074DD122C2AEAFEEBFF750A0090CF
:10D010000902E060076401600302D122900544E048
:10D020006E7003A3E06F701EEE4F700302D1169076
:10D0300005CB12CBBD700302D116750A0112C627AB
:10D0400012276602D122122F098A088B09EA4509A4
:10D05000700302D1168A828B83A3A3A3A3E0640189
:10D0600060108A828B83A3A3A3A3E06402600302FF
:10D07000D116851882851983E412D12F740B122ED4
:10D0800015E8F0A3E912CA23122ECDE9700302D1EC
:10D090001685088285098312D12812C8D979001211
:10D0A00030E385088285098312DA6B7403122E152A
:10D0B000AC82AD837418122E15AA82AB8312468BF4
:10D0C00085088285098312B8F07420122E1512C8C3
:10D0D000D97422122E15E4F07C028508828509831A
:10D0E000A3A3A3A3E0F9740D122BEE1233718508EC
:10D0F0008285098312B8F07401122E15E8F0A3E9B5
:10D1000012CA23122ED3750A01E508240C12C8BCDA
:10D110001297DDF0800C90055112B682FAEFFB12E7
:10D12000348BA90A7423801E12D13890102E22123B
:10D13000AECB12D13622A3A312D13DF922E0F8A33F
:10D14000E022A90A7403122B807F06022805C08200
:10D15000C08374FE122C2A900902E06004640170FE
:10D1600029790190052912C62412276612D18F90C1
:10D170000544E8F0A3E912CA237953124817851829
:10D180008285198312D377123F3574020284E385B6
:10D190001882851983EAF0A3EB12D19EF92212BC02
:10D1A0008AF8A3E02274F512258074F3122C2A8ADF
:10D1B000088B09ECFEEDFF750A12EA450970057946
:10D1C0000002D2B2900544E065087004A3E065094E
:10D1D0007019123311EAFCEBFDEEFAEFFB124685F3
:10D1E000E97005750A018003750A008518828519A2
:10D1F00083E4F004122E15E508F0A3E50912CA2312
:10D20000122EC1E960297403122E15AA82AB831273
:10D210002EA3E964017018750A017403122E15AC6F
:10D2200082AD83EEFAEFFB124685E9701E801F7413
:10D2300012650A7019900590E064027011EEFCEF1F
:10D24000FDAA08AB09122EF1E96003750A00EEFC95
:10D25000EFFDAA08AB091234A9E9F8740A68700551
:10D26000750A01804274A0687037EEFCEFFDAA08D1
:10D27000AB091234BB7E008023EE75F017A4F8A929
:10D28000F012E8247004A3E06509700F12E960123F
:10D290002EA3E9700612E4FF1234970E12D2B540A5
:10D2A000D87401650A70097900AA08AB091233E93C
:10D2B000A90A02EF32904FD1E493F8EEC39822749A
:10D2C000F6122580EAFEEBFF8908900902E060046F
:10D2D0006401701E1233D7E508F5097809122B5640
:10D2E000790DEEFCEFFD7AFC7BFF1233F574011231
:10D2F0002B8002C51074F7122580EAFEEBFF8E82A8
:10D300008F83A3A3A3A3A3A3A3A3E0601312D35C5F
:10D310001298861233E3E96401700512C8A7802DC4
:10D320008E828F83A3A3A3A3A3A3A3E0602912CA21
:10D33000B912D37BFAA3E0FB1233E3E9640170175F
:10D340008E828F83A3A3A3A3A3A3A3A3A312D377A4
:10D350001233CB79018002790002B193EE12D364CB
:10D360003FF583222415F582E4228E828F83A3A3C6
:10D37000A3A3A3A3A3A3A31298952212D387A3A325
:10D38000A3A3A3A3A3E02212B0A08E828F83A3A3A2
:10D390002274F212258074FD122C2A8A088B09EC63
:10D3A000FEEDFF890B750A017401122E157404122B
:10D3B000CA23123395EA4B60477411122E15E060B0
:10D3C0001AEA2417F582E43BF583E412DC178A821B
:10D3D0008B83E0D2E7F012D403E4F012C9E57403C2
:10D3E00012D671EE88828983A3A3F0EF88828983A5
:10D3F000A3A312AEC6A3A312F00F122F81E9F50A60
:10D4000002D142EA2414F582E43BF5832274F0123F
:10D410002580EAFEEBFF890A750B0112CAD1F50CD3
:10D4200088828983A3A3E0FA8882898312D54A126D
:10D43000BB986404600A7AD37B0012426B02D54524
:10D44000E50C122A160200025AD4030BFAD4030C7C
:10D45000E1D40DB9D40EFAD4F8D4900902E06007F3
:10D460006401600302D4FA90053EE0A2E1400302A9
:10D47000D4FA7900AB09123179EA4B60318A828B98
:10D4800083A3A3A3A3A3A3E05418602212C8A712E6
:10D4900029918A828B83A3A312299179008E828F8E
:10D4A0008312D5691231917404122B80802E790178
:10D4B000AA08AB091230478041900902E060046479
:10D4C00001703790053EE0A2E1502FAB091233C541
:10D4D000AA08AB091233CBE964C5701E750B008036
:10D4E00019900902E060046401700F90053EE0A20B
:10D4F000E15007123F598002880AEE2409F50EE434
:10D500003FF50FAC08AD09A90C850E82F58312D347
:10D510007712305F850E82850F8312D3771233B373
:10D52000E96022EE241112BB9BC39402401712C87B
:10D53000A712DB317003A3E069600AE50BA2E0509B
:10D5400004A90A8002790002C164A3A3A3E0F8E45D
:10D55000C8F9EA28F508E439F50922E508240CF5AC
:10D5600082E43509F58312B640A3A3A3A3A3A3A322
:10D57000A3A312B09C8A828B831298952274EE1218
:10D58000258074F5122C2A8A0A8B0B890C8C0E8D3F
:10D590000F7E01EE122E15740AF0741D122E15E086
:10D5A000F50DE9700FE50DC333240AC0E0EE122E2D
:10D5B00015D0E0F0AA18AB191233958A088B09EA46
:10D5C0004509700302D66612B770350912D7F37495
:10D5D0000912D7FF450D12D691AC0EAD0FEEFAEF42
:10D5E000FB12468BEE2408FE50010FE50C70247CE4
:10D5F00000741E122E1512B8F08012EC12DB1DE81A
:10D600002AFAE93BFB12D677A30EAF830CECC39545
:10D610000D40E8E508241712C8BC7401F01233115C
:10D62000E508241AF582E4350912DA697403122B2D
:10D63000F6AA0AAB0B122EA9E96019E50824161206
:10D64000C8BC7401F07403122BE6E508241812C854
:10D65000BC12C8D985088285098312D66DAA08AB89
:10D6600009122F81E9FEEEF9740B02BEAEA3A3E509
:10D670000AF0A3E50BF0228A828B8312D68B12D696
:10D68000918A828B8312D68AF022A3E08E828F83C6
:10D6900022F0A3AE82AF832274F012258074F812B8
:10D6A0002C2A8A088B0912D757350912D878F50B1E
:10D6B000880AA3AE82AF83EEFCEFFDAA18AB191265
:10D6C000468BEE2408FE50010FAC18AD197A657B2D
:10D6D00005124685E9607474E0550A7067AA0BEA82
:10D6E0002AFA7B00123D5B8A0C8B0DEA450D605BCC
:10D6F0007C00801E8E828F8312C0FAEC12D750E518
:10D700000C28F582E50D3912DA69EE2402FE50018B
:10D710000F0CECC3950B40DC780C122B52780B12DB
:10D720002B567403122BF67900E508240B12C8BCA3
:10D7300012D37712340D7403122B80AA0CAB0D1286
:10D740003D6180077AD37B0012426B740802C1618D
:10D7500025E0F8E433F922EA241DF582E42274F08E
:10D760001225808A0A8B0B890C8C088D099007DEA4
:10D7700012CBBD607B7410122E15E0F50D12D75040
:10D78000E8240EFAE439FB123CBF8A0E8B0FAE0E72
:10D79000AF0FEE4F605A8E828F8374D4F0A3A3E54F
:10D7A0000AF0A3E50B12BEA1E50CF0AC08AD09EE42
:10D7B0002405FAE43FFB12468B12B277E50DF074B4
:10D7C00011122E1512DC017808122B4EAC0DEC2C28
:10D7D000FCE433FDEE240EFAE43FFB123C9B7403A1
:10D7E000122B80EEFAEFFB9007DE12C6241227669A
:10D7F00002C164F583E0FEA3E0FF8E828F8322F0F6
:10D80000A3E50CC43354E02274F612258074F81298
:10D810002C2A890812D7573B12D878F98809A3AE69
:10D8200082AF837401697042EEFCEFFDAA18AB1958
:10D8300012468BEE2408FE50010FAC18AD197A6524
:10D840007B05124685E9602974E05509701C8E82BB
:10D850008F83A3E0FA8E828F83A312C0FC8E828F07
:10D8600083E0F9123425A90880097AD37B0012429B
:10D870006B7900740802C50DF583E02401FEA3E076
:10D880003400FF8E828F83E0F8741F582274F612E2
:10D89000258074DF122C2AEAFEEBFF12CBB8605011
:10D8A0008E828F8312D377AC18AD1912CDB212329B
:10D8B000F97409122E1512DB317003A3E069603090
:10D8C00012C6201229917508FE7509FF7808122BDF
:10D8D00052741C122E15E0F9740D122E1512B09808
:10D8E000740F122E1512D3771231917404122B80FB
:10D8F000742102C50D74F7122580E9FC7A007B00C3
:10D900007E00800B12D997E02AFAA3E03BFB0E9031
:10D910004FE512D2B85029EE75F016A4F8ADF0ED2F
:10D92000F912E813F460E7743328F582740A3912A7
:10D93000CBBB60DAEC60CD12D997E4F0A3F080CED7
:10D940007E00800B12D984E02AFAA3E03BFB0E1282
:10D95000D2B5502DEE75F017A4F8ADF0EDF912E93F
:10D96000717003A3E0F460E6740628F582740C3944
:10D9700012CBBB60D9EC60CC12D984E4F0A3F08068
:10D98000CD02B193EE75F017A4F8EDF9740628F501
:10D9900082740C39F58322EE75F016A4F8EDF97453
:10D9A0003328F582740A39F5832274EC12258089B4
:10D9B0000CEAFEEBFF90059DE0C3950C503B123343
:10D9C000659005CD12DA5C900537E0F508E4F509BD
:10D9D000F50AF50B9080FC7810122DBE78087910AE
:10D9E00012241B7808122B4A7A007B0290059EE0D5
:10D9F000F9123E217404122B8002977474F61225DA
:10DA000080EAFEEBFF9005B7801388828983E06E81
:10DA10007003A3E06F603688828983A3A312CBBD15
:10DA200070E87A047B00123D5B8A088B09A808A97C
:10DA300009E84960188882898312DA5C9005B71278
:10DA4000DA50A3A312DA6B9005B712C8D902C51039
:10DA500012989588828983228A828B83EEF0A3EFC5
:10DA6000F022EE241AF582E43FF583EAF0A3EBF00E
:10DA70002274F41225807E009005B780070E8882FC
:10DA80008983A3A312CBBD70F4EE12DB1D123D5BA4
:10DA90008A088B09EA4509607E7F009005B78021DE
:10DAA0008882898312B098EF12DB1DE5082AF5827F
:10DAB000E5093BF583ECF0A3EDF00F88828983A3A1
:10DAC000A312CBBD70DA90059912DB317003A3E08D
:10DAD000697808701C122B52EEF50A780A122B5640
:10DAE0007C657D05790090059912D37712340D80FD
:10DAF0001A122B52EEF50A780A122B567C657D0518
:10DB0000790090059912D3771234017403122B8097
:10DB1000AA08AB09123D61122F9902989F25E0FADD
:10DB2000E433FB228E828F83A3A3A3A3A3A3A3A387
:10DB3000A312D138900544E06822C082C0838012CD
:10DB40008A828B83A3A312B8F09005B712C8D912AA
:10DB50003D619005B712B03B70E602C19C74F512AE
:10DB6000258090055112B8F79005CD12DBF512C84B
:10DB7000D97ACD7B0579501248179005CD12DC017A
:10DB8000801512E3B365087004A3E065096006120E
:10DB9000E507123497050A12DBEA5018E50A12E489
:10DBA000F37003A3E06F70DA74FB28F582740B1234
:10DBB000F00C80E19005CD12B8F79007E012CBBDD4
:10DBC00060257A067B00123CBFEA4B601A8A828B82
:10DBD0008374D5F0A3A3E412DC080412DC179007C9
:10DBE000E012C62412276602EF37904FD1E493F873
:10DBF000E50AC3982212DBF92212D13DF9900551B2
:10DC00002212AD22750A002212DC0C2212DC102234
:10DC100012AECBA3A3A32212DC0CA3EEF0A3EFF071
:10DC200022C082C0839005CF744FF0A37434F0906B
:10DC300005D17449F0A37434F09005D37467F0A350
:10DC4000743402AAADC082C083900544E064FE70C3
:10DC500003A3E0F4600E90053EE0A2E1500612340A
:10DC6000AF12345502C19C74F0122580900592E0E9
:10DC70006053F50CE4F50DF50EF50F9080F0780883
:10DC8000122DBE780C790812241B123CB98A088B1D
:10DC900009A808A909904FC3E49358F508A3E49391
:10DCA00059F509E4F50AF50B780C7908122CF3788C
:10DCB0000C122B4A7A007B0190059EE0F9123E2758
:10DCC0007404122B8002C16474EE1225807E007FE2
:10DCD000008E0A8E0B122F5D8E0D803E850D08AAD8
:10DCE000087B00122F578A088B09A808A909E84960
:10DCF000602688828983A3A3A3A3E06004640470E0
:10DD00001788828983A3A3A3A3A3A3A3A3A3A3E0A8
:10DD1000F91234C1E960010F050D904FE5E493F865
:10DD2000E50DC39840B61234858A0E8B0F8E0C8099
:10DD300023AA087B001234918A088B09A808A90934
:10DD4000E849600EE8240F129779F91234C1E960AE
:10DD5000010E050C850C08C3E508950EE4950F40EF
:10DD6000D0EF2EFE700302DE618E0875090074028A
:10DD70007808122D2CAA08AB09123D5B8A0A8B0B7E
:10DD8000EA450B700302DE5F750C008E0875090012
:10DD900074027808122D2CAC08AD0979FF123CA74B
:10DDA000750D00805D850D08AA087B00122F578A2B
:10DDB000088B09EA450960488A828B83A3A3A3A341
:10DDC000E06004640470398A828B83A3A3A3A3A3B5
:10DDD000A3A3A3A3A3E0F91234C1E96023050C783F
:10DDE0000A122B52EEFD850882850983A3A3A3A303
:10DDF000A3A3A3A3A312DF0712345B7402122B8028
:10DE0000050D904FE5E493F8E50DC3985006E50C39
:10DE1000C39F4091750C00850C08C3E508950EE47E
:10DE2000950F503DAA087B001234918A088B09EAAD
:10DE300045096027EA12DEF312DF01F91234C1E965
:10DE40006019780A122B52EEFDE508240E12C8BCA8
:10DE500012DF0712345B7402122B80050C80B87E2F
:10DE600000750E6290053CE0600CF9122E61E9F835
:10DE70007454C398F50E75F003E50E84F50D9420E7
:10DE80004003750D1F850A08850B09750C00E50E0A
:10DE90006006750C20750E00E50DC39E5004AF0D95
:10DEA0008008EEFFE50CD2E6F50CAC08AD09AA0C33
:10DEB000EFF9123461E9F50FE50CA2E6401A1F787C
:10DEC00000800BE5082404F5085002050908E8C3A2
:10DED0009F40F0EFCEC39EFEE97006E50CA2E6502F
:10DEE000AAE50A450B6007AA0AAB0B123D61A90F10
:10DEF00002BEB1240FF582E422748E2508F58274E7
:10DF00000F3509F583E022E0FC850882850983123C
:10DF100098952274F2122580EAFEEBFF89088C099D
:10DF20008D0A7C007D00740E122E1512D3778C0B97
:10DF3000800DEAFCEBFDEA2404FA50010B050BE529
:10DF40000BC3950A400302DFDE8A828B83E0F47004
:10DF500003A3E0F46077EC4D600C8C828D83C3E00A
:10DF60009EA3E09F50CC8A828B8312E322EE98EF2F
:10DF70009950BFEAF8EBF988828983E0F47003A333
:10DF8000E0F46010E82404F8500109050BE50BC328
:10DF9000950A40E3E8FCE9FDE824FCF8E934FFF9E0
:10DFA000888289831297CE8C828D83E50CF0A3E55D
:10DFB0000D12DFE18C828D83A3A312E6B6E08C8282
:10DFC0008D83A3A3A3F0C3EA98EB9940C712DA5854
:10DFD0008A828B83A3A3E50912DC08E508F002D14D
:10DFE0004912DFE7A3E022F088828983A32274F23A
:10DFF00012258074FD122C2A89088A09ECFEEDFF97
:10E00000750A0175F003E9A42402C0E07401122E20
:10E0100015D0E012CA23123395EA4B607812C9E595
:10E020007408F0741F55084509A3F0E82402F8505D
:10E030000109750A0080388E828F83E08882898387
:10E04000F0A3A882A9838E828F8312C9F98E828F52
:10E0500083A3A3E05407C4FC8E828F83A3A3A3E011
:10E0600054074C12C9FBEE2404FE50010F050AE5CB
:10E070000AC3950840C18A828B83A3A374FCF0A3D2
:10E0800074FFF0EA2413F582E43BF5837401F01287
:10E090002F81E9F50A02D14274F11225808A0A8B98
:10E0A0000B7508007AFE7BFF7CFE7DFFE50A12D728
:10E0B00058350B12CAD8F509741F5509F50CE82418
:10E0C00002F8500109E509A2E7406FE50A2417F5B7
:10E0D00082E412E292FE75F003E50CA424026E7055
:10E0E00059E50C600B88828983E0FEA3E0FBEEFA21
:10E0F000750D00801DE05407F50EA3A882A983EEDC
:10E10000FC900544E06E7003A3E06F7003850E0879
:10E11000050DE50DC3950C502B88828983E0FEA385
:10E12000E0FCE4CCFDEE2CE43DFFE82402F85001D5
:10E130000988828983E0548860BB7AD37B001242CD
:10E140006B02E287E508700BA90912346DE97003D0
:10E1500002E28712E2A412D377122F098A0C8B0DE8
:10E16000AE0CAF0DEE4F605A8E828F83A3A3A3A394
:10E17000A3A3A3E4F0904FD493F88E828F83A3A33C
:10E18000A3A3A3A3A3A3E0C398402412E2AE50012B
:10E19000097A027B00122323E88E828F83A3A3A334
:10E1A000A3A3A3A3A3F0E508C39407500205088E18
:10E1B000828F83A3A3A3A3A3A3A3A3A3E508F00231
:10E1C000E2877CFF7DFF12E2A412D3771234798AB2
:10E1D0000C8B0DAE0CAF0DEE4F704F12347F8A0CCE
:10E1E0008B0DAE0CAF0DEE4F700302E2877C177DF6
:10E1F000007900123CA712E2A412CBAE1284D58E95
:10E20000828F83A3A3A3A3A3A3A3A312CA1012B6AE
:10E210005974AA12E2CD5001097A027B001223231D
:10E2200012B277E812E2B97401F0904FD4E493F897
:10E23000EE240D12BB9BC398401912E2AE500109A7
:10E240007A027B0012232312E298E508C394075058
:10E2500002050812E91FE50812E2BEE4F0129CC6AE
:10E26000122EA3E97021850A82850B83A3A3A3A3A1
:10E27000A3A3A3A3E06010E50A12D364350B12B682
:10E2800080129CC712468B02A8C3748E250AF582A1
:10E29000740F350BF583E022EE240DF582E43FF593
:10E2A00083E8F022E50A12EDE6350BF58322904F64
:10E2B000D4E49379002401F822F012E92322F01229
:10E2C000E2C322EE240CF582E43FF58322F0904F66
:10E2D000D4E49379002401F82274F7122580E9FE32
:10E2E00074FE6A700374FF6B603474605E64606017
:10E2F0002DEEA2E5401CA2E6900544500DC3E09A25
:10E30000A3E09B5019790002B193C3E09AA3E09B6C
:10E3100040F390054412E322EC98ED9940E779012F
:10E3200080E512D138C32274F71225807E00800761
:10E3300012E4FF1234970E12D2B540F47E00EE12B2
:10E34000E355129B9088828983E4F00EEEC3940318
:10E3500040EC02B19375F003A4F8A9F074B928F861
:10E36000740539F988828983A32274F71225807F86
:10E370000080010F904FD1E493F8EFC398502DEF38
:10E3800075F017A4F8A9F012E7FF6A7003A3E06B19
:10E3900070E112E3B36C7003A3E06D600A74FF6C6C
:10E3A000700374FF6D70CC12E50780047A007B0067
:10E3B00002B19312E3B72274FB28F582740B12E8C2
:10E3C0000E2274F61225807CFF7DFF7AFE7BFF1201
:10E3D0003479EA4B703C7508008032E50875F01717
:10E3E000A4F8A9F0740028F582740C12977C6005DB
:10E3F00012E7F4701674F128FE740B39FF8E828FC9
:10E400008312D377123197EEFAEFFB050812E41569
:10E4100040C902C510904FD1E493F8E508C3982293
:10E42000C082C0837A007B007D00801012E9697091
:10E4300003A3E0F460050AEA70010B0D904FD1E4EC
:10E4400093F8EDC39840E502C19C74F41225808ACC
:10E45000088B09ECFEEDFF800B123497EEFCEFFD0C
:10E46000AA08AB09123479EA4B70EE02989F74F651
:10E470001225807D007E0080020D0E12D2B550184C
:10E48000EE12E96A7003A3E0F460EF8D08EA650814
:10E490004B70E612E50780047A007B0002C5107419
:10E4A000F7122580EAFEEBFFEE4F601A7C177D0025
:10E4B0007900123CA78E828F8374FEF0A30412AD04
:10E4C00045A314129B9202B19374F7122580EAFEC1
:10E4D000EBFF7508008014E50812E4F37003A3E075
:10E4E0006F600612E507123497050812E41540E73D
:10E4F00002B19375F017A4F8A9F012E3B76E22EEFB
:10E5000075F017A4F8A9F074F128FA740B39FB22FE
:10E5100074F41225808A088B09ECFEEDFF90090245
:10E52000E0600464017020900551E06E7003A3E088
:10E530006F7014122F098A0A8B0BA80AA90BE849DD
:10E540006005E82408801AEEFCEFFDAA08AB09126A
:10E5500034798A088B09A808A909E8496009E824E0
:10E560000DFAE439FB80047A007B0002989F74F472
:10E570001225808A0A8B0BECFEEDFF7508007509E9
:10E58000008034E50912E959122EA3E96027E50954
:10E5900075F017A4F8A9F012E81E7004A3E0650B4B
:10E5A000700375080AEEFCEFFD12E960124685E97A
:10E5B00060034308A00509904FD1E493F8E509C32F
:10E5C000985004E50860BC02BF3174F61225807EC5
:10E5D00000805C8E08AA087B00122F578A088B09DE
:10E5E000A808A909E849604688828983A3A3A3A350
:10E5F000E06401603988828983A3A3A3A3E0640255
:10E60000602CE82407129779FA74012AF090059398
:10E61000E0C39A501988828983A3A3A3A3A3A3A3C9
:10E62000A3A3A3E412E6ADA312E6BC1231970E90A9
:10E630004FE512D2B8409C7E008059EE75F017A4C9
:10E64000F8AAF0EAF912E9717003A3E0F4604474E7
:10E65000F128F8740B39F9E8240C129779F8740151
:10E6600028F0900593E0C3985029EE75F017A4F8B0
:10E67000EAF974F128F8740B39F9E812DEF339F588
:10E6800083E4F0E8240EF582E439F583E412E6BC75
:10E690001231970E12D2B540A27B00EB12CFAE60C2
:10E6A0000214F00BEBC3940340F102C51012E6B65E
:10E6B000A3A3A3A3A32212DFE7A3A32212E6C4FA13
:10E6C000A3E0FB22F088828983E02274F312258084
:10E6D0008A088B09ECFEEDFF750C007B007C017451
:10E6E0000D122E15E0F50AA3E0F50B8010123CB9CF
:10E6F000E50CF5F0EA84ABF0750C007C007D008041
:10E70000010D904FD1E493F8EDC398504912E96997
:10E710007003A3E0F460EA12E8247004A3E0650942
:10E7200060DF12E7FF6E7003A3E06F60D412E81E93
:10E730007004A3E0650B60C912E7F460C4C39407DA
:10E7400050BFEC050C70BAE50CC39B40B474F128C3
:10E75000F582740B80787A0080010A904FE5E4938B
:10E76000F8EAC3985070EA75F016A4F8A9F012E818
:10E770002A64FE7003A3E0F460E012E82A650870E2
:10E7800004A3E0650960D312E82A6E7003A3E06F6A
:10E7900060C812E82A650A7004A3E0650B60BB74C8
:10E7A0002C28F582740A12977C60AFC3940750AA94
:10E7B00012E813640160A3E06402609EEC050C7033
:10E7C00099E50CC39B4093742328F582740A39F5AC
:10E7D0008312D3778019E50C6011EB700E7401651C
:10E7E0000C600302E6ED7B0102E6F87AFE7BFF7F18
:10E7F0000502280574FF28F582740B12E80E221218
:10E80000E8032274F128F582740B12E80E2239F520
:10E8100083E022742728F582740A12E80E2212E897
:10E8200003650A2212E803650822742328F582741E
:10E830000A12E80E2274F51225808A088B09ECFE74
:10E84000EDFF750A008002050A12DBEA5022EEFC99
:10E85000EFFDE50A12E959124685E960EAE50A7515
:10E86000F017A4F8A9F074F128F582740B12F00CDB
:10E8700002EF37E9F87907C3940D40047901801954
:10E88000E8C3940740047903800FE8C3940340046D
:10E8900019198005E870027900022B3274F01225F4
:10E8A000808A088B098C0A8D0B890C12347F8A0EA2
:10E8B0008B0FAE0EAF0FEE4F60627C177D007900BC
:10E8C000123CA78E828F8312F00F8E828F83A3A3B8
:10E8D000A3A3A3A3A3A312D66DE50C600712B65899
:10E8E000E50C800512B6587401F09005D112CBBD2D
:10E8F0006015900598E06401700612E91FE4800C31
:10E9000012E91F7407800512E91F740112E2CD504D
:10E9100001097A027B0012232312E29802C16412D9
:10E92000E92322EE240EF582E43FF5832274F712E8
:10E9300025807E00801BEE12E96A7003A3E0F4607C
:10E940000F12E960122EA3E9700612E4FF12349749
:10E950000E12D2B540E002B19375F017A4F8A9F0F9
:10E9600074F328FA740B39FB22ED75F017A4F8A99B
:10E97000F012E80364FE22C082C0839005D574D9EA
:10E98000F0A37434F09005D774DFF0A37434F090E2
:10E9900005D974E5F0A3743402AAAD74F71225808A
:10E9A000EAF8EBF990051412E9E4CA2406F582E4CA
:10E9B0003AF583E0702B88828983A3A3A3A3A3A342
:10E9C000A3A3A312299190051412E9E9122DE68858
:10E9D000828983A3E0F91230537402122B80122F24
:10E9E0009902B193E0FAA3E02212E9E4F5838A8266
:10E9F00022C082C08390059B12EAB4F090059B125E
:10EA0000CBBD7005790112341F02C19C74F612252A
:10EA10008074FC122C2AE9FE904FDAE4937008749B
:10EA2000E16E600302EAAFEA2408F8E43BF9888269
:10EA3000898312EAB412EABD700E90059BE4F0A33C
:10EA4000F0790112341F8067900904E06061FA9048
:10EA5000059B12E322EA98E4995054790012341F7E
:10EA60008A088B09AC08AD09ECF8EDF9E875F0649B
:10EA7000A4F8AAF075F064E9A42AF990059B12D3D2
:10EA80007712232BE8941AE9940040239007D812B8
:10EA9000CBBD601B90059B12C8D57402122E15ECDD
:10EAA000F0A3ED12CA239007D812C6241227667469
:10EAB0000402C50DE02401F0A3E034002212E6C4F4
:10EAC000F8A3E0F9E84922C082C08374F8122C2A26
:10EAD00090809AAC18AD197408122AAEAC18AD1912
:10EAE000124685E96401700479008002790102848C
:10EAF000E1C082C0839005DB7463F0A3742FF090B3
:10EB000005DD7469F0A3742FF09005DF74FDF0A3A8
:10EB10007434F09005E17403F0A37435F09005E3CC
:10EB20007409F0A37435F09005E5740FF0A3743503
:10EB3000F09005E77415F0A37435F074FD4434606B
:10EB4000031234FD02C19C74F412258074E9122C66
:10EB50002A8A088B097404122E157402F004122BF1
:10EB6000EE1233958A0A8B0BAE0AAF0BEE4F700391
:10EB700002ED8D12EE2A700888828983A37420F03A
:10EB8000850882850983A3A3A3A3A3E06401700978
:10EB900088828983A3E0D2E6F0850882850983A371
:10EBA000A3A3A3A3A3E06401700A88828983A3E0DE
:10EBB000D2E7800312EDA112EE1B70198508828541
:10EBC0000983A3A312CBBD6006EE241612EDC11279
:10EBD000EDFD12C8D9850882850983A3A3A3A3A349
:10EBE000A3A3E06401700312EDD285088285098336
:10EBF00012D3771233B3E9600312EDCB12EDBE12DC
:10EC0000331112CBC3FAA3E0FB8E828F83A3A3122E
:10EC1000DA6B1233B3E9600312C9C9EE241312BBD5
:10EC20009B700D904FDEE493C0E012CAB9D0E0F0C3
:10EC30008E828F83E0A2E7500454038019EE2414DF
:10EC400012BB9B7012900530E0C0E012ED97D0E04F
:10EC5000F0900530E004F012EDB070199008E1E09A
:10EC6000600D90053BE0700D8E828F83E07006EEA4
:10EC7000241112C9CCAC18AD19EEFAEFFB1232ED2B
:10EC80008A088B09EA4509700302ED817A217B002D
:10EC9000123D5B7406122E1512DA6B7406122E15D5
:10ECA00012CBBD700302ED75900902E060046401AF
:10ECB000700812B658A3E04404F07401122BEE79E8
:10ECC000501248117401122E1512B8F07406122E4B
:10ECD0001512E9E4CA2409F582E43AF58312C8D989
:10ECE00090054412B8F07415122E1512C8D9740686
:10ECF000122E1512B8E212EDDCF07406122E151267
:10ED0000AE17740212EE147406122E1512E9E912EF
:10ED1000BC7EC0E07406122E1512B8E212EDA7D028
:10ED2000E0F0EE240E12EDB9C0E07406122E1512BA
:10ED3000EDECD0E0F07406122E1512866412F00D80
:10ED4000EE240F12B8EA740C122E1512C8D98A825A
:10ED50008B83E0C0E0740E122E15D0E0F074061222
:10ED60002BEE123269E9F50A7406122E1512D377CA
:10ED7000123D618003750A10AA08AB09123D61803B
:10ED800003750A10EEFAEFFB123D618003750A105D
:10ED9000A90A741702989CEE2414F582E43FF583C7
:10EDA0002212CABD740122241EF582E438F58322A2
:10EDB000EE241112B66464012212B64BE022EE2456
:10EDC00017F582E43FF5837401F02212B661440422
:10EDD000F02212C9DD7401F0A3E4F02212EDE6384E
:10EDE000F583740222EA240BF582E42212EDF0226C
:10EDF00012D13DC8240CF582E438F58322850882BF
:10EE000085098312D136EE12EE0B222418F582E426
:10EE10003FF5832212B69A12D1372212EE22E06415
:10EE2000012212EE43A3A3A3A32212C8AB12C9EF7F
:10EE30007404F0A3E412EE3FA3A3A3E06401221242
:10EE4000EE4322F0850882850983A32274F61225F9
:10EE5000807E00801F7C047D0079FF8E088D097400
:10EE6000027808122D2C748E2508FA740F3509FBD0
:10EE7000123CA70E904FE012D2B840D902C51074D0
:10EE8000F512258074F7122C2A750A00801E850A57
:10EE90000875090074027808122D2C74902508F565
:10EEA00082740F12C8BF12EF25F0050A904FE012CE
:10EEB000DBED506D850A0875090074027808122D83
:10EEC0002C12DEF9F47003A3E0F460DE850A087505
:10EED000090074027808122D2C74902508F58274AC
:10EEE0000F350912CBBB70A67408122E157402F0F0
:10EEF000850A087509007808122D2C748E2508FEE5
:10EF0000740F3509FF8E828F8312C8D512EF2E122F
:10EF1000485F7C047D0079FFEEFAEFFB123CA7808E
:10EF2000897409800FE024FFF0A3E034FF2212F07F
:10EF30009C22740D122B807F0302280574F0122589
:10EF40008074F7122C2AEAFEEBFF8C088D09750CF1
:10EF5000FF7408122E1512F08E124859E9641A70C7
:10EF60000302F008750E00800B74FF650C700385BA
:10EF70000E0C050E904FE0E493F8E50EC398504850
:10EF8000850E0A750B007402780A122D2C12E28A83
:10EF9000F47003A3E0F460D1850E0A750B007402CF
:10EFA000780A122D2C12E28A6E7003A3E06F70C2F1
:10EFB000750F007402780E122D2C7490250EF582B8
:10EFC000740F350FF5838030E493650E702D74FF58
:10EFD000650C602E850C0A750B007402780A122DE0
:10EFE0002C748E250AF8740F350BF98882898312E8
:10EFF000DA5C88828983A3A312F00F790174090275
:10F00000C16112EF2E12485F790080F139F583E576
:10F0100008F0A3E509F02274F412258074F7122C8D
:10F020002AEAFEEBFF7408122E1512F08E12485FCA
:10F03000750A008002050A904FE012DBED504C8506
:10F040000A0875090074027808122D2C12DEF9F4F2
:10F050007003A3E0F460DE850A0875090074027885
:10F0600008122D2C12DEF96E7003A3E06F70C67CBF
:10F07000047D0079FF8D0B7402780A122D2C748E9A
:10F08000250AFA740F350BFB123CA702AE07740277
:10F0900012A514EEF0A3EFF012F09C22900551128D
:10F0A000B0A0AA18AB1922C082C08374F8122C2A0F
:10F0B00085188285198312DA6B7402122E15E4F01A
:10F0C000A3F07404122E157401F07405122E157439
:10F0D00001F07406122E15E4F07407122E15E412D6
:10F0E000CA231234F70284E174EE1225808A088B59
:10F0F00009ECFEEDFF750C00EE65087003EF650985
:10F10000600C123DD98A0A8B0BEA450B7006750C10
:10F110000102F1A4EEFAEFFB123DD98A0E8B0FAC7F
:10F120000EAD0FEC4D6007EEFAEFFB123DEBE4F590
:10F130000EF50F780E122B52AC0AAD0BEEFAEFFB68
:10F14000123DD37402122B80E96059AA0AAB0B124C
:10F150003D5B8A0E8B0FEA450F6046780E122B52EC
:10F16000780A122B527C007D00AA08AB09123DE5FB
:10F170007404122B80E9701D780E122B52780A123B
:10F180002B527C007D00EEFAEFFB123DDF7404127F
:10F190002B80E96003750C01AA0EAB0F123D618054
:10F1A00003750C10A90C02BEB174F71225809007EC
:10F1B000138008EAFEEBFF8A828B8312FC9CEA4BE9
:10F1C000603BEA2408F582E43BF583E014F070E349
:10F1D00012FE3AEA687002EB698A828B83700B1226
:10F1E000FE4312F912123D6180C412FE3D8E828FE1
:10F1F0008312F912123D618E828F8380BE12F785D1
:10F20000601AE0C812F77CE01412F774E0700D1277
:10F21000FC99123D61900715E4F0A3F090071312DA
:10F22000F788700512F78560269080F01229897A98
:10F23000087B00900719E0F9123E217404122B801C
:10F24000E9600C7A087B00900719E0F9123D017F14
:10F250000102280574F612258074FA122C2AEAF8A5
:10F26000EBF97E0088828983A3A3E0602B146034CD
:10F2700014603114603414602524F4603314700376
:10F2800002F35414700302F34E14700302F35A1481
:10F29000700302F39602F3E312397D02F3E51239AB
:10F2A0008302F3E512398902F3E512398F02F3E59F
:10F2B00088828983A3A3E0FFE82403F8500109882A
:10F2C000828983A3AA82AB8388828983E0606314E6
:10F2D000605514602F1470668A828B83A3A3E0F9B3
:10F2E0008A828B83E0FCA3E0FBECFA124721E96001
:10F2F000087403122E15E480077403122E1574018E
:10F30000F0E080328A828B83E0F912388DEA4B601C
:10F310000C124727851882851983E4802985188275
:10F320008519837401801F8A828B83E0F912471547
:10F33000800312471BE98518828519838008851888
:10F3400082851983740212FF53EFFA02F3DC12393B
:10F35000A102F3E51239A702F3E588828983A3A30A
:10F36000A3A3E0C0E07401122E15D0E012F96FA340
:10F37000A3A3A3E0C0E07402122E15D0E0F0740144
:10F38000122BEE88828983A3A3A3E0F91238BD1261
:10F39000FF4C7A1380469081547401122BF674024C
:10F3A000122AAE04122BEE88828983A3A3A3E0F96C
:10F3B0001238B77401122E15E0C0E07404122E1535
:10F3C000D0E0F07402122E15E0C0E07405122E1584
:10F3D000D0E0F07404122BF67B037A1479641239AE
:10F3E0005980020E0EEEF97406122B807F0202285D
:10F3F0000574F212258074FF122C2A8A088B0912D8
:10F40000F499F50A7A067B00123D5B8A0C8B0DAEEF
:10F410000CAF0DEE4F603F8E828F83A37419F0A363
:10F420007407F0EEFCEFFDE5082403FAE43509FB70
:10F4300012396BE9851882851983F0700FEEFAEFA7
:10F44000FB123857E9851882851983F0E06007EED2
:10F45000FAEFFB123D61AC18AD197B01AA0A796481
:10F460001239597401122B807F0602280574F71295
:10F47000258074FF122C2A12F499FE8A828B83A3B2
:10F48000A3A3E0F912385D12FF4CEEFA7964123949
:10F49000597401122B8002F24F85188285198374EA
:10F4A0001012F9862274EA12258074F2122C2A8B2B
:10F4B0000D851882851983740112F968E0F5128AA6
:10F4C000828B83A3A3E0F50FEA2403F50C50020519
:10F4D0000D7402650F7071850C82850D83E0F874E0
:10F4E0000A122E15E812F7567403687021850C086D
:10F4F000850D09750A007808122B4E7C087D007472
:10F5000005122BEE123C9B7403122B80800912F91A
:10F5100018122E1512F912E50C2408F50C500205EC
:10F520000DF582850D83E0C0E0740B122E15D0E03E
:10F5300012F756E0FAA3E0F9EAF8740C122E15124D
:10F54000F74A503A050D8036740A122E157402F0EF
:10F55000850C82850D8312F918122E1512F74A5068
:10F5600002050DF582850D83E0C0E0740B122E15A7
:10F57000D0E012F756740C122E15E4F0A3F0850CAF
:10F5800082850D83E0F912388D8A108B11850C82EB
:10F59000850D83A385820C85830D12F769F508E438
:10F5A00039F509E50C2402F50C5002050DF58285AC
:10F5B0000D83E0C0E07401122E15D0E012F760E078
:10F5C000F50BA3E0F50AA385820C85830D74026513
:10F5D0000F701A12F769FEE439FFEE2414F8E43FC5
:10F5E000F9E50C2402F50C5016050D8012E0FE7FA3
:10F5F00000A385820C85830D240AF8E43400F9E524
:10F600001045116011C3E894FBE99400500302F621
:10F61000EA12F785600B851882851983740202F758
:10F620002AEE2418FAE43FFB123D5B900715EAF03E
:10F63000A3EBF012F7858518828519837005741085
:10F6400002F72AE4F0900715E02418FAA3E034004A
:10F65000FB12FFACEAF0A3EBF07402122BE6880C6D
:10F66000890D750E00780C122B4E7C0C7D0012FF5C
:10F670005B123C9B7403122B8012FFA0E510F0A3D9
:10F68000E511F012FF94E508F0A3E509F012FF7F01
:10F69000EEF0A3EFF07401122E15E0C0E012FF8B24
:10F6A0002414F582E438F583D0E0F012FF73E50B03
:10F6B000F0900715E0F8A312FF68E50A12F77474DA
:10F6C0000FF09080F01229897A087B00900719E0EA
:10F6D000F9123E217404122B80E9604F7A087B00F6
:10F6E000900719E0F9123D018041780A122B5674F7
:10F6F00002122BE6881489157814122B52780C12FA
:10F700002B528E0C8F0D780C122B527808122B5224
:10F71000A90BAC10AD11740B122BEE12387B7409CF
:10F72000122B80E9851882851983F074E0551264E4
:10F7300020700DAC18AD197B01AA0F7964123959EC
:10F74000740E122B807F0E022805E8F0A3E9F0E585
:10F750000C2402F50C2212F76085820C85830D22A1
:10F76000F0850C82850D83A322E0FAA3E0F8E4C8BB
:10F77000F9EA2822F012FF8B12F77C222417F58277
:10F78000E438F58322900715E0F8A3E0F9E8492270
:10F7900074EC12258074F2122C2AEAFEEBFF851815
:10F7A00082851983740112F90BA3E0F50EEE240390
:10F7B000FE50010F7C0C7D0079007402122BEE12BA
:10F7C0003CA7740A122E157402F08E828F8312F9F0
:10F7D00018122E1512F912EE2402FE50010F8E821D
:10F7E0008F83E0C0E0740B122E15D0E012F90BE00D
:10F7F000F9A3AE82AF8312388D8A0A8B0B8E828F6B
:10F800008312FE54EE2402FE50010F8E828F83E09D
:10F81000C0E07401122E15D0E012F90BE0F50FA331
:10F82000E0F512A3E0F513A3AE82AF8325E0FAE47E
:10F8300033FB123D5B8A088B09EA4509700302F825
:10F84000EB7C00802412F76CE439FBEC25E0F8E453
:10F8500033F9E50828F582E50939F583EAF0A3EBE9
:10F86000F0EE2402FE50010F0CECC395138E828F34
:10F8700083E0FAA340CFAE82AF83E50A450B700A5E
:10F88000851882851983740280577808122B52E5F7
:10F8900013F5107810122B56E512F5107810122B74
:10F8A000567405122BE6881089117810122B528E8F
:10F8B000108F117810122B528A10751100781012C7
:10F8C0002B52780C122B52A90FAC0AAD0B740E12EE
:10F8D0002BEE123881740C122B80E9851882851961
:10F8E00083F0AA08AB09123D618009851882851949
:10F8F000837410F0AC18AD197B01AA0E796412392B
:10F9000059740E122B807F0C022805F08E828F8393
:10F91000A322E8F0A3E9F022E0FAA3E0F9EAF87400
:10F920000222C082C08374FD122C2A12F976C0E034
:10F930007401122E15D0E012F95DC0E07402122E8F
:10F9400015D0E0F0AC18AD197B037A8079441239F8
:10F95000597403122B80D083D082022B3212F962A9
:10F96000E02212F968A3A322F08A828B83A322F0FB
:10F9700088828983A3228A828B83A3E0851882856B
:10F98000198312F9862212F968A3E02274E912257C
:10F99000808A108B11EA242012FC2A12FE4CE50A00
:10F9A0002414F508E4350BF50975168175120075F8
:10F9B0001300EA12FC44E0F9EA241012FC2A12FCBB
:10F9C0009C124721E97017E510240E12FC2AE0640E
:10F9D00003600BC3E50894F1E5099400400E751629
:10F9E00082E508240AF508E43509F509C3E5089419
:10F9F000FBE50994004036E50A2409FAE4350BFBDF
:10FA0000123D5B8A128B13EA4513700302FC25EA50
:10FA10002409F8E43513F98A828B83A3A312F9121F
:10FA2000C3E508950AF508E509950BF509AA08ABA1
:10FA300009123D5B8A148B15EA45157010E51245D5
:10FA4000136007AA12AB13123D6102FC25AE14AF7E
:10FA500015E510240212FCAE240412FCA212FC8C48
:10FA600074826516705CE510240E12FC3612FC8C54
:10FA700088828983E064037025E5102406F50CE490
:10FA80003511F50D750E00780C122B4E7C087D009B
:10FA9000EEFAEFFB123C9B7403122B80800E12FCDB
:10FAA0003212FC8612F96F12FC86A3F0EE2408FED7
:10FAB00050010FE51012FC4412FCBE241012FCA2EF
:10FAC000800D12FC3212FC7C0E12FCB712FC4412A8
:10FAD000FCBE241412FC75AE82AF83E5102415120F
:10FAE000FC2A12FCBE241612FC2A12FCBE24191297
:10FAF000FC2A12FCBE241AFAE43511FB8A828B839D
:10FB0000780C122DBE12FC4E122DBEE50D8E828F8A
:10FB10008312FC54122DBE7410780C122BB512FCFB
:10FB20004E122DBE7418780C122BB58E828F83E581
:10FB30000CF0A30EAF8374826516700EE4F0A3E59B
:10FB40000AF0A3E50BF0A30E800BE510241F12FCB6
:10FB500075E50AF0A30E0EAF83E51245137003029C
:10FB6000FBE412FE3A85128285138312F912900784
:10FB700013E512F0A3E513F0851282F583A3A3A386
:10FB8000A3A3A3A3A3740FF09080F01229897A088D
:10FB90007B00900719E0F9123E217404122B80E9D2
:10FBA000600C7A087B00900719E0F9123D01E5101E
:10FBB000241A12FC2A122DF2851282851383A3A324
:10FBC000A3A3122DFE12FC60122B4EAC0AAD0B85C6
:10FBD0001282851383A3A312FC9C123C9B74031214
:10FBE0002B80801E12FC60122B4EAC0AAD0BEEFA7D
:10FBF000EFFB123C9B7403122B80EE250AFEEF35BF
:10FC00000BFFE510242412FCAE242612FC2A12FC61
:10FC100081AC14AD15AB08AA167944123959AA144F
:10FC2000AB15123D617F0F022805F582E43511F511
:10FC30008322E510240612FC3A22F8E43511F988F3
:10FC400082898322240FF582E43511F583228E8286
:10FC50008F83E50CF0A30EAF838A828B83780C220E
:10FC6000E5102422F582E43511F583E0F50CA3E0DC
:10FC7000F50D780C22F582E43511F58312FC81A391
:10FC80002212FC86F022E08E828F832212FC9022C8
:10FC900012FC86F0A30EAF8322900715E0FAA3E0D2
:10FCA000FB2212FC3A12FC9088828983A32212FC68
:10FCB0003A12FC81A3AE82AF8388828983A312FCAF
:10FCC00090E5102274EB1225808A088B09900713A7
:10FCD00012FE4C7A01751400E5082403F508500261
:10FCE0000509F582850983E0F50CE4F50DF50EF5BF
:10FCF0000FA3E0F510E4F511F512F5137408781070
:10FD0000122AEE780C7910122CF38508828509836B
:10FD1000A3A3E0F510E4F51174107810122AEE7820
:10FD20000C7910122CF3850882850983A3A3A3E024
:10FD3000F510E4F51274187810122AEE780C791088
:10FD4000122CF380078C828D8312FE4CE50A450B42
:10FD50006059AC0AAD0B8C828D83A3A3A3A3780C4E
:10FD6000122C5570E0E5082404F50850020509F549
:10FD70008285098312FE54850882850983A3A3E046
:10FD8000F514704512FE3AEC687002ED698C828DB4
:10FD900083700512FE43800712FE3D8C828D831214
:10FDA000F912AA0AAB0B123D617A00EA8508828536
:10FDB0000983F0A3E514F0AC08AD097B027A12794F
:10FDC000641239597F0D0228052402FAE43400FB3D
:10FDD000123D5B8A0E8B0FAE0EAF0FEE4F70077A9F
:10FDE0001075140080C58E828F83E4F0A3E514F0B3
:10FDF000850A82850B83A3A3E0250CF508A3E035D3
:10FE00000DF509750A007808122B4E851408AC0808
:10FE10007D00EE2402FAE43FFB123C9B7403122B9C
:10FE200080EEFCEFFD74022514FB7A12796412391E
:10FE300059EEFAEFFB123D61808A900713E0F8A3B8
:10FE4000E0F922E0F8A3E0F990071322E0F50AA315
:10FE5000E0F50B22E0FAA3E0F8E4C8F9EA28F50C93
:10FE6000E439F50D2274F512258074FF122C2A85D1
:10FE700018828519837401F0EA2403FA50010B8A71
:10FE8000828B83E0FCA3E0F8E4C8F9EC28FEE439B7
:10FE9000FF8A828B83A3A3E0FCEA2403FA50010BC0
:10FEA00012F785700B851882851983741002FF384C
:10FEB000EC705E12FF68E0F5087808122B56900788
:10FEC00015E02414F508A3E03400F5097808122B96
:10FED0005212FFAC12299112FF7F12299112FF9446
:10FEE00012299112FF73E0F912FFA0E0FCA3E0FDDC
:10FEF00012FF5B12387B7409122B80E9851882850A
:10FF00001983F012FC99123D61900715E4F0A3806B
:10FF1000278A088B09750A007808122B4E7D00127B
:10FF2000FFACE02EFAA3E03FFB123C9B7403122BC4
:10FF300080851882851983E412FF537A117964123F
:10FF400039597401122B807F03022805E985188234
:10FF5000851983F0AC18AD197B0122900715E024B8
:10FF600002FAA3E03400FB22E0C82416F582E4384C
:10FF7000F5832212FF8B2415F582E438F5832212D3
:10FF8000FF8B2412F582E438F58322900715E0F800
:10FF9000A3E0C82212FF8B2410F582E438F58322F7
:10FFA00012FF8B240EF582E438F58322900715E0CA
:10FFB000F8A3E0F5838882227401122B80D083D0CD
:10FFC00082022B327402F09070F9E0851882851954
:10FFD00083F075D1F775D608C28422C082C08374BD
:10FFE000FF122C2A901024E07013900902E06402A2
:10FFF00090102470057401F0800312FFC402FFB852
:020000040001F9
:10000000C082C0837900EA1282053BF583C082C0BA
:100010008390051012D3FFD083D082C3E09CA3E06D
:100020009D500CEA240B12805212803260010902AA
:10003000A37EEA75F00BA4FAA8F075F00BEBA428E8
:10004000FB900512E02AF8A3E03B8882F583E05498
:100050000F22F582E43B12B4F72274F7122580894F
:100060000812AB90A3E0F9E875F00BA4F8ACF075BA
:10007000F00BE9A42C1283B6E8FEE9FF74016508D1
:1000800060067402650870228A828B831286E2748D
:100090000265087021EA2403FA50010B122EA3E92D
:1000A00070148E828F83E4F0800CEA2403FCE43B1E
:1000B0001286D9122E9D8E828F83E0D2E7F0123FF6
:1000C0006B02A80974F412258012879C79008E8235
:1000D0008F83E06075890A890B8064E50A75F00BEF
:1000E000A4FAA8F075F00BE50B12803E7049E50A02
:1000F00075F00BA4F8AAF075F00BE50B12833A8E9D
:10010000828F83E085088285098312A1FC128659BB
:10011000EE2403FCE43F1281F8122E9D12A9CB12AB
:10012000BF281298EAD2E7F0123F6B7901900510D0
:10013000E0F50AA3E0F50B050AE50A7002050B12CB
:1001400085B5E50A9AE50B9B409102AE7E74F512E7
:100150002580EAFEEBFF750A01740B122E15129032
:10016000A9EC4D6015EC1282053D1287AA790112A7
:100170002E6DE508450960758023E5084509604452
:1001800012820335091287AA1281F9122EA3E9649B
:1001900001701BEEFAEFFB122E73E9F50A85088257
:1001A0008509831286517902AA08AB09801112864B
:1001B000DA122EA3E9640170347903EEFAEFFB1230
:1001C0002E6D80298E828F83A3E064FE7003A3E0EE
:1001D000F4700B1286DA122EA3E96401700CEEFAA9
:1001E000EFFB122E73E9F50A8003750A00028C14E6
:1001F000E50A2403FCE4350BFDE5082403FAE435A5
:1002000009FB22E50812C42E2274F71225809005FE
:100210001012AAE8EA4B602FEA75F00BA4FAA8F0D6
:1002200075F00BEBA428FBEAFEEBFF123D5B90059B
:100230001212AAE890051212B4E26012EEFCEFFD71
:100240007900123CA78007900512E4F0A3F002A801
:100250000974F6122580E4F508F5097808122B5286
:100260009005101290A475F00BA4FCA8F075F00B8B
:10027000EDA428FD7A237B00123DD37402122B805B
:10028000E9FE6003122E8BEEF9028B2774F612251D
:100290008074FF122C2A7E007F00803C85188285A6
:1002A0001983E4128E13122B527508017509007818
:1002B00008122B52EEFCEFFDEC75F00BA4FCA8F03D
:1002C00075F00BEDA428FD7A237B00123DDF74044A
:1002D000122B800EEE70010F1283C240BF74010218
:1002E0008B2474F61225807E007F008039EEF8EFB3
:1002F000F912832E7808122B5275080B75090078B5
:1003000008122B52EEFCEFFDEC75F00BA4FC75F01F
:100310000BEDA42AFD7A237B00123DE57404122B19
:10032000800EEE70010F1283C240C2028B27E87567
:10033000F00BA4F8AAF075F00BE9A42AF9900512C5
:10034000E028F508A3E039F5092274F61225807E2D
:10035000007F00804AEEF8EF1283A788828983E04D
:10036000A2E75036C2E7F085820885830978081233
:100370002B5275080B7509007808122B52EEFCEF12
:10038000FDEC75F00BA4FC75F00BEDA42AFD7A23AF
:100390007B00123DDF7404122B800EEE70010F12F1
:1003A00083C240B1028B27F9E875F00BA4F8AAF0DC
:1003B00075F00BE9A42AF9900512E028F8A3E039BA
:1003C000F92290051012A7F0C3EE98EF9922C0828F
:1003D000C083EC4D600512468B80097C087D007956
:1003E00000123CA702A37E74F61225807900EA4B26
:1003F00060177800EA28F582E412BC3F60047901B6
:10040000780808E8C3940840EB028B2774F712259C
:100410008074F3122C2AECFEEDFF85188285198377
:10042000E4F004122E15EAF0A3EB12A7E2122EC19B
:100430007403122E15AC82AD83EEFAEFFB122E9DE3
:10044000EEFAEFFB122EA302A80474F712258074B3
:10045000F3122C2AECFEEDFF851882851983E4F057
:10046000EAFCEBFD7403122E15AA82AB83122E9DBB
:10047000AA18AB19122EC77401122E1512A2098EDA
:10048000828F8312A7D374FE68700374FF696004BF
:1004900079018002790002A80474F7122580EAFE2F
:1004A000EBFF122E67E9F5087401650870111285DB
:1004B00002F4FA88828983E05A4480F0123F6B028A
:1004C000985F74F7122580EAFEEBFF7508008E82B4
:1004D0008F83E0602A122E67E9F5087401650870C1
:1004E0001E128502FA88828983E05A70128E828FEA
:1004F00083E04480FA88828983E04AF0123F6B02ED
:10050000985F12A9CF129A371283A78E828F83E049
:100510002274F41225808A088B097C007D00EA127F
:1005200081FB122E9DE5081286737900850882856D
:100530000983A3E064FE7003A3E0F460757E007F8E
:10054000008066EEFAEFFB1280326058EEFAEFFBA5
:10055000EA75F00BA4FAA8F075F00BEBA428FB9059
:100560000512E02AF50AA3E03BF50B850882850910
:1005700083A312BC1A850A82850B83A3E06A7003E9
:10058000A3E06B701FE50A2403FAE4350BFB122E7F
:10059000A3E9640170061281F0122E9D128668791B
:1005A0000112D2330EEE70010F1285B5EE9AEF9B59
:1005B000409102AE7E90051012B4F9C32274F3127A
:1005C00025808A088B098A828B83128651EA1286DB
:1005D00073750C00EA1281FB122EA3E96401706AA4
:1005E0007E007F00805FEEF8EFF9E875F00BA4F86D
:1005F000AAF075F00BE9A42AF990051212D2A5E031
:10060000540F603CEEF8EFF9E875F00BA4F8AAF08F
:1006100075F00BE9A42AF9900512E028F50AA3E089
:1006200039F50B1281F0124685E964017012850AD2
:1006300082850B83128659128668750C0112D2339B
:100640000EEE70010F1283C2409CA90C7F05022898
:1006500005A374FEF0A304F022A312A7F08508827C
:10066000850983A3129F0E22E50812867DEEF0A372
:10067000EFF02212867D74FEF0A304F02212C43241
:100680003509F5832274F5122580EAFEEBFF8E8290
:100690008F831286517C007D001286DA122E9DEE29
:1006A000FAEFFB122E67E9F50A7401650A7027124A
:1006B000A7E912832E850882F5831286E21281F95A
:1006C000122EA3E96401700EE5082403FCE4350949
:1006D0001286D9122E9D028C14FDEE2403FAE43FFB
:1006E000FB22A312BC24129F0E2274F212258074E6
:1006F000E6122C2A12879C750C01750800750900FA
:10070000750A00750B00851882851983E4F0EE24C4
:1007100003FCE43FFD7403122E15AA82AB83122E54
:100720009DAA18AB19122EC7E96401701F740B1231
:100730002E151287AC7401122E1512BC1E7003A365
:10074000E069604AA818A91988088909740D122E51
:100750001512A1FBA312A209740E122E1512A7D313
:10076000740D122BEE122EC1E964017009740D1282
:100770002BE6880A890B780A122B52AC08AD09EED9
:10078000FAEFFB122E797402122B80E9F50CEEFAC7
:10079000EFFB122EBBA90C741A02BB7AEAFEEBFF28
:1007A00012A9CF74FEF0A304F022F583129A37F950
:1007B00012A9CF129F0E22C082C0837800790080D8
:1007C0000508E87001091285B5E89AE99B5029E807
:1007D000FAE9FBEA75F00BA4FAACF075F00BEBA4A8
:1007E0002CFB900512E02AFCA3E03B8C82F583E011
:1007F000540F70CD79008002790102A37EC082C0BF
:1008000083904FE5E49375F016A4FCADF079FF7A80
:10081000237B0A123CA702A37E74F6122580EAF815
:100820007508007D008012ED12BC31C3994009E0CB
:10083000FAE8C39A400205080D904FE5E493FAEDFB
:10084000C39A40E3AA087B00028B2774F01225802C
:1008500074F3122C2A8A0C8B0D8C088D09890AECF2
:1008600045096016AA08AB09122F0F8A0E8B0FAE2E
:100870000EAF0FEE4F600302893E7B0080010B122A
:10088000BF1E500F1289E670F5742328FE740A39D2
:10089000FF80047E007F00EE4F7003028992904F2C
:1008A000C91289B960217403650A60067404650A77
:1008B00070157A047903122EE5904FE5E493FC90CD
:1008C0004FC91289BF5029904FC71289B960287447
:1008D00001650A60067402650A701C7A02790112C9
:1008E0002EE5904FE5E493FC904FC71289BF400777
:1008F0007A007B000289B68518828519837401F01D
:10090000122E15E50CF0A3E50DF0AC08AD0974034B
:10091000122E15AA82AB83122E9DAA18AB19122E85
:10092000D3740B122E15129F078E828F83A3A3A35D
:10093000A3A3A3E412D3FBAA0CAB0D12348B780053
:10094000E50A6007C39405500278048E828F83E520
:100950000CF0A3E50D12C9DFE50AF0E88E828F8363
:10096000A3A3A3A3A312BF2F5001097A027B0012F5
:10097000232312942AA312BB5AA312946EE50A6091
:100980000DC3940350081293F91289D7800312946F
:1009900010F07A047900122EE58A08904FE5E4936E
:1009A000FAC3E5089AEB94004005901028E4F01291
:1009B000335FEEFAEFFB028D721289CFE849221203
:1009C00089CFECC398F8E499F9C3EA98EB9922E44B
:1009D00093F8740193F922F9EE2414F582E43FF5BB
:1009E00083E8F0A3E922EB75F016A4F8A9F01294BD
:1009F00063F42274F212258074F3122C2A8A088B75
:100A000009ECFEEDFF750A00EEFAEFFB122F0F8ADC
:100A10000C8B0DA80CA90DE8497003028AB78882D7
:100A20008983E065087004A3E065097003028AB752
:100A300088828983A3A3A3A3E0C394055079888205
:100A4000898312C85F12AC4CE0603488828983A32A
:100A5000A3A3A3E0C394035026904FBFE493FA747A
:100A60000193FB12974C904FC1E493FA740193FBEE
:100A7000E82414F582E439F583EAF0A3EB800DE86D
:100A80002412128ABEF0E82414128ABEF08518825D
:100A90008519837401F0122E1512C85FF0EEFCEF79
:100AA000FD7403122E15AA82AB83122E9DAA18ABD9
:100AB00019122ED3750A01A90A740D02BB7AF582A8
:100AC000E439F58374FEF0A3042274F61225801233
:100AD0002F098A088B09A808A909E84960148882A7
:100AE0008983A3A3A3A3E06009C3940550047901FB
:100AF00080027900803174F6122580122F098A084D
:100B00008B09A808A909E849601488828983A3A3EE
:100B1000A3A3E06009C39403500479018002790023
:100B200080057402122B807F0202280574F61225BC
:100B300080122F098A828B83E5824583600BA3A3F1
:100B4000A3A3E0700479018002790080DAC082C03A
:100B500083EAFCEBFD7A007B0002A37BC082C083AA
:100B60007C007D0002A37B74F512258074F3122CA7
:100B70002AEAFEEBFF8C088D09C3EC94F8ED94FF94
:100B80004004EE4F606A750A00801974FF650870B2
:100B90000474FF6509600B12CB5C7004A3E0650967
:100BA000603B050A904FE5E493F8E50AC39850408E
:100BB000E50A1289E760EBEE4F60D0128BFB122E34
:100BC0001512A7DE122ECDE960D87403122E15ACD3
:100BD00082AD83EEFAEFFB124685E960C5E50A7542
:100BE000F016A4F8A9F0742328FA740A39FB8004DB
:100BF0007A007B00740D122B80801B85188285196A
:100C0000837401F0742528F582740A39F58312A7DC
:100C1000F0740B22A90A7F0302280574F4122580C0
:100C200074F3122C2A750800122F0F8A0A8B0BAE50
:100C30000AAF0BEE4F601F128C7E128C0E122E1517
:100C400012A7DE122EB57C167D0079FFEEFAEFFBBF
:100C5000123CA77508017A047900122EE58A0A90E1
:100C60004FE5E493FAC3E50A9AEB9400500990101B
:100C7000287401F012335FA908740D02AE7B851849
:100C8000828519837401F08E828F83A3A32274F767
:100C9000122580E9FC74FE6A700374FF6B7D00709E
:100CA00003802C0D128CF05026ED1289E760F412AF
:100CB000D6406A7003A3E06B70E98012ED75F01600
:100CC000A4F8A9F012D6336018E0640360130D1283
:100CD0008CF05015EC60E512945760F2C394055007
:100CE000ED12CDA012BC1780047AFE7BFF02A8098A
:100CF000904FE5E493F8EDC39822122F2102A37ED2
:100D0000C082C083790180F274F01225808A0A8B38
:100D10000B7A047901122EE58A0C8B0DEA450D60E1
:100D200040EA2AFAEB33FB123D5B8A088B09AE08D6
:100D3000AF09EE4F60267AFE7BFF122F2774FE6A02
:100D4000700374FF6B601E85088285098312AAE810
:100D5000E5082402F50850E2050980DE750C0080E4
:100D6000047E007F00850A82850B83E50C12AA1C95
:100D70008005740D122B807F08022805E493F8EC9F
:100D8000C3982274F6122580E4F508F50978081254
:100D90002B52904FE5E493F50874037808122D2C3C
:100DA000129096123DD37402122B80E9FE740A6EE3
:100DB0006024E4F508F5097808122B52904FE5E419
:100DC0009325E0FCE433FD7A3F7B00123DD37402AF
:100DD000122B80EE6003122F3902828774F61225DF
:100DE0008074FE122C2A851882851983E4F0A312E0
:100DF0008E13122B527508027509007808122B52B7
:100E00007C007D007A227B00123DDF7404122B806F
:100E1000028B22F0A818A919880889097808227479
:100E2000EE12258074E4122C2A8A0E8B0F8C088D0A
:100E300009750C007A227B00123DD98A0A8B0B7A45
:100E40003F7B00123DD98A108B11AE10AF11E50A1D
:100E5000450B6017E508650A7004E509650B600B32
:100E6000AC0AAD0B7A227B00123DEB7430122E15CA
:100E7000E0F50AA3E0F50BEE4F6015E50A6E70038E
:100E8000E50B6F600BEEFCEFFD7A3F7B00123DEB54
:100E9000E4F510F5117810122B52AC08AD097A2246
:100EA0007B00123DD37402122B80E9640A700302A6
:100EB000908CE4F508F5097808122B52AC0AAD0BBA
:100EC0007A3F7B00123DD37402122B80E9640A70D2
:100ED0000302908C7404122BE688088909780812A2
:100EE0002B527508027509007808122B527C007D80
:100EF000007A017B03123DE57404122B80E9600344
:100F000002908C851882851983E4F0A3F0FE02908C
:100F1000037406122BE6880889097808122B52758B
:100F200008087509007808122B528E087403780897
:100F3000122D2CE5082402FCE43509FD7A017B031F
:100F4000123DE57404122B80E9600302908C740852
:100F5000122E15E0F47003A3E0F470030290027403
:100F600006122BE6880889097808122B52750808A2
:100F70007509007808122B527404122E151290A9CC
:100F800074037808122D2C129096123DDF7404120F
:100F90002B80E9600302908C7402122BE68808898A
:100FA000097808122B527508027509007808122B6F
:100FB00052EE25E0FCE433FD7A027B03123DE5743A
:100FC00004122B80E970387402122BE68808890914
:100FD0007808122B527508027509007808122B52F6
:100FE0007404122E151290A42CFCED33FD7A3F7B75
:100FF00000123DDF7404122B80E9600302908C1212
:10100000955F0E851882851983C082C083904FE555
:10101000E493F8D083D082C3E098A3E094005021F9
:10102000851882851983C082C0837404122E15121C
:10103000A209D083D082C3E098A3E0995003028F25
:1010400011A818A919880889097808122B5275085F
:10105000027509007808122B527C007D007A227BF1
:1010600000123DDF7404122B80E97020AC0EAD0F2E
:101070007A017B03123DEBE97012742E122E1512C9
:10108000D3FF7A027B03123DEBE96003750C01A9E3
:101090000C741C02B143E5082402FCE43509FD7A16
:1010A000227B002212D403EC22E0F508A3E0F5092C
:1010B0002274EC12258074FE122C2A750A00851801
:1010C00082851983E4F0A3F0904FE593F510F508BD
:1010D00075090074037808122D2CE5082402F50820
:1010E00050020509E51025E0F510E433F5117A22E8
:1010F0007B00123DD98A0C8B0DAE0CAF0D7A3F7B75
:1011000000123DD98A0E8B0FA818A919880C890DD9
:10111000780C122B52750C02750D00780C122B52A4
:101120007C007D007A227B00123DE57404122B8046
:101130007A017B03123DD98A0C8B0D7A027B031254
:101140003DD98A128B13A812A913E50C450D700A1C
:10115000E5086E7003E5096F7025E849700CE5102D
:10116000650E7004E511650F7015E50C450D607B8B
:10117000EE4F604E85188285198312AAEE60437C7B
:10118000017D037A227B0012351BE9F8880A705B27
:101190007C027D037A3F7B0012351BE9F8880A70D8
:1011A0004AEEFCEFFD7A227B00123DEBE9700EACBB
:1011B0000EAD0F7A3F7B00123DEBE96011750A011D
:1011C0008029AE0CAF0DE8496004880E890F7810B5
:1011D000122B52780E122B52AC08AD09EEFAEFFB2F
:1011E000122F3F7404122B80E9F50AA90A74021227
:1011F0002B807F0C02280574F112258074D9122CE3
:101200002A7402122E15E4F0A3F0122F45E96003B0
:101210000293E87402122BE6880889097808122BD9
:10122000527508027509007808122B527C007D0067
:101230007A227B00123DE57404122B80E9600302E0
:1012400093E8904FE5E493FA7402122E1512A20966
:10125000C3EA98E49950030293E8750A00750B00FD
:10126000750800803E85188285198312BD0312CD52
:101270009312A7D3851882851983129A371289D7BA
:10128000F07A047900122EE58A0C904FE5E493FA87
:10129000C3E50C9AEB94004005901028E4F012335B
:1012A0005F0508904FE512BB3940030293E87402D2
:1012B000122E1512A209C3E50A98E50B9940030204
:1012C00093E87411122BE6880C890D780C122B52BE
:1012D000750C08750D00780C122B5285080C7403E0
:1012E000780C122D2CE50C2402FCE4350DFD7A223D
:1012F0007B00123DE57404122B80E970A474131274
:101300002E15E0F47003A3E0F46096050AE50A7078
:1013100002050B7404122E157401F07413122E15AD
:1013200012A209740F122E1512A7D37404122BEEF9
:10133000122ECDE970030292A112D3FC7411122E69
:101340001512BC1A12348BE50875F016A4F8A9F032
:10135000742328FE740A39FF7411122BE6880C8955
:101360000D750E00780C122B4E7C087D00EEFAEF06
:10137000FB123C9B7403122B8012BF345001097A7C
:10138000027B0012232312942A12946EA818A91922
:10139000880C890D780C122B52750C02750D007893
:1013A0000C122B52AC08EC2CFCE433FD7A3F7B0092
:1013B000123DE57404122B80E960030292818518C6
:1013C00082851983E0F47003A3E0F4600302926560
:1013D000E508129458600BC3940350061293F90267
:1013E000927D1294100292807402122E15E0F9740C
:1013F00027122B807F07022805904FBF1289CFEE5E
:1014000012CD97129F0E904FC1E493F8740193226E
:10141000EE241212941EF0EE241412941E22F58271
:10142000E43FF58374FEF0A30422E88E828F83A349
:10143000A3A3A3A3A3A3A312944F740112944FA335
:1014400074AAF0EE2410F582E43FF583E4F0221252
:10145000CA02A3A3A3A322ED75F016A4F8A9F01263
:10146000946322742728F582740A12D4EF22A3F021
:1014700012A9CFE4F0EE240CF582E43FF583E4F00A
:10148000A3F0A3F0A3F02274F312258074FE122CB3
:101490002A851882851983E4F0A3F0F50C029520C3
:1014A000E50C75F016A4F8A9F0742328F50A740A5F
:1014B00039F50B850C82AE82780A122B527508081A
:1014C0007509007808122B528E0874037808122DC3
:1014D0002C129096123DDF7404122B80E50A24141E
:1014E000F508E4350BF5097808122B5275080275DA
:1014F00009007808122B52EE2EFEE433FFEEFCEFCB
:10150000FD7A3F7B00123DDF7404122B80850A8236
:10151000850B83A3A3A3A3E0F4600312955F050CDE
:10152000904FE5E493F8E50CC39850030294A0A80B
:1015300018A919880889097808122B5275080275AC
:1015400009007808122B527C007D007A227B001261
:101550003DDF7404122B807402122B8002864C85AE
:101560001882851983E02401F0A3E03400F022C042
:1015700082C0837D008009EA24FF1AEB34FFFB0D53
:10158000128CF05016129457C3940550F2EA4B7027
:10159000E6742328FA740A39FB80047A007B00027F
:1015A000A37E74F712258074F3122C2A7E00029613
:1015B0003AEF75F017A4F8A9F012D61612BD00750F
:1015C000F016A4FAABF074232AF582740A12BF5203
:1015D0007003A3E0696040EF75F017A4F8AAF0EA81
:1015E000F912D61639F58312A2097401122E15E0EC
:1015F000687003A3E069601FEF75F017A4F8EAF9BB
:1016000074F328FC740B39FD7403122E15AA82ABF7
:1016100083124685E96013EF75F017A4F8A9F074FA
:10162000F128FA740B39FB1234970F904FD1E493E1
:10163000F8EFC39850030295B10E904FE512D18593
:10164000501FEE12D639F47003A3E0F460EB128B56
:10165000FB122E1512A7DE122ECDE960DC7F008072
:10166000CA02A80474F712258074F3122C2A90057C
:10167000E312B4E27003029710750800802BE508AE
:1016800075F016A4F8EAF9743728F582740A12D4B2
:10169000EB64FE7003A3E0F4600D743528F58274EA
:1016A0000A39F58312BB700508904FE512BB39501B
:1016B0005FE50875F016A4F8AAF0EAF912945F60E5
:1016C000E6C3940350E1743528F582740A12B4DF3E
:1016D00070ACE50875F016A4F8EAF9742328F874DC
:1016E0000A39F9E8FEE9FF1297AE1297A4122766AD
:1016F000128C7E128C0E122E1512A7DE122ECDE940
:1017000060A57403122E15AA82AB83122F1B80973B
:1017100002A80474F6122580122F098A088B09A8E2
:1017200008A909E849602088828983A3A3A3A3E0CC
:101730006011C39403500CE82414F582E412BC1722
:1017400012974C790180027900028B27E82412F568
:1017500082E439F583EAF0A3EBF02274F7122580D6
:10176000EAFEEBFF9005DD12B4E260309005E31273
:10177000B4E260289005E712B4E2602012CEE112D4
:101780002766E9701712979F122766E96401700CAB
:101790008E828F83A3A312CECE12276602A80912CF
:1017A00097AEA3A312B4F99005E312CED822904FBE
:1017B000C1E493FC740193FD8E828F8322C082C0AA
:1017C00083900519741BF0A37432F090051B7415F7
:1017D000F0A37432F090051F7411F0A37430F0027E
:1017E000A37EC082C08390051D740FF0A37432F0F5
:1017F00002A37E74F7122580EAFEEBFF900553E00A
:101800006408601CE0640460178E828F83E05403D8
:101810006401704112B8D2F8129864E06406703521
:101820008E828F83A3A3E064FE7003A3E0F460259F
:101830008E828F83A3A312C4147003A3E06970087F
:10184000EE241512C40960051232DB80031232E166
:10185000E9F50880037508C2EEFAEFFB123D61A9B5
:101860000802A809A3E0F58388822274F412258077
:101870008A088B09129A33FAE82AFAE43400FB1238
:101880003D5B8A0A8B0BAE0AAF0BEE4F60558508A5
:1018900082850983E0FC7D007900123CA78E828F4F
:1018A00083A31286511233178E828F83A3A3A3A31F
:1018B000EAF0A3EB1298EAF8EE28F8E43F1287AFBB
:1018C000850882850983A3E0C0E012BF14D0E0F050
:1018D00012332912BF0AE9129EEAE0C0E0129EE02C
:1018E000D0E0F0EEFAEFFB02AE7EF08508828509CB
:1018F00083E02274F412258074E8122C2A8A088B63
:10190000098C0A8D0BE9FE900553E064046005E044
:101910006408700479C2803CA37808122DAFEE9061
:10192000055A129B76123CA7851882851983780880
:10193000122DAF7405122E15EEF07404122E1574CC
:1019400001F07407122E15E4F0900553740212A7EB
:10195000E212482F02AE7974F412258074E8122C3A
:101960002AEAFEEBFF90051412B4E26003029A2EFD
:101970007A077B00123D5B90051412AAE8900514CB
:1019800012B4E27003029A2A8E828F83122DF29093
:101990000514E0FCA3E0F5838C82122DFEEE2404F6
:1019A000F50AE43FF50B850A82F583E0C0E0900577
:1019B0001412B4B6A3A3A3D0E0F0EE2405F508E416
:1019C0003FF509850882F583E0C0E090051412B464
:1019D000C4D0E012A7D8C0E0900514129A37C824EA
:1019E00006F582E438F583D0E0129B76123CA78E90
:1019F000828F83122DF2851882851983122DFE8520
:101A00000A82850B83E0C0E07405122E15D0E01227
:101A100098EAC0E07404122E15D0E0F07407122E7C
:101A200015E412A7E212482F80067910800279018E
:101A300002AE798A828B83E0F8A3E022C082C08361
:101A400090051412B4E2601090051412BC1A123DF5
:101A500061900514E4F0A3F012324512343702A36A
:101A60007E74F412258074E8122C2A8A0A8B0BECFF
:101A7000FEEDFF89087428122E15E0FC7429122E41
:101A800015E0FD740F6C7005740F6D60129010936B
:101A9000E064026005ECC39D500579C1029B73743C
:101AA00024122E15122DF2900554122DFEE50890E9
:101AB000055AF0EC900558F0EDA3F0742A122E159B
:101AC000E090055BF074FF650A700474FF650B70AD
:101AD000249010A7E0F47003A3E0F4700C123CB95A
:101AE000900551EAF0A3EB80129010A712CDBDE84B
:101AF000F0A3E9800690055112BF28F0EE4F601761
:101B0000EEFAEFFB1234EBE96401700BEEFCEFFD33
:101B10007A657B0512468B900544E4F0A3F09005AE
:101B200047F0A3F0900564F0901093E06402700811
:101B3000900558740FF0A3F09005537405129B762E
:101B4000123CA77404122E15E4F0900554122DF2E5
:101B5000851882851983122DFE90055AE0C0E07425
:101B600005122E15D0E0F07407122E15E412A7E22C
:101B700012482F02AE79F07C187D007900AA18ABCC
:101B8000192274F7122580E9900518F07A807B00FD
:101B900090059EE0F9123E2D122FB1790002A8099E
:101BA000C082C083900518E070031240AF122FB1BD
:101BB00002A37E74F0122580900518E09010277023
:101BC0000FE060057900123F2F901027E4F0804A63
:101BD000E064016008900518E0F9123F2F9010278B
:101BE0007401F0900518E0F46030E0F50CE4F50DB8
